:100000000C94E90D0C9400000C9400000C9400007A
:100010000C9400000C9400000C9400000C947C578D
:100020000C9400000C9400000C948D150C940000AE
:100030000C9400000C9400000C9400000C94000040
:100040000C9458150C9400000C9456550C94000018
:100050000C9472550C9400000C9400000C94000059
:100060000C9400000C9400000C9400000C94000010
:100070000C9400000C9400000C94DB550C940000D0
:100080000C941B570C9400000C940000000001001D
:100090000200040008001000200040008000000161
:1000A0000002000400080010002000400080000151
:1000B00002040810204080000C03780B8010000020
:1000C0001003780B821F00001A03780B81030000D5
:1000D0002203780B010402002C03790B01060200B5
:1000E00036037B0B018000004203820B020F0000ED
:1000F0004A037C0B020F000052037E0B020FD0124A
:100100005A03800B011000006403D00B01100000A3
:100110006E03810B000100007603840B01080100CF
:100120008003850B030801008E03860B0307000084
:1001300096039C0B017F3F00A0039B0B0104000072
:10014000AA03870B03040000B2039A0B01641E008C
:10015000BE03880B00010000CA03890B00010000E8
:10016000D603990B01020000E2038A0B0001000094
:10017000F0038B0B020F0000FC038D0B020FE70353
:100180000604CF0B016300006404D10B01100000D2
:100190006E04D20B0102020012048F0B030801004F
:1001A0001804900B030800001E04910B03080000C4
:1001B0002404920B030800002A04930B0308000098
:1001C0003004940B030800003604950B030800006C
:1001D0003C049D0B040A2E004404A70B040A2E00C5
:1001E0004C04B10B040A2E005404BB0B040A2E006D
:1001F0005C04C50B040A2E0000000000FF00000094
:10020000760400027E040404840408078A040C05B2
:100210008A048C06900480099804100BA004500CEA
:10022000AA044003B204140ABC041808C4041C0144
:100230000000000200002A0054007F00800E5631AA
:1002400000810E563200820E5633000031000B0042
:100250003120414243000032000B00322044454629
:10026000000033000B003320474849000043000CD6
:10027000004300000000000034000B0034204A4B13
:100280004C000035000B0035204D4E4F000036006D
:100290000B003620505152000030000B003020205F
:1002A0002E202C0037000B00372053545500003807
:1002B000000B003820565758000039000B00392039
:1002C000595A2F00003D000A004352000000000070
:1002D000706F7274696F6E696572656E00002E666C
:1002E0006F6C67650000506F7274696F6E656E2089
:1002F0007369636865726E0050726F64756B742009
:100300000000537061727465202000005F49440052
:100310005F5273323332494400005F526F7461742C
:1003200065005F54617374656E5800005F546173BB
:1003300074656E5900005F44656661756C744B6549
:1003400079002A436F64653000002A436F64653189
:1003500000002A436F64653200002A4D61784D6FBA
:1003600064756C005F4572774D6F64756C002A543C
:100370006973636845005F4D795465726D4E720014
:100380005F4D61737465725465726D7300005F45F3
:100390004D6F646500005F45437265645774720079
:1003A0005F5273304D6F646500005F5634756E6444
:1003B00035005F50756C736554696D6500005F4171
:1003C000736B43726564697400005F53656E6444C7
:1003D0006562697400005F4372656469744D6F649F
:1003E00065005F4372656469744D61737465720082
:1003F0002A5461626C655374617274002A5461629C
:100400006C65456E64002A4669727374426F6E5063
:1004100000002A4A6F6231002A4A6F6232002A4A7B
:100420006F6233002A4A6F6234002A4A6F623500D5
:100430002A4A6F6236002A4A6F6237005F4572723D
:100440006F7231005F4572726F7232005F45727277
:100450006F7233005F4572726F7234005F45727263
:100460006F7235005F4672656967616265005F4B58
:100470006F6D6D61000054617374657200004C69AA
:10048000745A00004C656974540050756C73000018
:10049000546173742030000073657269656C6C0080
:1004A00073657269656C2032000054617374203288
:1004B000000054617374207061720000466F6C67B5
:1004C000655400005377697463680000436865668B
:1004D0002D4D656E75004B206C697374656E000060
:1004E0004B206C6F65736368656E00004B2064720F
:1004F00075636B656E0054206C697374656E0000E3
:1005000054206C6F65736368656E000054206472DC
:1005100075636B656E0053797374656D0000506F81
:100520007274696F6E004B726564697465004B721A
:1005300065642E436C7200006D616E2E506F727494
:10054000696F6E00546573740000506172616D656F
:100550007465720050726F64756B746500004B6552
:100560006C6C6E65720056656E74696C6500436FE5
:100570006C6F7273000030CC0431D60432E0043367
:10058000EC0434F604350005360C05461605411E0C
:1005900005432605442E054A3805000000003016A4
:1005A00005374405394A05385405425E0545660558
:1005B000636E050000004572726F72004F70742EFA
:1005C0000000496D70756C73000054696D656F753E
:1005D0007400B605E60B00030000BC05E90B000340
:1005E0000000C205E70B00030000CA05E80B001479
:1005F00000002E202C3041424331444546324748CA
:1006000049334A4B4C344D4E4F355051523653546A
:10061000553756575838595A2F390500C11100001F
:100620000300D90B00000300C1110300170E0300E3
:10063000D90B00000500E00800000A00C1110A0003
:10064000170E0A00D90B0A00C1110A00170E280064
:10065000D90B000000000F00E003EF0300780F78D3
:10066000E07BEF7BF7BD1F00E007FF0700F81FF8F6
:10067000E0FFFFFF0000000000000000000000009D
:10068000000000000000000000000000000000006A
:1006900000000000070018C0202020204D904D9041
:1006A00040104010489047102020202018C007001C
:1006B0000000000007001FC03FE03FE07270727052
:1006C0007FF07FF0777078F03FE03FE01FC00700D9
:1006D0000000000000000000000018C03DE03FE006
:1006E0003FE03FE01FC00F80070002000000000055
:1006F00000000000000000000000020007000F8062
:100700001FC03FE01FC00F80070002000000000074
:10071000000000000000000007000F800F800F8025
:1007200037607FF07FF07FF0326007000F800000BD
:1007300000000000000000000200020007000F801F
:100740001FC03FE03FE03FE01AC007000F800000FD
:100750000000000000000000000000000000000099
:1007600006000F000F00060000000000000000005F
:1007700000000000FFF0FFF0FFF0FFF0FFF0FFF0DF
:10078000F9F0F0F0F0F0F9F0FFF0FFF0FFF0FFF01B
:10079000FFF0FFF00000000000000000060009006C
:1007A00010801080108010800900060000000000FA
:1007B00000000000FFF0FFF0FFF0FFF0F9F0F6F0AE
:1007C000EF70EF70EF70EF70F6F0F9F0FFF0FFF000
:1007D000FFF0FFF000000000000001E000601EA03C
:1007E000332061806180618033001E0000000000C2
:1007F000000000000000000007800CC018601860B6
:1008000018600CC00780030003000FC00300030042
:100810000000000002000300038003C002C002C009
:100820000280020002000E001E001E000C000000EC
:10083000000000000C000E000B0009800CC00E40F0
:100840000B4009C038C07840784031C003C003C0B5
:100850000180000000000200020027201FC018C015
:1008600030607070306018C01FC027200200020086
:100870000000000000000000100018001C001E0016
:100880001F001F801F001E001C0018001000000029
:10089000000000000000000000800180038007804D
:1008A0000F801F800F800780038001800080000080
:1008B000000000000000020007000F801FC00200BF
:1008C00002000200020002001FC00F8007000200A9
:1008D000000000000000198019801980198019801B
:1008E00019801980198019801980000019801980D9
:1008F0000000000000001FE036C066C066C066C091
:1009000036C01EC006C006C006C006C006C006C06F
:100910000000000000001F8030C0300030001F8049
:1009200030C030C01F8000C000C030C01F80000039
:1009300000000000000000000000000000000000B7
:10094000000000000000000000001FE01FE01FE0AA
:1009500000000000020007000F801FC0020002001C
:1009600002000200020002001FC00F800700020008
:100970001FC000000000020007000F801FC002001F
:100980000200020002000200020002000200020057
:10099000000000000000020002000200020002004D
:1009A00002000200020002001FC00F8007000200C8
:1009B00000000000000000000000000001000180B5
:1009C00001C03FE001C00180010000000000000004
:1009D00000000000000000000000000004000C0007
:1009E0001C003FE01C000C000400000000000000A0
:1009F00000000000000000000000000000000000F7
:100A000000000000400040004000400040007FE047
:100A1000000000000000000000000000088018C076
:100A200038E07FF038E018C00880000000000000C7
:100A300000000000000000000000000000000200B4
:100A400007000F801FC03FE07FF0000000000000A3
:100A500000000000000000000000000000007FF027
:100A60003FE01FC00F8007000200000000000000F0
:100A70000000000000000000000000000000000076
:100A80000000000000000000000000000000000066
:100A900000000000060006000F000F000F000F000E
:100AA0000F00060006000600000000000600060019
:100AB00000000000000000001980198019801980D2
:100AC0000000000000000000000000000000000026
:100AD0000000000000000660066006603FF00CC0E9
:100AE0000CC0198019807FC0330033003300000030
:100AF00000000000060006001F803FC036003600E0
:100B00003F801FC006C006C03FC01F800600060011
:100B1000000000000000000000103830387038E09D
:100B200001C0038007000E001C0038E070E060E0A8
:100B300000000000000007000D80198019801B00D4
:100B40000E001E003E00336033C031803BC01E608B
:100B5000000000000E000E000E00060006000C0053
:100B60000000000000000000000000000000000085
:100B700000000000038006000E000C001C001C009A
:100B80001C001C001C001C000C000E000600038052
:100B9000000000001C000600070003000380038023
:100BA00003800380038003800300070006001C000D
:100BB0000000000000000000000036C036C01F80AA
:100BC0000F003FC00F001F8036C036C0000000007D
:100BD0000000000000000000000000000600060009
:100BE00006003FC03FC006000600060000000000EF
:100BF00000000000000000000000000000000000F5
:100C0000000000000000000000000E000E000E00BA
:100C100006000C00000000000000000000000000C2
:100C200000003FC03FC000000000000000000000C6
:100C300000000000000000000000000000000000B4
:100C4000000000000000000000000E000E000E007A
:100C500000000000000000100030007000E001C043
:100C6000038007000E001C003800700060000000C8
:100C7000000000000F803FE03060607060F061B005
:100C8000633066306C307830703030603FE00F8019
:100C900000000000030007001F001F000300030006
:100CA0000300030003000300030003001FE01FE034
:100CB000000000001FC03FE070706030607000E016
:100CC00001C0038007000E001C0038007FF07FF099
:100CD000000000001FC03FE0707060300030007006
:100CE0000FE00FC000600030603070703FE01FC048
:100CF0000000000001C003C007C00EC01CC038C007
:100D000070C060C07FF07FF000C000C000C000C0B5
:100D1000000000007FF07FF06000600060007FC096
:100D20003FE0007000300030603070703FE01FC066
:100D30000000000003C007C00E001C003800300097
:100D40007FC07FE070706030603070703FE01FC027
:100D5000000000007FF07FF00060006000C000C075
:100D60000180018003000300060006000C000C0057
:100D7000000000000F801FC038E03060306038E0B5
:100D80001FC03FE070706030603070703FE01FC087
:100D9000000000001FC03FE0707060306030707075
:100DA0003FF01FF0006000E001C003801F001E0044
:100DB0000000000000000000000000000E000E0017
:100DC0000E000000000000000E000E000E000000EB
:100DD0000000000000000000000000000E000E00F7
:100DE0000E000000000000000E000E000E000600C5
:100DF00006000C0000C001C0038007000E001C00AC
:100E0000380038001C000E000700038001C000C03D
:100E100000000000000000000000000000003FE0B3
:100E20003FE0000000003FE03FE000000000000065
:100E300000000000300038001C000E000700038096
:100E400001C001C0038007000E001C003800300004
:100E5000000000001F803FC070E0606060E001C0E3
:100E600003800700060006000600000006000600DA
:100E7000000000001FC03FE0306067B06FB06DB091
:100E80006DB06DB06DB06FE067C070003FC00FC057
:100E900000000000060006000F000F000F00198080
:100EA0001980198030C03FC03FC0606060606060E2
:100EB000000000007F007F8061C060C060C061C032
:100EC0007F807FC060E06060606060E07FC07F80A6
:100ED000000000000F801FC038E03060600060003C
:100EE0006000600060006000306038E01FC00F806C
:100EF000000000007F007F8061C060C060606060B3
:100F0000606060606060606060C061C07F807F0022
:100F1000000000007FE07FE0600060006000600093
:100F20007F807F8060006000600060007FE07FE085
:100F3000000000007FE07FE0600060006000600073
:100F40007F807F8060006000600060006000600063
:100F5000000000000FC01FE038603000600060003B
:100F600063E063E060606060306038601FE00FE065
:100F700000000000606060606060606060606060F1
:100F80007FE07FE060606060606060606060606023
:100F9000000000001F801F800600060006000600FB
:100FA0000600060006000600060006001F801F80DF
:100FB00000000000006000600060006000600060F1
:100FC0000060006000606060606070C03FC01F80B3
:100FD00000000000606060E061C0638067006E0038
:100FE0007C007C006E006700638061C060E0606030
:100FF00000000000600060006000600060006000B1
:101000006000600060006000600060007FE07FE0E2
:1010100000000000606070E070E079E079E06F60EF
:101020006F606660666060606060606060606060A5
:101030000000000060607060706078606C606C60E0
:10104000666066606360636061E060E060E060600D
:10105000000000000F001F8039C030C06060606079
:10106000606060606060606030C039C01F800F00E9
:10107000000000007F807FC060E0606060606060B2
:1010800060E07FC07F806000600060006000600002
:10109000000000000F001F8039C030C06060606039
:1010A000606060606060636033C039C01FE00F60E3
:1010B000000000007F807FC060E060606060606072
:1010C00060E07FC07F806700638061C060E0606037
:1010D000000000001F803FC070E060606000700092
:1010E0003F801FC000E00060606070E03FC01F8074
:1010F000000000003FC03FC00600060006000600DA
:1011000006000600060006000600060006000600AF
:10111000000000006060606060606060606060604F
:101120006060606060606060606030C03FC01F8071
:101130000000000060606060606030C030C030C09F
:101140001980198019800F000F000F00060006009B
:10115000000000006060606060606060606060600F
:101160006060666066606F6079E070E070E06060AB
:10117000000000006060606030C030C019800F0067
:10118000060006000F00198030C030C0606060604B
:10119000000000006060606030C030C019801980BD
:1011A0000F000F00060006000600060006000600FD
:1011B000000000007FE07FE000C000C0018003006D
:1011C000060006000C001800300030007FE07FE0D1
:1011D00000000000666066600F000F000F001980BD
:1011E0001980198030C03FC03FC06060606060609F
:1011F000000000006F605FA039C030C060606060B8
:10120000606060606060606030C039C01F800F0047
:10121000000000006060606000006060606060600E
:101220006060606060606060606030C03FC01F8070
:10123000000000001F801F80180018001800180010
:101240001800180018001800180018001F801F80D0
:10125000000000000000000000000000000000008E
:10126000000000000000000000000000000000007E
:101270007FF07FF00000070007000700060006006F
:10128000030000000000000000000000000000005B
:1012900000000000000000000000000000001FC06F
:1012A0003FE000601FE03FE0606060607FE03FE0A3
:1012B00000000000600060006000600060006F805F
:1012C0007FC070E060606060606060E07FC07F80D1
:1012D00000000000000000000000000000001F806F
:1012E0003FC0706060006000600070603FC01F80A1
:1012F00000000000006000600060006000601F608F
:101300003FE071E060606060606070603FE01FE03F
:1013100000000000000000000000000000001F802E
:101320003FC070607FE07FC0600070003FC01F80E2
:101330000000000007800F801C0018001800180033
:101340007F007F001800180018001800180018000F
:1013500000000000000000000000000000001FE08E
:101360003FE07060606070E03FE01F60006000E0A0
:101370003FC03F80600060006000600060006F0060
:101380007F8071C060C060C060C060C060C060C06D
:1013900000000000000000000600060000000E0033
:1013A0000E00060006000600060006001F801F80D3
:1013B00000000000000000000180018000000380A8
:1013C00003800180018001800180018001801980FB
:1013D0001F800F00300030003000300030003180BE
:1013E000338037003E003E003700338031C030C0CC
:1013F000000000000E000E000600060006000600B9
:101400000600060006000600060006001F801F807A
:1014100000000000000000000000000000005980F3
:101420007FC07FE06660666066606660666066607A
:1014300000000000000000000000000000003F80ED
:101440003FC030E03060306030603060306030602D
:1014500000000000000000000000000000001F80ED
:101460003FC070E060606060606070E03FC01F80FF
:1014700000000000000000000000000000007F806D
:101480007FC060E06060606070E07FC06F8060007F
:1014900060006000000000000000000000001FE08D
:1014A0003FE070606060606070E03FE01F6000607F
:1014B000006000600000000000000000000037C075
:1014C0003FE0386030003000300030003000300045
:1014D00000000000000000000000000000003F00CD
:1014E0007F8060007F003F80018001807F803F001F
:1014F00000000000000018001800180018007F000D
:101500007F00180018001800180018001F800F80B6
:10151000000000000000000000000000000060600B
:101520006060606060606060606070E03FE01F600D
:1015300000000000000000000000000000006060EB
:10154000606030C030C0198019800F000F000600A5
:1015500000000000000000000000000000006660C5
:1015600066606660666066606F603FC039C010800C
:10157000000000000000000000000000000060C04B
:1015800071C03B801F000E001F003B8071C060C017
:10159000000000000000000000000000000030C05B
:1015A00030C0198019800F000F00060006000C00E3
:1015B0000C001800000000000000000000007FC0C8
:1015C0007F80030006000C00180030007FC07FC041
:1015D00000000000000000006060000000001FC06C
:1015E0003FE000601FE03FE0606060607FE03FE060
:1015F00000000000000000006060000000001F808C
:101600003FC070E060606060606070E03FC01F805D
:10161000000000000000000060600000000060604A
:101620006060606060606060606070E03FE01F600C
:101630000000000000003F007F8060C060C061C00B
:10164000678067C060E06060606060E067C067807E
:1016500000000000000000000000000006000F0075
:10166000198030C0606060607FE07FE000000000B3
:10167000000000000000F8000000FF000000FF0074
:1016800000007F80001E0F80007FE7C0007FFFE02A
:10169000003FFFE00007FFC00001FFC00001FF8026
:1016A0000001FF0003FFFE0007FFFC0007FFF00042
:1016B00003FFF00003FFFE00001FFFC001FFFFF06B
:1016C00001FFFFF801FFFFF8007FFFF80007FE00B1
:1016D000003FFF00007FFF80007FFF80007FC10090
:1016E000001FE000001FF000001FF000000FE000EE
:1016F0000007C0000007C0000007C000000780000E
:1017000000030000000300000002000000000000D1
:10171000000000000000E000000000000003900056
:1017200000000000000E1800000000000038080053
:101730000000000000C018000000000003807000DE
:10174000000000000C01C00000018006300700000E
:101750000003C00F401C00000006E01DC070000028
:10176000000C3039C1C0000000181871C718000003
:10177000001C0CE1DC7C0000000E07C3F1C400007B
:1017800000070386070600000003800E1C0200000D
:101790000001C01C300300000000E0381801008088
:1017A000000070700FC183C0000038E003E08E605D
:1017B00006001DC00020FC200F000F80003070309C
:1017C000198007000010003030C00000001800E051
:1017D000606000000008038060300000000C0E0014
:1017E0003018000000043800180C00000006E0006B
:1017F0000C0600000003800006030000000000004B
:1018000003018000000000000180C0000000000013
:1018100000C0C000000000000060C0000000000028
:101820000030C000000000000030C00000000000D8
:101830000030C000000000000030C00000000000C8
:101840000030C000000000000030C00000000000B8
:101850000030C000000000000030C00000000000A8
:101860000030C000000000000030E0000000000078
:101870000030700000000000003018000000000080
:1018800000300C00000000000030040000000000E8
:10189000003FFC0000000000003FFC0054696E792E
:1018A0002062616400507772552000424F757420A9
:1018B0000057646F672000454570726F6D20006CA3
:1018C0007C736368656E203F0058006E65696E002A
:1018D0006A61003E3E006B65696E204B726564690B
:1018E0007400546573740020204B653A0020204931
:1018F0006E3A0043616C6962726174696F6E004F89
:101900004B00567320312E353200546F74616C20B9
:10191000002D2D2D2D006B65696E20454570726F71
:101920006D006E6F20546F75636800496E6974694D
:10193000616C697A65640049442000540000666166
:101940006C7363686572205469736368200054691E
:1019500073636820766F6E204B20004665686C6567
:1019600072200056656E74696C20616B7469760034
:1019700054696D656F757400435349204E722000A1
:10198000436F646520006B65696E204B7265646906
:10199000740066616C736368657220546973636870
:1019A00000546973636820766F6E204B005831399C
:1019B0003931303000504C5520203A00436F646577
:1019C000203A005469736368203A004D4200505336
:1019D000004D31004F310053500043500044590036
:1019E00062757379004D500020676573706572727F
:1019F000740025640000533F000041627265636813
:101A00006E756E67004B656C6C6E65722000546F6E
:101A100074616C004D6F64756C2000202000433FA2
:101A20000073656300496D7000504C553A200053B7
:101A300070617274653A20005072313A2000507221
:101A4000323A200046756E6374203A200054797053
:101A50003A20003A20563A2020302B2030003A001D
:101A60003A20544F3A20003A2050733A20005370E5
:101A70003A004B204D6F6465204A6F62204A6F62C6
:101A8000466C616773004B20004D6F646520004A0F
:101A90006F62202000562020204572722050676C13
:101AA00020496D7020544F005620005061757365B9
:101AB000004B656C6C6E65723A004D49004D4200FA
:101AC0004D43004D50004D4C0074657374202E2E14
:101AD000004F4E004B23004253004221004246007B
:101AE000542300544F004952004D5A0042510042C5
:101AF0005200435300565300564300494C0042667F
:101B00000000253032580025303458002536640056
:101B10002533642E253032640025356400256400A9
:101B20002532640025336400444400004B230054F4
:101B300023004245004345004241004453004342D4
:101B40000023502241534349492D492F4F222C2233
:101B5000312E3030222C323030382D30312D303192
:101B60003B0023482245636F222C22312E30302245
:101B70002C323030382D30312D30313B0023532280
:101B800045636F222C22312E3030222C32303038F7
:101B90002D30312D30313B00504F00504632333B19
:101BA0005055002564002B302B303B002564002568
:101BB000303258002E3030004F4E0000206E616EE3
:101BC0006F0001002D4E414E00000100A10EC21B0E
:101BD0000000F894EE27ECBBF1E0F5BFE5BFE09321
:101BE0006C00F8E1F1BDE1BD8DE0A2E0BB27ED9313
:101BF0008A95E9F780E090E1A0E0B1E0ED930197EC
:101C0000E9F7EAECFBE185919591009761F0A591E8
:101C1000B59105901590BF01F00105900D920197C7
:101C2000E1F7FB01F0CFEFEFEDBFE0E1EEBFC0E089
:101C3000D3E00C94FA160A9902C0E1E00895E0E0BE
:101C400008951A931FEFE2E00E94E365E3EFE1BB22
:101C50008BE18A95F1F7E0EFE1BBE4E4E0937400F7
:101C600085E88A95F1F70E948160E03091F4E9817E
:101C7000EE0FE0520E94EC6541F4EDB7FEB7FA9327
:101C8000EA931F930E94F1651F910E9492600E9447
:101C9000F565E0E0E09371000E94F565E12F3EC438
:101CA0001A9310E0E0E0E093E907E0E0EA93C9DF8F
:101CB000E43549F4E1E0EA93C4DFE093E907A09159
:101CC000E907A130C8F41F5F0E94FA650E9479738A
:101CD000A091E907A03011F4153008F001C0E5CF5C
:101CE0000E94FF650E9404660E94F45CECE9F8E142
:101CF0000E940966A895FECF19910895E881E03009
:101D000011F01D9801C01D9A219608950E940D663C
:101D10000E940D660E9412660E9417660E941C6651
:101D200008951A930A930E94195D10E0143020F56B
:101D300000E00430F8F4A12FE8E20E942066FA9354
:101D4000EA93A02FB0E0E8E1F0E00E94F473FA9388
:101D5000EA93E7E2F0E0FA93EA93E7E1F0E0FA933E
:101D6000EA93E02FEE0FEE0FE10FEA930E949A48FC
:101D70000F5FDFCF1F5FDACF0E94246609911991B0
:101D800008950E9428660E942E6619F50E94346606
:101D90000E940D660E943966E1E2EA930E940D6698
:101DA0000E940D660E9442660E9417660E94396674
:101DB0000E9445660E940D660E9442660E94486627
:101DC0000E944D660E940D660E942F46EBE9F0E0EE
:101DD00022C00E9450660E940D660E943966E1E2B0
:101DE000EA930E940D660E940D660E9455660E944D
:101DF00017660E9439660E9445660E940D660E9421
:101E000055660E9448660E944D660E940D660E94BB
:101E10002F46E1EFFFEFFA93EA930E9458660E9483
:101E20005D660E940D660E942F4608951A93E0E0B9
:101E3000E0930B0410E0133020F50E9460663196A9
:101E4000049000920A040E946666E2E3F0E00E94B9
:101E5000F47334960E946966EEE2F0E0FA93EA9336
:101E6000E3E2F0E0FA93EA930E946066E491EA9379
:101E70000E94606632960E9470660E942F461F5F25
:101E8000DACFE0910B04E0930A040E94736646C324
:101E90000E947C760E94195D0E947766ECE00E94A9
:101EA0007D66E8E7F0E0FA93EA930E940466E3E2D5
:101EB000F0E00E948366E1E2EA93E9ECF8E10E9437
:101EC00070660E942F46EBE00E947D660E940466C9
:101ED0000E940466EEE6F0E00E948366E091F10B5A
:101EE000F091F20BE491EA93E091F10BF091F20B97
:101EF00031960E94A7740E9470660E942F4631E0BE
:101F00000E948A660E948D6611F03F5FF9CF0E94A1
:101F10009B66301718F4E0E0E093BB050E949B66D7
:101F200011E00E94A3660E948D6611F0143008F043
:101F300023C00E9404660E946666E0E2F0E00E9410
:101F4000F4733496FA93EA930E94A666EAE1F0E00D
:101F50000E94AB660E94AE66E491EA930E94A3667B
:101F60000E94AE6631960E94A7740E9470660E941D
:101F70002F460F5F1F5FD5CF0E9473660E94837646
:101F80002EC327970E947C7630E00E9477660E94DD
:101F9000286610E0133010F00C94161000E00430A6
:101FA00010F00C9414100E94BA66329604900092BD
:101FB0000A04E0E0E0930B04FE013496FA93EA93FE
:101FC0000E94BA663496FA93EA930E94EA62EB851D
:101FD000E03039F4AD81A13210F4E0E0ED83E0E0CF
:101FE000EE83A02FB0E0E8E2F0E00E94F4733296B6
:101FF000FA93EA930E946666E0E2F0E00E94F473CE
:10200000B096FA93EA93E4E2F0E00E9483660E94BD
:10201000BA66E491EA930E940D66FE013F960E9423
:10202000C0663F5F0F5FBBCF1F5FB4CF0E94955F5D
:102030004DC40E947A760E940D660E940D660E9431
:10204000F45C3091D5070E94C4660E94776610E068
:10205000E091790B1E1700F500E0E091780B0E1768
:10206000C8F40E94D16699F00E94D8660E94E46686
:10207000519FF0010E94EE660E94F366E1E4FBE0EE
:102080000E94C0664E2F3A934A930E9491193F5F77
:102090000F5FE3CF1F5FDCCF0E9473660E948176E3
:1020A000DAC122970E947A76E9E0F7E0EE83FF83B7
:1020B00040E0443190F4AE81BF8111960E940167E7
:1020C0001396EFEFEC93AE81BF81EC93EE81FF812D
:1020D0003496EE83FF834F5FECCF0E94C46630914D
:1020E000D5070E94066710E0E091790B1E17D0F526
:1020F00000E0E091780B0E1798F50E94D16669F127
:10210000A091510BE0E8EA23E03819F40E94D86668
:1021100006C0E7E0E0930B04E8E0E0930A040E94C5
:10212000E4660E940D670E9466660E94F47333960F
:10213000FA93EA930E94F366E1E4FBE00E94C06632
:102140004E2FA091D507E32F0E941067EA0FFB1FC7
:1021500043833A934A930E9491193F5F0F5FC9CF1F
:102160001F5FC2CFE0910B04E0930A040E942E6629
:1021700041F50E94176771F40E9434660E940D6653
:102180000E943966EFE7EA930E940D660E940D6691
:102190000E942F460E9434660E9417660E9439668C
:1021A0000E9445660E940D660E9442660E94486633
:1021B0000E944D660E940D660E942F46EBE9F0E0FA
:1021C00027C00E94176771F40E9450660E940D6636
:1021D0000E943966EFE7EA930E940D660E940D6641
:1021E0000E942F460E9450660E9417660E94396620
:1021F0000E9445660E940D660E9455660E944866D0
:102200000E944D660E940D660E942F46E1EFFFEF8F
:10221000FA93EA930E9458660E945D660E940D66DA
:102220000E942F460E94955F0E94952E0E94817603
:10223000289608950E940667E0E0E0930B04ECE026
:10224000E0930A040E9404660E941C67E1E2EA939C
:10225000EBECF8E10E9470660E942F46EAE0E09302
:102260000A04E2E5F0E0FA93EA930E941C67EDE3CA
:10227000EA93E0EDF8E10E9470660E942F460E940A
:10228000955F08951A93A981A23019F40E941767E7
:1022900009F024C00E9429670E942C67BF01E981D0
:1022A0000E9433670E943D671E2FEFE00E947D660B
:1022B000E7E8F0E0FA93EA93EB810E943367329605
:1022C0000E9446670E944D67FA93EA93EFE7EA930C
:1022D000E3EDF8E10E9470660E942F461FC10E9444
:1022E000195DE0E0E0930B04A881A13051F40E9455
:1022F000FF650E9450670E94F45CE6EDF8E10E94E1
:1023000009660E94176769F4E2E0EA93BBDFE8E33D
:10231000F2E00E945567EAE3F2E00E9455670E94EE
:10232000AF5F2FDD4AC1E8810E943367FA93EA93D9
:102330000E945A670E942C67FA93EA930E944B5DB1
:10234000E881EA939FDF39C11A930A93EC81EA93FB
:10235000EADF1BE90E945D670E942C67BF01EC81E8
:102360000E9433670E943D670E2FAC81A43019F4A0
:102370000E94176709F009C012E8AA81BB811B9669
:10238000E0E0EC93EC81EA937DDF0E94D866EC817B
:102390000E946067FF93EF930E945067EE810E9456
:1023A000336731960E9466670E94AB66FA93EA93A0
:1023B000EC85E058EA930E940D66ED85FE850E944B
:1023C000C066AF91BF91EC93EC810E943367FA93A2
:1023D000EA93EE81F0E00E942C67FA93EA930E9460
:1023E000AF5F1981088125960895E7C01A930A9373
:1023F000E091790BAFE70E94FE730E2F11270E9428
:102400000D660E940D660E9412661A930A930E943E
:102410001C660E94FF650E94FF650E94F45CEC81CF
:10242000FD810E940966AA81BB81A030E0E8BE0759
:1024300031F0EA81FB81FA93EA930E94C7430E943C
:10244000FA650E94A5450E940D661A930A930E94A0
:10245000AF5F19810881269608950E947D62E0E0B1
:10246000E0930A04E0930A040E942E6619F4E1E95D
:10247000F0E002C0E1EFFFEFFA93EA93E0E6F0E06C
:102480000E948366EEE1F0E0FA93EA930E945D66B3
:102490000E940D660E942F4608951A9311E00E9433
:1024A000911B0E9469670E946E67B8970CF414E054
:1024B0000E940D660E944D670E947467E9810E9428
:1024C0007A670E9486670E9474670E948A670E94EA
:1024D0008F67E981EA930E94381BE983ADEFB6E08C
:1024E0000E9429670E9493673B9754F0ADEFB6E0D6
:1024F0000E9429670E9493670E949A67E9E40BC0D3
:10250000ADEBB6E00E9429670E9493670E949E6728
:102510000E94AF43E3E7EA930E948A5C1881229607
:1025200008950E940D660E940D660E94F45CE2EE22
:10253000F8E10E9409660E940D660E94A3670E944E
:102540001266ECE3F0E00E94A8670E940D660E940C
:10255000FF650E94F45CE09116060E94AB67E7EE0F
:10256000F8E10E940966E091E807EA930E94D943E6
:102570000E940D660E94AD67E0912D060E94AB6738
:102580000E940D660E9450670E94F45CE091440630
:102590000E94AB67EDEEF8E10E940966E0910B0640
:1025A000EA930E94D9430895E881E064E7B9369A36
:1025B000349BFECF349AE4B1F5B121960895E881B9
:1025C000F981AA81BB81AE17BF071CF4EA1BFB0B84
:1025D00006C0A881B981EA81FB81EA1BFB0B249626
:1025E000089528970E947C76EFE0E09361000E94B6
:1025F0002E6611F4E1E001C0E4E4E093620085E8B6
:102600008A95F1F7E5E0E093610085E88A95F1F7B6
:102610000E94B067E0936A05F0936B05E091760540
:10262000F0917705E0936805F0936905E1E0EA939E
:10263000BBDFE0937605F0937705EFE0E093610070
:102640000E942E6611F4E2E001C0E8E0E09362002F
:1026500085E88A95F1F7EAE0E093610085E88A95DC
:10266000F1F70E94B567E0936605F0936705E09186
:102670007405F0917505E0936405F0936505E0E05D
:10268000EA9392DFE0937405F09375050E94B567B5
:10269000A0916605B0916705EA0FFB1FA091740534
:1026A000B09175050E94BA678F010E94B067A09132
:1026B0006A05B0916B05EA0FFB1FA0917605B091FA
:1026C00077050E94BA679F01E0916605F091670562
:1026D0000E94C167FF93EF930E94B5670E94C16794
:1026E000AF91BF91EA0FFB1FFF93EF93E091740549
:1026F000F09175050E94C167AF91BF91EA0FFB1F72
:10270000E0937005F0937105E0916A05F0916B0517
:102710000E94C767FF93EF930E94B0670E94C7674C
:10272000AF91BF91EA0FFB1FFF93EF93E091760506
:10273000F09177050E94C767AF91BF91EA0FFB1F29
:10274000E0937205F0937305A0917005B091710547
:10275000E4E1F0E00E94C6730E2EA0917205B091E4
:102760007305E4E1F0E00E94C673E02919F00E94CD
:10277000DF47ACC000936C0510936D0520936E0588
:1027800030936F05A0915F05A23328F4E0915F05B7
:10279000EF5FE0935F050E94CD67989724F40E9455
:1027A000D26798970CF00EC0A0915F05AA3019F47B
:1027B000E1E0E0935C05A0915F05A83219F4E2E046
:1027C000E0935C050E94CD67AB35E0E0BE0734F0D6
:1027D0000E94D267AB35E0E0BE070CF477C0E09111
:1027E0006205EF5FE09362050E94D7670E94CD67A4
:1027F0000E94DC670E94E3670E94E867E0EAF0E07D
:1028000060E070E00E94F9737F936F93FF93EF9302
:102810000E94ED670F010E94D767DF01F001EA1BFC
:10282000FB0BAF91BF918F919F910E94F2670E9425
:10283000E3670E94F7670E94D2670E94DC670E94EC
:10284000FC67E0E8F0E060E070E00E94F9737F93DD
:102850006F93FF93EF930E9405680F010E94F76743
:10286000DF01F001EA1BFB0BAF91BF918F919F91AC
:102870000E94F2670E94FC670E94747664F4AC8147
:10288000BD818E819F81A038E0E0BE07E0E08E0729
:10289000E0E09E070CF01AC0E885F985E093540546
:1028A000F0935505EC81FD81E0935605F0935705B3
:1028B000E0915405F0915505FA93EA93E09156059D
:1028C000F0915705FA93EA930E9467470E94837636
:1028D0002C9608950E94195DEAE0F0E00E94466798
:1028E0000E940D5DE3EFF8E10E940966E4E1EA93DE
:1028F0000E9440430E940A68E4E1EA930E94404338
:10290000A0916205A13010F0A895FACF0E940D6643
:102910000E9410680E940D5D0E941568EBE10E9404
:102920001B68A0916205AF3110F4A895FACF0E9400
:102930001F68A0E0B0E00E94D2740E940D660E9461
:1029400010680E9428680E940D660E942F680E94ED
:102950000D5D0E94D7670E949A67A0916205AE3113
:1029600010F0A895FACF0E9415680E9434680E9462
:102970000D5DEAE10E941B68A0916205AF3110F481
:10298000A895FACF0E941F68A2E0B0E00E94D2741E
:102990000E9434680E9428680E942F680E942F6855
:1029A0000E940D5D0E94ED670E949A67A0916205EA
:1029B000AE3110F0A895FACFE2E0E0930804E6E427
:1029C000F0E00E9470660E940D5DE8E1EA930E94CB
:1029D0008A5CE1E0E0930804A0916205AF3110F455
:1029E000A895FACF0E943968A4E0B0E00E94D274A2
:1029F000E6E4F0E00E947066E8E1F0E00E944667DD
:102A00000E941C660E9442680E9447680E940D5DF9
:102A10000E94F7670E949A67A0916205AE3110F09C
:102A2000A895FACF0E9415680E942F68EFE5F0E0A4
:102A30000E944C68E9E10E941B68A0916205AF31D9
:102A400010F4A895FACF0E943968A6E0B0E00E9481
:102A5000D2740E942F68EFE5F0E0FA93EA93E8E180
:102A6000F0E00E9483660E941C66E8E2F0E00E94AB
:102A700069660E940D5D0E9405680E949A67A09198
:102A80006205AE3110F0A895FACFE2E8F0E00E94BE
:102A900050680E940D5DEFEFF8E10E9409660E9408
:102AA0005368A8950E945368A8950E94195D0895DF
:102AB0000E945968E2EBE2BF7894A9E1BBE00E9472
:102AC00068680E9429478DDD0E94D11BE2B3EF7830
:102AD0000E2EA091CB07B091CC07E7E0F0E0AE2737
:102AE000BF27EA23FB230E94A273E029E2BB0E94D6
:102AF000C65BE091F90BEF5FE093F90BA091F90B46
:102B0000AE3149F4A0910504E3E8EA27E093050417
:102B1000E0E0E093F90B199112C00E9459680A9302
:102B2000E3E8E4BDE0B1E295E7700E2F11271A93B8
:102B30000A930E94A81B0E94A05B09911991E99138
:102B4000EFBFF991E991B991A99199918991799101
:102B50006991F990199009901895E8EFFFEFE093CB
:102B6000020CF093030C0E94195D0E947D620E948A
:102B7000FF650E94AD67E2E0F9E10E9409660E94EC
:102B80008C620E946E680E94797308950E944F5B68
:102B90000E94E7400E94D01808951A93A8950E94B9
:102BA0005345E13011F00C941E16E091C105E1503F
:102BB0001E2FA091C005A13021F40E947368E0305F
:102BC00009F40BC00E947A68BF010E947A68E08114
:102BD000E260DB01EC930E948068A091C005A23006
:102BE00011F0A43089F40E947368E093D6050E9426
:102BF0007368E03029F00E947A68E081E27009F49D
:102C000003C01A930E948568A091C005A33019F4EF
:102C10001A930E948621A091C005A53029F4E09165
:102C2000C105EA930E94B621A091C005A73031F4F6
:102C3000E091C105E093D6050E946243E09105044E
:102C4000E07839F1E0910504EF77E09305040E9404
:102C5000D35FE0910504E07131F0E0910504E2708A
:102C6000EA930E94F25BA091E907A13330F0E2E021
:102C7000EA930E94210E1E2F01C010E0103808F0C8
:102C800010E0E091F70BE11711F41093E8071093AF
:102C9000F70B7CDF4EC01A930E94195D0E94FF65FE
:102CA0000E940D660E94F45C10E00E9477660E940C
:102CB0000D660E944D670E948F67E091D807E03053
:102CC00049F4EAE0F9E10E9409660E9489680E94DD
:102CD00099431E5FA091D807A130F0F0E091D8078A
:102CE000E150EA930E94F130A0916A0BAD3229F4D1
:102CF0000E9494680E946C7679F00E94A1680E94FC
:102D0000A6680E948A670E948F670E9494680E944A
:102D1000AB740E9499431E5FE091D807EF5FE09388
:102D2000D807163020F4A091D807AB3008F001C0C6
:102D3000BECF199108951A930E94195DE981E03080
:102D400019F4E0E0E093D507A981A230A9F410E0DE
:102D5000A091D507A13010F0163008F00DC0E09119
:102D6000D507E150E093D5070E94AA6819F40E94A4
:102D7000B86809F01F5FECCF0E94776610E00E94F0
:102D80000D660E944D670E948F67A091D507A336FC
:102D900000F50E94AA6819F40E94B868B9F0E091A1
:102DA000D5070E947A670E9486670E948F670E94FB
:102DB000C3680E949A67E8E7EA930E948A5C0E94CF
:102DC000C8680E94CC680E9499431E5F0E94D76821
:102DD00007C0E1E1F9E10E9409660E94D7681E5F21
:102DE000163020F4A091D507A53608F001C0C7CF52
:102DF0000C940B1B14B7E0E0E4BFE5BFE0936D005B
:102E0000E0936C00EBBBEFEFEABBE0E0E8BBE7BBB5
:102E1000E5BBEFEFE4BBE0E7E2BBE1BBE0E3E3B936
:102E2000E8EBE2B9E0E0E0936200E0936100E09358
:102E30006500EFE0E0936400E0E0E0BFE7E0E3BFBF
:102E4000E2EBE2BFE0E0E1BFEFBDEEBDEDBDECBD0A
:102E5000E7BDE6BDEBBDEABDE9BDE8BDE0937900A5
:102E6000E0937800E3E0E5BDE3E8E4BDE0E0E3BD46
:102E7000E0938B00EAE0E0938A00E0E0E0938900D1
:102E8000E0938800E0938100E0938000E2E1E0932A
:102E90008700E4E3E0938600E0E0E0938500E093C0
:102EA0008400E0938300E0938200E0936A00E0E313
:102EB000EABFE0E4E9BFE8BFE1E4E7BFE0E0E093B8
:102EC0007D00EBB9E8EDEAB9E6E0E0939500E0E0DB
:102ED000E0939000E3E3E9B9E0E0E0939B00E8EDE4
:102EE000E0939A00E6E0E0939D00E0E0E093980034
:102EF000E9E1E0939900E0E8E8B9E0E0E0BDE0E472
:102F0000E7B9E7E8E6B9E0B5EF7EE0BDE0E1E093E0
:102F10007000E0E0E0937200E4E4E0937400EEE11E
:102F2000E1BDEEE0E1BD0E9424480E94024810FF8E
:102F300003C0AAE0B0E00CC012FF06C0ABE0B0E0F6
:102F40000E94C6740E94DD6813FF06C0ACE0B0E0CA
:102F50000E94C6740E94DD680E94E768E057F84F3F
:102F600010830E94E768EF56F84FA9E00E94ED68D1
:102F7000F4DD0E94FF650E94F4680E9433550E94B0
:102F8000500EE4E0E0936100EFE0E09362000000A7
:102F900000000000E0B1E170E13019F0E1E0E09301
:102FA000F80BEBE0E0936200000000000000009BE3
:102FB00003C0E1E0E093F80BE8E0E0936100EFE0AC
:102FC000E0936200000000000000E0B1E270E23037
:102FD00019F0E1E0E093F80BE7E0E0936200000015
:102FE00000000000019B03C0E1E0E093F80B0E94A9
:102FF000CF2FE030D1F40E94FF650E94F468E6E133
:10300000F9E10E940966A8950E94F7680E94FC6891
:103010000E9447680E9479730E94F7680E94FC68CA
:10302000ECE2F1E00E940269EECF0E94802F7894DA
:10303000E091F80BE03021F0E2E2F9E10E9409664C
:10304000A091F80BA03089F40E94D7670F010E946D
:10305000ED670E161F0644F40E94F7670F010E94E9
:1030600005680E161F060CF001C002C00E946A140B
:103070000E948C33E030C9F00E94FF650E94046614
:103080000E94F45CEBE2F9E10E9409660E94FA6595
:103090000E947973A8950E94FA650E947973A89599
:1030A0000E94FA650E947973A8950E94FF650E94AC
:1030B00004660E94F45CE7E3F9E10E9409660E945D
:1030C0000669EA930E94D9430E94FF650E94F46852
:1030D000EBE3F9E10E940966E091E907EA930E94B7
:1030E0008A5CE091F80BE030D9F4E0E0E093040C66
:1030F000A091040CA03540F4EAE0F0E00E940269DF
:10310000A8950E940B69F4CFA091040CA03520F083
:10311000A0916205AF3108F402C00E946A1438C061
:10312000E0E0E093040C0E940669A091040CAE1745
:1031300060F4A8950E9411690E94FC680E94A6662E
:103140000E9479730E940B69EECFA8950E940A68CD
:10315000E0E0E093040C0E941669A091040CAE1705
:1031600060F4A8950E9411690E94FC680E94A666FE
:103170000E9479730E940B69EECFA8950E940A689D
:10318000A8950E940A68E0910504EF77E093050492
:103190000E94D85B0E94CD150E94F82AFBCFFFCF7A
:1031A0001A930A93A091D007A43009F43FC010915C
:1031B000E60700910F0CE091E807E03059F0E0934A
:1031C000E607689424F80E941B69E0E0E093E707B3
:1031D000E0E520C0E091E707E03021F0E093E6076A
:1031E000E2E518C0E0E0E093E607E0930F0CE09121
:1031F0007B0BE03031F0E0917B0BE150EA930E94D1
:103200001D31A091EB0BA17039F0E0917B0BE093A5
:10321000E607E4E4E0930F0CA091E6071A1721F407
:10322000A0910F0C0A1711F0689423F809911991D5
:1032300008951A930A930E94E768E057F84F8F01A8
:10324000D8011196EBE0EC93EC81D8011696EC9343
:10325000EB81D8011796EC93D8011896E0E0F0E0E6
:10326000ED93FC93D80112960E942169D80114961F
:103270000E9421690E9426691EC11A930A930E9426
:10328000E768E057F84F8F01D8011196ECE0EC9316
:103290000E94266944C21A9318E0113108F5E091A2
:1032A000CB07F091CC07A981BA81EA27FB27BF01A0
:1032B0000E943269E623F723309781F00E94326939
:1032C000A981BA81EA23FB23309731F01A93E0E019
:1032D000EA931A93AEDF02C01A93CFDF1F5FDDCFF0
:1032E0001DC2A091D10BA93030F0E091170CA09134
:1032F000160CEA1709F414C0E091170CE03021F421
:10330000E3E6EA93BADF08C0E091D10BEA93E0E08C
:10331000EA93E3E6EA938DDFE091170CE093160C55
:1033200008951A9310E0153088F40E943D69E081F9
:10333000E03029F00E944369AA81EA1709F004C02D
:103340000E944A690E944F691F5FEDCFE7C1A091BB
:10335000510BECE1EA230895A091510BA07411F0F8
:10336000E2E00895A091510BA07809F0EFC10DC0E3
:10337000A091400BAF3F09F4E9C1E9DFE43009F463
:10338000E5C1E5DFE03109F4E1C1E1E00895089528
:10339000A881AF3F11F4E0E07DC1D9DFE43011F442
:1033A000E1E078C1E0E076C1A881A23019F4CFDF76
:1033B000E83011F0E1E06EC1E0E06CC1A881B981B4
:1033C000AC91A130A8F0A881B981AC91A43180F46E
:1033D000A881B981EC910E946967E050FD4FE081BE
:1033E000EF770E2EA881B9811296EC91E01509F0C5
:1033F00002C0E1E011C1E0E00FC1A881A13118F0E5
:10340000E881E051E883E8810E9454690E945E6986
:10341000A091870BA13018F0A881A43009F006C054
:10342000E6E9F0E00E94A7740E945E6933C1A881BA
:10343000A13010F0A43008F006C0E8810E9469694C
:10344000EC5DF94F26C1E0E025C1A881A13010F064
:10345000A43008F006C0E8810E946969E75DF94F71
:1034600018C1E0E017C10E947C76EC81EA93EDDFA1
:10347000EF731E2F1030E1F0EC81EA93E6DFE07489
:103480003E2FE12FE150A1E00E949A73A09108061F
:10349000EA230E2F303011F4003009F002C0E1E0D1
:1034A00008C0303011F0003009F402C0E1E001C082
:1034B000E0E00E948376259608950E947A7600E0E7
:1034C0000330A0F50A930E9463310E946E69A7E160
:1034D0000A9FF001E95EF94F0E9475690E94A36797
:1034E0000E94BF62E091E70BDA015096EC93A09145
:1034F000E60BEFE3EA23AE2FE091E90BE295E07FE4
:10350000EE0FEE0FEA0FDA015596EC93E091E70B20
:10351000E1503E2F3F3F41F0E091E80B0E947A6975
:10352000DA015196ED93FC930F5FCACF10E013368A
:10353000D0F51A930E94B1301A932ADFE13089F551
:10354000E091540BEA9373DFE1500E2F0F3F49F1E6
:103550000E946E69E12FDA011396EC93E091540B0F
:10356000DA011496EC93E0915A0BF0915B0BDA01BF
:103570001696ED93FC930E9480690E94B673A4E6B0
:10358000B0E080E090E00E94F973DF01CB01E091B0
:103590005A0BF0915B0B0E94F267DA011A96ED93D9
:1035A000FC931F5FC4CF0E94817626960895A09158
:1035B000D007A23031F0A83021F0A73011F0A530AB
:1035C00009F40AC00E948569EFEFF0E00E94886963
:1035D00074DFE0E0E093590608951A93E981E0581A
:1035E000E98310E01530B0F40E944369AE2FE98101
:1035F000EA1759F4A3E21A9FF001E55AF94FE08166
:10360000AE2FE091E607EA1709F002C0E12F03C0F0
:103610001F5FE8CFEFEF1881229608950E947C7615
:10362000ED81EA93DADF1E2F1F3FF1F00E943D6922
:103630009F01D9011296EC91EF77EC93EC81D901BF
:10364000EC930E946967E45FFC4FBF01EC810E942C
:103650006967E45FFC4FE081EF77DB01EC93EC817D
:103660000E9469670E944F69E12F0E948376DAC445
:103670000E948C69E081E03051F4E091090CEF5F29
:10368000E093090C0E948C69A091090CA0830E9410
:103690008C69E081219608951A931FEFE0918B0BBE
:1036A000F0918C0BA981BA81AE17BF073CF0E09175
:1036B0008D0BF0918E0BEA17FB070CF412C00E94E1
:1036C00091690E94F62F1E2F103031F01F3F21F01C
:1036D000E091E607E11729F4E1E0E093170CE0E060
:1036E0001DC0E0E0E093170C18C01A930E94916986
:1036F000D3DF1E2F103089F01F3F39F4EEE3F9E1DC
:10370000FA93EA93EB81FC8104C0EEE4F9E10E94B4
:103710006667FA93EA930E94F611E12F18812396C7
:103720000895E0916005E03009F00895E0911106F8
:10373000E03009F008950AC0E0916105E03009F039
:103740000895E0911206E03009F00895E0E0089550
:103750000E947C76E0910B06F0910C06AC81BD8155
:10376000EA27FB279F0110E0133090F4F901E17084
:1037700049F0A7E11A9FF001EA5EF94FDF01EC91F1
:10378000EF5FEC93D9010E9496699F011F5FECCF18
:10379000EC81FD81E0930B06F0930C060E9483768A
:1037A00041C428970E947A7630910B0610E01330BE
:1037B000B8F5A7E11A9FF001E65DF94F0081E12F0E
:1037C000A1E00E949A732E2FE22FE32391F000389C
:1037D00010F0003C08F001C00F5F003C31F4E22F14
:1037E000A0910806EA2BE0930806003808F400E8E8
:1037F0000FC0003408F40F5F003439F4EFEFE22714
:10380000A0910806EA23E0930806003808F000E0DB
:10381000A7E11A9FF001E65DF94F00831F5FC7CF54
:10382000E0E0E0931106E0E0F0E0E093CD07F093F4
:10383000CE07E091170CE03021F0E091D10BEA9334
:10384000DCDDE091D407EF5FE093D407E0919A0BC1
:10385000A091D407EA1751F4E0919A0BF0E0A0E0B0
:10386000B1E00E94BB74EA1BE093D407A091D0079B
:10387000A13019F0A93009F096C0A091190BB091B0
:103880001A0BE4E1F0E00E945174309719F4E1E082
:10389000E093D60746DFE03019F04EDFE07809F418
:1038A00062C04ADFEF775E2F5A930E94B1300E94C8
:1038B0000D67E65AF94F5081503011F40C94B31C47
:1038C00057DDE13031F4E091D107EA936DDDE0306E
:1038D00009F449C00E949B69AE0FBF1FEC91EC71C7
:1038E000EC3021F4E091D407E07851F40E94A16912
:1038F000EC91EA9382DD0E94A969EC91EA937DDD67
:103900000E94A169AC91A63070F5ADEBB6E00E94C3
:103910000D670E94B1690E9468680E94A169EC91DC
:10392000EA9385DD1E2F1130F0F00E94B6690E94E7
:10393000B969CF010E94B6690E94B1696D917C910D
:10394000E12F0E946969EA5EF94FE081F0E0E60F3D
:10395000F71FDC01ED93FC93E12F0E946969EA5E99
:10396000F94FA0E0A08310E01330E8F40E94BE6994
:1039700013965C915F3FA9F05A937ADE5E2F0E9406
:10398000C8690E94B6690E94B969BF010E94B66900
:103990000E94B1690E94CE69AE81BF811296E0E0BB
:1039A000EC931F5FE1CFA091D007A23039F0A8308F
:1039B00029F0A53019F0A73009F0ECC1E0E0E09360
:1039C000D70700E0053010F00C94CA1EA3E20A9F4E
:1039D000F001E65AF94FEA87FB87AA85BB85AC91CF
:1039E000A03019F0A281A07809F0D2C1E091D707E8
:1039F000EF5FE093D707AA85BB8513960E94987462
:103A0000309771F0AA85BB8513960E94DB690E94EE
:103A1000E16929F4AA85BB8513960E942169B8C182
:103A20008BDEE03021F00E94E16909F4B1C120E0B1
:103A300030E0333010F00C94731E0E94EB69DF010C
:103A40000E948A660E94F169A27031F4E885F985C6
:103A5000A481B581109709F414C1E885F985A18185
:103A6000A47011F40C94961DA181A87021F40E94F9
:103A70006A2CE03009F459C00E94E7680E94FC6992
:103A8000EBE0EC93A885B9850E94046AA885B98506
:103A90001396EC91AC85BD851796EC93EC85FD856E
:103AA00038960F01E885F985A181E1E0EA230E94BB
:103AB0000B6AED93FC93A885B98514960E949874BF
:103AC000AC85BD851296ED93FC930E940E6AAC8581
:103AD000BD851496ED93FC93A02FEAE0EA9FF001D8
:103AE000E30FEF5F0E94146AE885F985A085B18530
:103AF000E2E0F0E00E94F473A885B9851896ED9392
:103B0000FC930E940E6A309739F4A885B9851896FF
:103B1000E8EEF3E0ED93FC93E885F985A181E8E018
:103B2000EA2BA885B9851196EC936CC0E885F985D8
:103B3000A181A17031F4A885B98514960E94DB6932
:103B400041C00E941D6A73DCE1501E2F0E94BE69B5
:103B50001296EC91E030F1F4AE81BF8153960E9451
:103B60006868EE81FF81A189B289109751F00388BE
:103B70001488AE81BF8151960E949874E015F105BA
:103B80000CF007C00E94226A11F00E942A6A0E946B
:103B9000326A0EC0E885F98534960E943A6A0E941E
:103BA0000B6A0E94426A0E94476A53960E942169EA
:103BB000E885F985A581AA232AF4A885B9851496F4
:103BC0000E942169A885B985EC91EC71EC3021F453
:103BD000E091D407E078B1F4E885F985A481B58156
:103BE0005E971CF4A181A07209F404C0E885F985F0
:103BF000A28106C00E941D6A00DCE885F985A381C8
:103C0000AA93FBDB0E940E6A309781F0A885B985E4
:103C100018960E94DB690E940E6A309739F40E9460
:103C2000226A11F00E942A6A0E94326A0E941D6A6A
:103C30001ADCE03031F10E94226A89F00E942A6A7F
:103C4000AA85BB85EC910E946967E45FFC4FBF01C8
:103C5000AA85BB85EC910E9469670E944E6AAA857D
:103C6000BB851296EC91E058AA85BB851296EC9321
:103C7000E3E0E09309060E941D6AE7DBEF73E0933F
:103C80000A06A885B98514960E949874309749F55C
:103C90002F5F323030F5A885B98516960E9498744A
:103CA000309789F0E885F985A681B7810E94556A29
:103CB000AA85BB851396ED93FC93A885B9851696C6
:103CC0000E9421690EC00E94EB69DF01E32FEF5FC4
:103CD000F0E00E94F169EDEFEA23A885B98511961D
:103CE000EC933F5FA6CE233011F00C94C81E0E94C7
:103CF0006A2CE03079F00E94E7680E94FC69E8E0F5
:103D0000EC93AA85BB850E94046AAA85BB85EC91C9
:103D10000E94146A0E94226A11F00E942A6AAA85EF
:103D2000BB85E0E0EC93EA85FB85A581ECE1EA2325
:103D3000E83071F50E940669AE2FEA85FB85E38DB8
:103D4000EA1741F4EA85FB85E48DE150EA930E948D
:103D5000AC2F1EC00E946A2CE030D1F00E94E768B0
:103D60000E94FC69E3E0EC93AC85BD85EFEFEC933A
:103D70001896EA85FB85E38D0E945A6AAC85BD855D
:103D80001296EA85FB85E48D0E945A6A0E945E6A5B
:103D90000F5F18CE0E94646A49F4A091D007A23048
:103DA00021F0A83011F0A53009F401C050C010E096
:103DB000133010F00C94271F0E94BE6913965C917B
:103DC0005F3F11F40C94251F0E94C869AE81BF812A
:103DD000BD010E94CE69EE81FF8138960E943A6A49
:103DE0000E946A6A0E94476A0E949874DF010E94DA
:103DF0007076B4F4EE81FF81A681B7810E9470765F
:103E00007CF4AE81BF810D901C90AE81BF8116966F
:103E10000E949874D001AE1BBF0B0E9470760CF00C
:103E200014C0AE81BF81BD010D901C90EE81FF8159
:103E3000A681B781F001EA1BFB0BDB01ED93FC933C
:103E40005A93E5E0EA930E9473451F5FB1CFE0917A
:103E5000D307E03041F4E091CD07F091CE07E09335
:103E6000CB07F093CC070E9481762E9608950E948E
:103E70007C760E946E6A1E2F2FE330E00091D507FA
:103E8000A091CF0BA13080F0E091CF0BE150A09139
:103E9000D507AE1728F0E091CF0BE1503E2F04C0BC
:103EA000E091CF0BE2502E2FEC81E03049F1EF3F53
:103EB00051F4A091D507A11BA31720F0E091D507DD
:103EC000E11B0E2F1DC0EE3F59F4E12FA091D50745
:103ED000AE0FA21720F4A091D507EA0F0E2F10C045
:103EE000EC3F49F4A091CF0BA13020F0E091CF0B33
:103EF000E1500E2F05C0AC81A1501A9FF0010E2F8A
:103F0000E091D507E01751F00A930E94B130A091DB
:103F1000410BAD3209F4032F0093D5070E94195DC0
:103F2000A091D007A83019F40E94511002C00E943D
:103F300019100E948376259608950E947A7607DAF2
:103F4000E03111F40C940F2020E030E040E050E02C
:103F500010E0133050F50E94756A0E949367309705
:103F600011F10E94786A0E9454692E2B3F2B0E9407
:103F7000786AEA9378DAE03029F0E3E0E093090622
:103F8000E0E04EC00E947F6A0E9454692E2B3F2BB6
:103F90000E947F6AEA9367DAE03029F0E3E0E09379
:103FA0000906E0E03DC01F5FD4CF00E0053068F5B2
:103FB000A3E20A9FF001E65AF94FE081E03019F1DF
:103FC00010E0133000F50E94EB69DF010E944D679D
:103FD0000E94866AAE0FBF1F1296EC910E94546930
:103FE0004E2B5F2B0E94EB69DF010E944D670E9400
:103FF000866AAE0FBF1F1396EC910E9454694E2B38
:104000005F2B1F5FDECF0F5FD1CFF901E423F523D4
:10401000309729F0E1E0E0930906E0E001C0E1E03B
:104020000E948176269608951A93E0910D0CE03057
:1040300011F40C946020E0919B0BE13059F4A091B5
:104040000D0CA13311F4EFE001C0E0E0EA930E940F
:10405000AB5536C0E23059F4A0910D0CA13311F4E8
:10406000E6E001C0E5E1EA930E94AB5529C0E330E8
:10407000B1F410E0173040F40E944D67E950F74F5B
:104080000E948D6A1F5FF6CFA0910D0CA13311F431
:10409000E1E301C0E0E3EA930E94AB5511C00E9446
:1040A000916AE9E4EA930E94F558E0910D0CEA93D5
:1040B0000E94F558E0E0EA930E94F5580E94735A76
:1040C00040C222970E947A7630E0A091D007A230B9
:1040D00029F0A83019F0A53009F014C1A985A3363C
:1040E00010F00C948121E091E607E03009F40AC158
:1040F000E9850E94986AE03131F4E1E3E0930D0C28
:1041000093DFE1E0FFC034D9E03009F4FBC010E0F8
:10411000153080F40E943D69E081E03031F00E946A
:104120004369AE2FE985EA1709F002C0E0E0EAC072
:104130001F5FEECF02DFE03011F40C94812110E01C
:104140000E943D69EE83FF83AE81BF81EC91E03038
:1041500011F00C947A2113960E94216900E003303B
:1041600010F00C944B21A3E21A9FF001E15AF94F91
:10417000DF010E94A3660E949D6AAF01DA011696D4
:104180000E9421690E94A56ADA011296EC930E94AE
:10419000AC6ADA011396EC93A091510BEEEFEA238F
:1041A000DA01EC930E94B36ADA011196EC93CFD84E
:1041B000E43139F0FA01A181E2E0EA2BDA0111964B
:1041C000EC930A93F1D8E03011F40C942D21FA010C
:1041D000A281AA932CD9E1502E2F2F3F81F0A7E185
:1041E0002A9FF001EA5EF94FA0E0A083A7E12A9F91
:1041F000F001E95DF94FA0E0B0E0A083B1830E9437
:10420000BB6A0E949367DA011496ED93FC93013028
:1042100030F00E94BB6A0E949367309709F00EC08D
:10422000AE81BF811596E02F0E94BE6A0E94866A09
:10423000AE0FBF1F1196EC91E062EC93AE81BF818F
:104240005A96EC91E062EC93023030F40E94C16A1D
:10425000DA0116960E945A6A04C0DA0114960E9486
:10426000216975D8EC3019F4E0E0E093D4070E949E
:10427000C86A0E947A69DA011896ED93FC93FA01F4
:10428000A281A63030F0A181E4E0EA2BDA01119698
:10429000EC930F5F64CFA091D007A23011F0A5304E
:1042A00019F4A885AF3F08F007C0E091E607EA934C
:1042B000EA85EA930E940D32E885AE81BF81EC93D6
:1042C000E091E607AE81BF811196EC93E985AE815E
:1042D000BF811296EC93A885A43128F4E8850E944A
:1042E00069670E944F69AE81BF811696EC91ED7FA0
:1042F000EC9331E01F5F303011F4153008F001C04D
:104300001FCFE32F0E9481762A9608951A930A936D
:10431000A091D007A23011F0A53021F40E94CF6AFD
:104320000E948568A091D007A830E1F40E94CF6A6E
:10433000E1E0EA930E947E5DE091990BE03081F428
:10434000EA81ADE0EA9FF001E050FD4FE081EF77B8
:104350001E2FABE01A9FF001EF51FA4FA0E0A083AF
:10436000689420F8198108812396089564970E9423
:104370007A76A091D007A23039F4E091E607EA936B
:10438000EB8DEA930E940D32A091D007A83011F076
:104390000C9427220FEF20E0233050F4A7E12A9F4E
:1043A000F001E95EF94FE081AE2FEA8DEA1709F4DA
:1043B00002C02F5FF1CFA7E12A9FF001EC5EF94F19
:1043C000AF01DA0115960C910F3F11F40C942722DE
:1043D0000E94DA6A10810E94E06AECF4A3EEBBE06E
:1043E0000E94DB690E94EA6A0E94F06AA083B1839E
:1043F0001A930E944436ABE00A9FF001E752FA4F4D
:1044000030810A93FE0137960E94F56A3A93FE01C5
:1044100037960E94F96A0E94FF6AC9F40E94DA6A1C
:10442000AFEFA083DA011396EFEFEC93DA01159664
:10443000EC930E94EA6A0E94056B0E940A6B1A9331
:104440000E9444360A930E949311689420F80E94B7
:1044500081766B9608951A9310E01031B0F4A7E1BD
:104460001A9FF001E75DF94FE081EF73AE2FE9810C
:10447000EA1729F41A930E94331AE03009F403C0B2
:10448000E1E01881DFC01F5FE8CFE0E01881DAC00B
:104490001A93E091100CF091110CFA93EA930E9498
:1044A0006E680E946562E030F9F00E94136B10E0C4
:1044B0001330D0F4A091140CAF5FE3E00E944E746F
:1044C000E093140CEF5FEA93C6DFE03059F0E3E0CD
:1044D000E0930906E091140CF0E0EF5FFF4EE093EB
:1044E0000A062FC01F5FE4CF2CC01A93E091080684
:1044F000E0930C0CE8E7F0E0FA93EA93ECEDF0E0DF
:10450000FA93EA930E944B5D10E01330D0F4E12F50
:10451000EF5FEA93A0DFE03091F00E940D66E12F9B
:10452000EA5F0E941A6BEBE5F9E10E940966ADE9CA
:10453000BBE00E944D670E949D6A0E941C6B1F5F3A
:10454000E4CF19910895A4DFE0910906E13029F440
:10455000E3E6F9E10E941F6B3CC0E23029F4E0E79A
:10456000F9E10E941F6B35C0E33051F4EBE5F9E14E
:10457000FA93EA93E0910A06F0E0E050F04F29C088
:10458000E43019F4E8E7F9E11FC0E53031F4E091D7
:104590000A06EA930E94F51120C0E63019F4E0E81B
:1045A000F9E112C0E73029F4E6E8F9E10E941F6B57
:1045B00010C0E83029F4E2E9F9E10E941F6B09C05C
:1045C000E93059F4E1EAF9E1FA93EA93E0910A0655
:1045D000F0E0FA93EA930E94F611E0E0E093090616
:1045E0000895A881B9811196E1E0EC930E94246BB3
:1045F000A881B9811296ED93FC930E94AC19A88111
:10460000B9811796EC930E940669A881B981189622
:104610000E945A6AE091C105A881B981EC93E091AA
:10462000E00BA881B9811696EC93E091400BA8812C
:10463000B9811A96EC930E948069A881B981149679
:10464000ED93FC932296089564970E947C76A09146
:10465000990BA230E1F4EB8DEA930E94B1300E94F5
:10466000AC19A3EEBBE00E945A6AA1EEBBE0EB8D51
:104670000E945A6AE091E607E093E00B0E94296BE2
:10468000309721F00E94296B0E942E6B14C0AA8DD6
:10469000AF3F09F4CEC0EA8DEA930E943D36AB8D60
:1046A000AF3F29F40E94246B0E94336BEB8FEB8D9C
:1046B000EA930E94B1300E94AC190E2FA98DAF3F32
:1046C00021F00E94B819E03009F001C0B2C00E9488
:1046D000F06A0E94A366AE17BF071CF02EDCE13023
:1046E00009F0A7C0A091880BA03021F4A091990BEC
:1046F000A23021F50E940669E13041F00E946A2C47
:10470000E03021F00E94802CE03009F004C00E94CB
:10471000E7680E94376B0E940669E13021F40E942D
:10472000702CE03009F409C00E943E6BE75AF84F44
:10473000FA93EA9356DF0E94446B79C0EB8DEA93BB
:10474000EA8DEA93BEDC1E2F113011F00C94172471
:10475000A0918A0BA13069F4E091E607EA930E94E8
:10476000246BFA93EA93EFEFFFEFFA93EA930E9438
:104770001B430E94F06A0E94A3660E94426A0E9444
:104780004A6B689420F8A091990BA03019F4A88D79
:10479000AF3F09F437C00E944F6BE352FA4F0E94BB
:1047A000F06AA083B183E88D0E9460673081E88D54
:1047B000EA93FE0135960E94F56AE88D0E946067D3
:1047C000E081EA93FE0135960E94F96A0E94A719DA
:1047D000E03131F00E944F6BEF51FA4FA1E005C07C
:1047E0000E944F6BEF51FA4FA2E0A0830E944F6BE3
:1047F000E152FA4FFF93EF930E945962AF91BF913C
:10480000ED93FC930E94FF6A19F4E0E0E093E00B63
:10481000EA8DEA930E944436E091E607EA930E940B
:10482000296B0E94AB66FA93EA930E94C934E1E0D7
:1048300001C0E0E00E9483766C9608957EDBE13053
:1048400041F40E946A2CE03021F00E94802CE0307C
:1048500009F009C00E94296B0E942E6B0E94E76834
:104860000E94376B1BC223C20E94546B0E945A6B7A
:104870000E940D660E940D660E94F45CA091D20712
:10488000A23021F4E5EBF9E10E940966A091D2077C
:10489000A13021F4ECEBF9E10E940966E091D20726
:1048A000E03021F4E3ECF9E10E9409660E94646BB8
:1048B0000E94F45C0E94696B0E946E6BFA93EA930B
:1048C000E0915A05F0915B050E94746B0895E1E058
:1048D00003C0E0E001C0E2E0E093D207C5DF089545
:1048E0000E94A719EC3109F0E2C1E091500BE336C8
:1048F00031F4A091D007A23009F4EBDF17C0E23603
:1049000031F4A091D007A23009F4E5DF0FC0A091E7
:10491000C005A23011F0A63021F4E091500BEA93CB
:10492000A6DAA091C005A43009F4D1DFB7C1E1E057
:10493000E09309040E940D660E940D660E94786B48
:104940000E940D660E940D660E94F45CE0EDF2E0AC
:104950000E940966E091D1070E947C6BEEEDF2E0C7
:104960000E940966E2E0E093090408950E948569C7
:10497000E3EEF0E00E948869E881E03009F406C0C7
:10498000A091D107AF5FE3E00E944E74E093D1079E
:10499000E1E0E093090C0E945D1A6FC20E947C76F0
:1049A00010E0133610F00C9421250E944D67E65A52
:1049B000F94F30813F3F11F40C941F251A930E9448
:1049C000B13000E00E94806B0E9493673B97C4F077
:1049D0000E94836B0F010E94806B0E949367D0013D
:1049E000ED93FC930E949B69EA0FFB1F0F010E944D
:1049F0009B69AE0FBF1FEC91EE7FD001EC9301E0FD
:104A00000E94896B0E9493677597A4F00E94836B44
:104A10000F010E94896B0E949367D001ED93FC9374
:104A20000E949B69EA0FFB1F0F010E949B690E9475
:104A30008C6B01E0013019F41A930E94DA301F5F89
:104A4000B0CF1AC41A930A9323FE03C00E94936B3B
:104A500014D70E948645E030C1F1E0E00E949A6BD5
:104A6000103820F5113219F40E94936B06D71D34CB
:104A700039F40E94A16B0E94165AE3E0E093CF073D
:104A80001B3271F40E94A66BEAE2EA93EEECF9E1C4
:104A9000FA93EA93E091D107E05DEA930E94165AF7
:104AA0001F3219F4E1E0EA93E2D941DF103868F0EF
:104AB0000E94AC6B1A930E94381B12DFE03011F495
:104AC000103208F002C0E1E6F0E20E949C1B0E2FBB
:104AD0000038C8F10F770336A8F5E091D607E0302B
:104AE00031F00A930E944D12E0E0E093D607E09186
:104AF000150CE01739F10A930E94B1300E94A169A8
:104B0000AC91A83028F40E94A969AC91A830A8F013
:104B1000E02FEF5FE09359060A930E94381B0E9432
:104B2000A169EC91EA930E94A969EC91EA93E09162
:104B30005906EA930E94191903C0E0E0E093590670
:104B40000093150C0EC0A091150CAF3F51F0E091F1
:104B50005906E03019F0EA930E943D19EFEFE09317
:104B6000150C099119910895A881A03310F0AA336A
:104B700008F01DC00E94B06BE8EEF3E00E94517493
:104B8000AAE0B0E00E94F473DF01E8810E94B56BF7
:104B9000EA0FFB1FE093DC07F093DD07E1E0E09311
:104BA00009040E94646B0E94786B0E94696BA88163
:104BB000A33441F40E945A6B0E94646B0E94786B8C
:104BC0000E94696B5AC11A930A93A0E023FCA1E0EA
:104BD000A03019F0AA81A03009F016C0E89423F89B
:104BE000E7E0E093CF070E94355CA091E807A03092
:104BF00019F40E94B86B09F407C0E7E0EA930E9439
:104C0000BD6B3BD6E89424F824FE25C0E091EA076A
:104C1000F091EB070E9469660E946562E13019F02D
:104C2000AA81A130B9F456D6E030A1F00E94C06B41
:104C30000FEF1FEF0E94C76BE03021F40091DE07F9
:104C40001091DF07EB81EA93E091E607EA931A936C
:104C50000A9313D610C0E091EA07F091EB07FA939C
:104C6000EA93ECE2F1E00E94CF6BE13021F40E9484
:104C7000D36BE093E7071981088100C3E0917E0BB5
:104C8000F0917F0B0E94D76B11F4E2E00895E09160
:104C90007C0BF0917D0B0E94D76B11F4E1E008953D
:104CA000E091820BF091830B0E94D76B11F4E0E04E
:104CB0000895EFEF0895E0E0E093D207A091D007C8
:104CC000A23021F40E94195D0E941910A091D00712
:104CD000A83009F430D6A091D007A53009F434D11A
:104CE0000895E2E0EA930E944043E1E0E093090482
:104CF000E881EA9339DFA881AF3721F4E09110060B
:104D0000E37009F403C0E2E0E093CF07A881A13289
:104D100039F0A33421F40E94B06B109709F004C05D
:104D2000A091D007A23009F00FC0A091D207A33004
:104D300009F4D1DDA091D207A23009F4BCDFE091E3
:104D4000D207E03009F4C5DDA881AD3311F00C9431
:104D5000FD260E94355CE091D207E03089F4E091B5
:104D6000DC07F091DD070E94DB6B41F4E091DC078A
:104D7000F091DD070E94E16B9EDF01C0AADD3DC01E
:104D8000E13069F47BDFEF3F41F0E3E00E94E66B46
:104D90000E94A16B0E94EC6B01C08DDF2EC0E2303F
:104DA000F1F40E94B06BA336E0E0BE07B4F4E091EA
:104DB000DC07EA930E94F36BE1E0E09309040E94B0
:104DC0000D660E940D660E94F45C0E94F76B0E94C3
:104DD0001A11E3E0E093D20701C07DDD0EC0E3309D
:104DE00061F4E091DC07EA930E94B130E091DC07C6
:104DF000EA93EEEFEA9365D96EDDA881AD3409F44C
:104E000066DDA881A43521F4A091D007A23009F075
:104E100001C05FDDA881AB3219F4EEEFEA9327D829
:104E2000A881AD3219F4EFEFEA9321D8A881A73415
:104E300021F4E1E0EA930E94371FA881AB3421F40A
:104E4000ECEFEA930E94371F18C00E94D71A0E9405
:104E5000195DE0E0E093D207A881A13039F40E9407
:104E6000B86B21F0A091810BA03009F402C031DDB4
:104E700004C00E9419100E94C76B219608951A93CE
:104E80000A930E94FA6B0E9471190E948645E030D5
:104E900071F10E94036C58F10E94AC6B21DDE0308F
:104EA00031F50E940B6C0E940E1BEF3F09F0E2C42B
:104EB0000E94106C21F40E94B819E13009F017C06B
:104EC0000E94A719E83119F40E94156C09F001C07D
:104ED000D1C40E940B6CF5D80E2F013021F4A091A3
:104EE000500BA03009F403C01A930E94F511A09151
:104EF0001306AF3F41F110911306EFEFE093130655
:104F00001A930E94B1300E94106C21F40E94B819CB
:104F1000E13009F018C00E94A719E83119F40E9485
:104F2000156C09F001C0A6C41A93EEEFEA93C9D834
:104F30000E2F013021F4A091500BA03009F403C0D2
:104F40001A930E94F51196C40E94D71A0E945D1A06
:104F5000E89421F8E0E0E093D5070E941C6C0E94E1
:104F6000195D0E940D660E940D660E94F45CE0913E
:104F700017060E94AB67E09118060E94AB670E947B
:104F80000D660E94FF650E94F45CE09124060E9479
:104F9000AB67E0911E06F0911F060E949A67089584
:104FA0000E947C760E94FA6B0E948645E03049F0B0
:104FB0000E94036C30F00E94AC6B92DCE03009F48C
:104FC0003DDCE091120CF091130C0E9450680E949D
:104FD0006562E03011F40C944F280E941C6C0E9412
:104FE0000D66E2E0F0E00E947467E0911C06F0912B
:104FF0001D060E949A67E0912006F09121060E940A
:105000009A6700E0033010F00C944F28A7E10A9F44
:10501000F001EC5EF94F9F01F901A381AF3FE9F187
:10502000D9011A960E9498740E94B6737F936F9369
:10503000FF93EF930E94236CAF91BF918F919F914B
:105040000E94B6730E94F973DF01CB010E94286CA5
:10505000D9011C96ED93FC93F90104841584D901C0
:105060001E960E949874E015F105B9F0F9010484C8
:105070001584A685B785F001EA1BFB0BE093630B53
:10508000F093640BDBDBE13041F4D9011C960E9404
:105090009874D9011E96ED93FC930F5FB3CFECC0CB
:1050A0000E947C760E94FA6B0E9471190E948645CC
:1050B000E03011F40C94E6280E9489450E2F0A93E3
:1050C00010DE003820F0A091C105A03808F42BC0F4
:1050D0000F770A930E942F6CFA93EA930E940B3683
:1050E0001E2FA091990BA03011F41F3F09F416C098
:1050F00030E0333098F4ABE03A9FF001E952FA4FD8
:10510000E081E11749F43A9FF001E752FA4FE0815C
:10511000EF5FE093C105232F3F5FEBCF0A930E941F
:105120000B6C2A9352C0A091990BA03021F4003847
:1051300010F0033808F00AC00F770E94DA6A108175
:10514000EFEFEA930E940B6C0A937EDAA091990B21
:10515000A03011F0003808F439C00F770A930E948C
:10516000B130BEDBE03091F50E94326C0E940E1B24
:10517000EF3F09F081C00E94B819E13039F50E9473
:10518000AC19E03049F40E94326C0E946120E0309A
:1051900011F00E94376C1AC00E94A719E83141F43F
:1051A0000E94156C21F00E94326C0E9461200EC09A
:1051B000A091D507E02F0E941067AE0FBF1F1C9172
:1051C0000A930E940B6CEFEFEA933EDAA09113066C
:1051D000AF3F09F100911306EFEFE09313060A9336
:1051E0000E942F6CFA93EA930E940B361E2F0A93AB
:1051F0001A93EEEFEA93EFEFEA9326DA1F3F41F4BA
:10520000A091540BA03021F4A091570BA03009F0CD
:1052100002C00E94376C20FE0AC0E89420F8E0919A
:10522000990BE03019F4CFD31CD501C07ED530E006
:10523000333010F50E943D6CE03031F00E94446C38
:105240000E944D6CE03069F40E943D6CE23041F404
:105250000E94446C0E9450680E946562E03009F42C
:1052600009C0ABE03A9FF001EF51FA4FA0E0A083F4
:10527000689420F83F5FDCCF0E94837624960895DF
:105280000E947A76A091D007A33011F40C94F72AEB
:10529000E091F107ED3411F00C94222AE091F2072D
:1052A000EA3511F00C94D72924FC81C0E091F30772
:1052B000E0532E2FE091F407E0533E2FE5EFF7E0A7
:1052C0000E94526C0E94576CAB3429F40E945D6CB2
:1052D0000E9435580E2F0E94576CA43529F40E9465
:1052E0005D6C0E943558AF01E091840BE31731F5F6
:1052F000E0E0E0930B0C0E94C06B4093DE075093FC
:10530000DF07A091E7070A1759F0E7E0E093CF071E
:105310000093E70720930A0CE0E0E093E6070DC056
:10532000A0910A0C2A1721F0A091E507A03009F0FE
:1053300004C02093CF0720930A0C35C0A091E70743
:10534000A03049F4A091850B0E948A66E255FF4F78
:10535000E491EA2309F40CC0E7E0E093CF0720933F
:105360000A0CE0E0E093E607E091F007E0930B0C15
:10537000E091F007A0910B0CEA17A9F44093DE0727
:105380005093DF070093E7070E94C06BA0910A0CBF
:105390002A1721F0A091E507A03009F004C020935E
:1053A000CF0720930A0C273011F40E941B69E0916B
:1053B000F207E93439F4E7E00E94E66B0E94D36B10
:1053C000E093E607E091F207E23439F4E4E00E946A
:1053D000E66B0E94D36BE093E607E091F207E035BD
:1053E00019F4E1E0E093CF07E091F207EC3449F4DF
:1053F000E4E0E093CF07E091F307E053EA930E94E3
:105400009B16E091F207E334E9F4A091F307A1338E
:1054100020F0A091F307A93308F014C00E94606C3B
:10542000E091D907EA930E943233E091F007EA93C2
:10543000E1EDF9E1FA93EA930E94666C0E94AB7485
:105440000E940A5AE091F107E03521F4A091D007BB
:10545000A13009F003C00E94A66B69DAE091F10760
:10546000EF3459F4E091F207EE3439F4E091F007AB
:10547000EA93E4EDF9E10E946B6CE091F107E3350A
:1054800069F5E091F207EF3349F5A091F307A033F6
:1054900020F0A091F407A03308F420C00E94606CB3
:1054A000E091F407E0531E2FA091D907A13210F428
:1054B0001A3008F013C0103011F40E947932E091D4
:1054C000F007EA93E7EDF9E1FA93EA930E94716C31
:1054D0000E94786C0E94AB740E940A5AE091F10716
:1054E000E33411F00C94BF2AE091F207EF3311F08E
:1054F0000C94BF2AE091F407E03319F4EFEFE09346
:10550000DA07A091F307A033F8F00E94606CA09135
:10551000D907A132C8F4E091DA07EF5FE093DA0728
:10552000E091D907EA93E091DA07EA930E94FC320E
:10553000A091D50BB091D60B109721F4A091DA076A
:10554000A33608F001C0E7CFE091DA07EA930E94A2
:10555000B1300E947D6CEAEDF9E10E94826C0E94FC
:10556000C3680E949E670E94866C0E94CC680E945D
:10557000866C0E948C6C0E9480590E94D259E091E6
:10558000F107E434A1F5E091F207E43481F514E089
:10559000E1E0E093F008103538F40E944D67E151E6
:1055A000F84FE081E03208F41AC00E944D67E151E3
:1055B000F84FE081E33259F40E944D67E051F84F13
:1055C000E081E053EA930E94AB551F5F06C00E9442
:1055D0004D67E151F84F0E948D6A1F5FDCCF0E943A
:1055E0007D6CEDEDF9E10E94826C0E94D25984C479
:1055F0001A930A930E94646A11F40C94642BE0E0FD
:10560000E093170CE091CF07EF770E2F0093CF07B1
:105610000E94195D0E94FF650E9404660E94F45C6E
:10562000013021F0A091D007A13009F00BC0E6EEC7
:10563000F2E00E940966B2D90E946E680E94A545F8
:105640000E94195D073049F40E94D71AE0E0E09308
:10565000D2070E942D120E947522043031F4E0EE30
:10566000F9E10E9409660E94C10E083019F40E94F7
:10567000916C61D1053019F40E94916C65DC0130A8
:1056800039F40E949E6C0093D00751D90E941910E2
:10569000093059F40E949E6C0E9419100A93E1E0AF
:1056A000EA9391DAE1E0E093170C023029F40E94CA
:1056B000916CE1E0EA93C9DB033011F40E941740DA
:1056C0000093D0070E947119A091D007A73011F064
:1056D0000C94132CE091100CF091110C0E94506866
:1056E0000E946562E03021F0A091D207A03009F05D
:1056F0000AC00E94136BE0910C0CA0910806EA17F7
:1057000011F00E9475220E948645E030E9F0E2E047
:105710000E949A6B1A9328DA1D3409F4D8D81D33E5
:1057200099F40E94355CAADAEF3F41F0E3E0E093A0
:10573000CF070E94A16B0E94EC6B06C0E7E8E093E4
:10574000CF07E0E0E093D207A091E607A03031F068
:10575000E091E607A091E507EA1709F455C0E0914A
:10576000E607E150EA930E941D31A091EB0BE1E0C6
:10577000EA23E13021F4E0911006EF7C09F429C01E
:10578000E0E0E093E507E0910A0CE03019F0E093E7
:10579000CF071EC012E0E0911006EC7009F018E08F
:1057A000E0917B0BA091E607EA1781F0E0911006EB
:1057B000E07439F011E0EAE2EA93E5EEF9E10E94E3
:1057C0006B6CE0911006E07809F019E01093CF07B8
:1057D0001BC00E94195D0E942D120E94FF650E944D
:1057E00004660E94F45CEBE4EA930E948A5CE09118
:1057F000E607EA930E94D943E8EEF9E10E940966C0
:10580000E091E607E093E507A091E607A03021F4D8
:10581000A091E507A03009F406C0E0E0E093E507B9
:10582000E7E8E093CF07A091D007A33011F40E94DE
:105830000F3EA091D007A13009F404D9A091D00760
:10584000A23009F41CDBA091D007A83009F428DCB1
:10585000A091D007A53009F4A3DBA091D007A9300F
:1058600049F4E0E0E093D707E091D007EA93E0E065
:10587000EA93A9D90991199108950E94E768EF5612
:10588000F84FA6E0A0830E94E768E057F84FAB818D
:10589000A0830E94E768EA56F84FAA81A0830E947D
:1058A000E768EE56F84FA881B981A083B1830E94C2
:1058B0005E6A0E94E7400C9482300E94A96CA88125
:1058C000B981AC91A53020F0A881B981E0E0EC93DA
:1058D00022960895A091CA07BB27E091C90705C089
:1058E000A091C807BB27E091C707F0E031960E945E
:1058F000426A3596DF01E5E0F0E00E9451740895B8
:105900001A931091CA07E091C907E11791F00E941C
:10591000AF6CE13021F00E94AF6CE23011F4E1E0B5
:1059200050C0EDB7FEB7FA93EA931F93C6DF1F91FD
:10593000EACFE0E046C01A930E94D71AE7EDF5E0FF
:105940000E947569E1E2F0E00E94886910E013307E
:1059500080F4ABE01A9FF001E952FA4FAFEFA08359
:10596000ABE01A9FF001E352FA4F0E94056B1F5FF4
:10597000EECF10E0133048F4A7E11A9FF001E75E84
:10598000F94FAFEFA0831F5FF5CFE0911006E370F2
:1059900019F00E94B86B09F402C0689401C0E89441
:1059A00021F8EFEFE093E407E091990BE03029F460
:1059B0000AD057D1E89420F804C00E94195D0E94D3
:1059C00051101991089522970E947A7600E00330D1
:1059D00058F40E94B66CA0E00E94BC6CE652FA4FEC
:1059E000A0E0A0830F5FF3CF00E00330C0F50E947A
:1059F000DA6AE081EF3F89F10E94DA6AE0810E9471
:105A0000C16CB9F00E94EA6ADF010E9498740E949A
:105A1000F06AEA17FB0751F00E94EA6A0E94F06AF6
:105A2000A083B1830E94C86CA1E0A0830E94B66CE1
:105A300012C0ABE00A9FF001EF51FA4FE081E03075
:105A400061F40E94DA6AAFEFA0830E94EA6A0E94C2
:105A5000056B0E94C86CA1E0A0830F5FC6CF0E94B7
:105A60002F361E2F1F3F11F0E1E001C0E0E0E09370
:105A7000170C1F3F11F40C948F2D50E000E0033001
:105A800048F40E94DA6AE0811E1711F451E002C066
:105A90000F5FF5CF5030E1F500E00330C8F50E940C
:105AA000DA6AE081EF3F91F50E94DA6A10830E9482
:105AB000EA6A0E94F06AA083B183ABE00A9FF0011A
:105AC000E552FA4FA091E00B0E94BC6CE452FA4FF1
:105AD000FF93EF930E94246B0E94336BAF91BF91B1
:105AE000EC930E94C86CA1E0A0830E94B66CA1E078
:105AF0000E94BC6CE152FA4FFF93EF930E945962EF
:105B0000AF91BF91ED93FC9351E002C00F5FC5CF01
:105B1000503029F01A930E9436361E2FAACF30E05B
:105B2000333010F00C94D52DA7E13A9FF001EC5ED4
:105B3000F94FEE83FF8350E000E0033048F550302A
:105B400029F5ABE00A9FF001E452FA4F20812A9335
:105B50000E94B1300E94B66CE081E13059F42A9382
:105B60000E94C819E13031F4A32FAF5FE091540BCC
:105B7000EA1709F00BC0E22FAE81BF811396EC93B8
:105B8000E02FAE81BF811596EC9351E00F5FD5CF2A
:105B9000503049F4AE81BF811396EFEFEC93AE81A4
:105BA000BF811596EC933F5FBBCF0C94AD300E9444
:105BB0007C76AC81BD81EBE4EC93EC81FD81319688
:105BC0000E94CE6CE552FA4FE0810E94D96C00E051
:105BD0000E94E36CEC91E03011F00F5FF9CF0E946E
:105BE000E36CE0E2EC930F5F0E94E96C0E94CE6CE4
:105BF000E352FA4FDF010E9498740E949E670E9450
:105C0000F06CEE81ABE0EA9FF001E452FA4F1081B4
:105C10001A930E94B13000E00E94E36CEC91E030F6
:105C200011F00F5FF9CF0E94E36CE8E7EC930F5F90
:105C30000E94E36CE0E2EC930F5F30E03A3050F406
:105C40000E94E96C0F01A1E4BBE00E94F56C0F5FBC
:105C50003F5FF4CF0E94E36CEC930E94837627961B
:105C6000089564970E947C7600E010E0133058F4A9
:105C7000ABE01A9FF001E952FA4FE081EF3F09F4DF
:105C80000F5F1F5FF3CF033021F0A091E407A03036
:105C900009F406C0E0E0E093E407EA930E946F1184
:105CA00010E0133088F5ABE01A9FF001E652FA4F8E
:105CB000E081E03039F11A9FF001E852FA4FE081BB
:105CC000E030B1F01A93FE0135960E94F56AABE020
:105CD0001A9FF001E452FA4F30813A930E94B1309A
:105CE0001A93FE013596FA93EA930E94A4110AC012
:105CF0001A930E949311ABE01A9FF001E652FA4FFB
:105D0000A0E0A0831F5FCDCF033021F4A091E40772
:105D1000A13009F406C0E1E0E093E407EA930E94B1
:105D20006F110E948376689608950E947A76A091FA
:105D3000990BA23009F4E0C030E0343168F40E94DD
:105D4000FC6C0E94FF6CDA011296E0E0EC93DA0141
:105D5000EFEFEC933F5FF1CF0E942F360E2F0F3FF6
:105D600011F0E1E001C0E0E0E093170C0F3FA1F17A
:105D70000E94246BFA93EA930E9465301E2F1F3F06
:105D800031F1A091D507E12FEA1B3E2F3431F8F411
:105D90000E94FC6C0E94FF6CFA0132960F01E081B8
:105DA000AE2F0E94056DB0E0EA0FFB1FD001EC930F
:105DB000FA01A281A43620F0DA011296E3E6EC9310
:105DC000DA01AC91AF3F19F4E02FDA01EC930A93BA
:105DD0000E9436360E2FCACF0E94C61530E03431ED
:105DE00010F00C947C2F0E94FC6C0E94FF6CFA0156
:105DF000A381AF3F11F40C947A2F0E940A6D0E9488
:105E0000986AE83131F40E940A6DEA9399D0E03043
:105E100009F407C00E940A6DEA9392D0DA01129643
:105E2000EC93A091510BA07839F4FA010280DA01C9
:105E30001196EC91E01509F45DC0DA0113962C91EE
:105E4000ADE02A9FF001E45FFC4F0F01DA011296EA
:105E5000EC91D001EC930E940A6DEA930E94ED1A36
:105E6000EF3F51F0ADE02A9FF001E45FFC4FBF012E
:105E70002A9FF0010E944E6ADA011296EC91E030FE
:105E800089F00E940F6DDF010E94156DEC93ADE06B
:105E90002A9FF001E75FFC4FDF01E0914F0BEF70AD
:105EA000EC9313C00E94156DE03021F40E940F6D39
:105EB000A0E003C00E940F6DA8E0A083ADE02A9F80
:105EC000F001E75FFC4FA7E0A0830E940A6DEA9310
:105ED0000E94ED1AEF3F19F0ECE0E0930A04DA01BA
:105EE0001296EC91DA011196EC932A93E1E0EA9391
:105EF0000E947E5D3F5F73CF0E9481762696089553
:105F0000E7E0E093CF076AD0A8950E948D34A8956A
:105F10000E944C36A895EFEFE093690BE093400B9D
:105F2000E093EA0BE093E50BE09313060E941A6DF1
:105F3000EC7F29F0A8E0B0E0E0E00E94DA74089578
:105F40000E941F6D0E94236D17FD02C0103011F4D6
:105F5000E0E09EC3E12F9CC30E941F6D0E94236D51
:105F600017FD10E01A3008F41F5FE0EAEA930E9480
:105F70005A670E942B6D8CC30E941F6D0E94236D77
:105F800017FD02C0103011F4E0E082C31150E0EAC6
:105F9000EA930E945A670E942B6DE1E079C31A933D
:105FA0000A9310E00E94FA650E947973A8950E94F6
:105FB0008160E03021F4E0EA0E94326D09F002C015
:105FC00001E001C000E00E9492601F5F003011F408
:105FD000153008F001C0E6CFE02F0BC30E94376DEB
:105FE00084C40E94376D0E94446D0895A881B981D0
:105FF0000E94707624F4A83EE3E0BE070CF005C0D2
:106000000E944A6D0E94F46044C3E0E042C3A8814C
:10601000B9810E94707624F4A83EE3E0BE070CF03C
:1060200005C0EA81E03011F4EFEFEA830E944A6D87
:10603000ED81EA930E942061FEC00E947C7620E000
:1060400030E0283EE3E03E077CF4A8953A932A939B
:10605000CDDF1E2F1F3F29F0EFEFEA933A932A93EB
:10606000D6DF2F5F3F4FEDCF0E9483764BC01A9350
:106070000A93E0E0F0E0E093180CF093190CAA8189
:10608000A33668F40E945A670E94536DE55FFD4E87
:106090008F010E94586DE8E1FCE00E94616DE09183
:1060A000180CF091190CC5C01A931FEF1F5F1A93BB
:1060B000DEDFA981BA81EA17FB0711F0143608F078
:1060C00001C0F4CFE12F1881B6C01A930A930E9441
:1060D0006E6AA091D507EA0F0E2F043608F002E68B
:1060E0001091D507101758F41A93C1DFAA81BB810C
:1060F000EA17FB0711F4E12F03C01F5FF3CFEFEFA7
:1061000019810881249608950E947A7610E013364A
:1061100018F50E946666E8E2F0E00E94F473E05031
:10612000FE4EAF01E0EAEA93FA0170960E94656DB7
:10613000EC713E2FE0EAEA93FA013F960E94656D0A
:106140000E2FEF81E31719F4EE81E01709F002C07A
:10615000E12F03C01F5FDBCFEFEF0E94817628960F
:1061600008951A930A93E091400BAA81EA1709F166
:10617000A336A8F40E945A670E94536DE050FE4E69
:106180008F01E0EAEA930E9442681A930A930E9400
:106190008C6C0E944161EA81E093400B0AC0EFEFF2
:1061A000E093400B0E948C6C0E94696DE0E0E093EC
:1061B0004B0B3FC00E946E6D0E94536DE050FE4E2F
:1061C0008F01AA81A33660F4E0EAEA930E94426854
:1061D0001A930A930E948C6CE0E2EA930E94A961F0
:1061E00028C01A930A93E091690BAA81EA17B9F0C3
:1061F0000E945A670E94716D40F40E947B6D0E945C
:10620000616DEA81E093690B0AC0EFEFE093690BDF
:106210000E94A1680E94696DE0E0E093740B09C0E0
:106220000E946E6D0E94716D20F40E947B6D0E9431
:10623000446D19810881239608951A930A93E09179
:10624000EA0BAA81EA1761F10E945A670E94866DE3
:1062500008F50E94586DEBEEFBE00E94616DEA814B
:10626000E093EA0BE0E0E0931006A091EC0BA13084
:1062700020F0A091EC0BA83008F00BC0AFE8BBE019
:10628000E091EC0B0E94BE6AAE0FBF1FEC91E09351
:10629000100606C0EFEFE093EA0BE0E0E093EB0BB3
:1062A000198108810C942D360E946E6D0E94866DB6
:1062B00030F40E94586DEBEEFBE00E94446D1981B2
:1062C00008810C942D361A930A93E091E50BAA816C
:1062D000EA17F1F00E945A670E948E6D70F4E0EAAE
:1062E000EA930E9404661A930A93E6EEFBE00E948A
:1062F000616DEA81E093E50B0BC0EFEFE093E50BF6
:10630000E6EEFBE00E9475690E9404660E94BF628F
:1063100019810881A2C40E946E6D0E948E6D50F496
:10632000E0EAEA930E9404661A930A93E6EEFBE021
:106330000E94446D1981088190C4E6EEFBE00E9442
:1063400075690E9404660E94BF62E881EF5FE09376
:10635000E70BA0C424970E947A76E3EDFBE00E944D
:106360007569E8E0F0E00E948869AA85A33658F5CF
:10637000AB85A13010F0A13208F007C0EB850E9478
:10638000BE6AA3E6B0E00E94966DEB85E030D9F4DA
:10639000E0E0EE83EF83E887E98740E050E020E02B
:1063A00030E02032E0E03E0764F4D901E3E6F0E0BB
:1063B0000E94966D0E94C3680E94AF6D2F5F3F4F91
:1063C000F0CF0E94C46D4AC11A930A93AB81A130E9
:1063D00010F0A13208F01DC0EB810E94BE6AA3E656
:1063E000B0E00E94F473DF010E945A67AE0FBF1F36
:1063F000E8E0F0E00E94F473E050F04D8F01E0EA35
:10640000EA930E94D56D1A930A93E3EDFBE00E9494
:10641000446D198108810C947B360E947C76EC8156
:106420000E94986AE83119F40E94837630C20E9473
:10643000296B309729F00E94296B0E94336BEC8303
:106440000E94AC190E2F10E0101710F00C94763249
:106450000E94DA6D7FDFA5EDBBE00E946868A09125
:10646000D70BB091D80B8091D90B9091DA0B0E9489
:1064700080690E94B6730E948973E093D70BF093F2
:10648000D80B6093D90B7093DA0B0E94DA6D9CDF06
:10649000E0EAEA93EE810E94BE6AEE0FFF1FE05031
:1064A000F04F0E94656DE270F9F4ED81E093DB0B33
:1064B0000E94296B309761F40E9406690E947A69F4
:1064C000EF5EF84DDF010E945D67EA0FFB1F02C01F
:1064D0000E94296BE093DC0BF093DD0BE091DE076B
:1064E000F091DF070E94DF6D1F5FAECF0E948376C1
:1064F000CEC11A930A930E948569ECE2F0E00E94F3
:1065000088690E94666C0E94E56D10E0133608F5FC
:106510001A9327DEE091D907EA931A931BDF0E94B2
:10652000EE6DEA0FFB1F0F010E94EE6D0E94786C6A
:10653000DF01CB01E091D70BF091D80B6091D90B23
:106540007091DA0B0E948973D0010E94A2741F5FC0
:10655000DDCFA091D007A330B9F500E00031A0F560
:106560000E94A3660E94F66D69F510E01A3050F59E
:10657000E02FE05DEA93E6EFF9E10E94FB6DE12F89
:10658000E05D0E94026EE1F40E94076E0E94716C51
:10659000EA0FFB1FFF93EF930E94716C0E94786CCF
:1065A0007F936F93FF93EF930E946458AF91BF91D5
:1065B0008F919F910E948973AF91BF910E94A274A5
:1065C0001F5FD4CF0F5FCACF10E01A3090F40E9443
:1065D000716C0E94786CA091E007B091E107809106
:1065E000E2079091E3070E9489730E94E56D1F5FA7
:1065F000ECCF09911991089524970E947A76EA8543
:10660000EA9335DD9F01022E032A19F13A932A936A
:106610004BDD1E2F40E050E0E0E0EE83EF83E887A3
:10662000E987AA851A1791F4012F033678F40A93A3
:106630001EDD2E173F0741F4EB85EA930A938ADEAD
:106640000E94C3680E94AF6D0F5FEFCF0E94C46DC0
:1066500005C0EB85EA93EB85EA937CDE0E948176A8
:106660002C9608951A93A895A981A13288F4E3ED98
:10667000FBE00E947569E8E0F0E00E94886910E0A4
:10668000133630F4E981EA931A939EDE1F5FF8CF48
:106690001881229608951A9311E0113220F41A936A
:1066A000E1DF1F5FFACFE0C2E1E0E093EB0BE093A4
:1066B000EC0BF0C2A8950E94A168E2E0F3E0FA9327
:1066C000EA930E94D56D0E940A6EE093720B0E94BD
:1066D000136EE093730BE0E0E093740BDBC2A895BC
:1066E000E0E4FBE00E947569E9E2F0E00E9488695D
:1066F0000E948C6CE8EFF2E0FA93EA930E94D56D69
:106700000E940A6EE093490B0E94136EE0934A0BBD
:10671000E0EBE0934F0BBEC20E947A760E941669AE
:10672000E03228F0AEE0B0E0E0E00E94DA7400E091
:1067300055DCA091750BB091760BA633E2E1BE0754
:1067400041F110E01A3030F41A93B4DF1A9368DD87
:106750001F5FF8CF10E0133630F41A93C0DF1A939E
:1067600029DD1F5FF8CF10E0103830F41A939CDF5A
:106770001A939ADD1F5FF8CF8EDFA9E0B0E0E0E06A
:106780000E94DA74E6E3F2E1E093750BF093760B86
:1067900001E010E0183210F00C9434340E944D6780
:1067A0000E941A6E9F010E944D670E941A6EAF01EF
:1067B0000E944D670E94226E3496E491E03011F001
:1067C000E13089F4D901AC910E944D670E94226E9C
:1067D0003596E491EA1730F40E944D670E94226ECC
:1067E0000E94276E3FC0E230B9F4DA010E9498742B
:1067F000E031A7E2FA072CF4DA010E949874FF2333
:1068000052F40E944D670E94226E36960E94A77431
:10681000DA01ED93FC9326C0E33059F4D901AC9131
:10682000AF3F31F40E944D670E94226E0E94276E96
:1068300019C0E430B9F4D901AC91AF3F99F400E04C
:106840000E944D670E94226E3596E4910E1750F417
:106850000E944D670E94226E0E94276E2F5F3F4F5D
:106860000F5FEECF1F5F96CFBCDB10E0133060F4FC
:106870001A9329DDA091E60BA43020F01A935DDD78
:106880001A9349DD1F5FF2CFE02F0E948176269692
:106890000895E881EF5FE883A881A43610F0E0E076
:1068A000E883E881F7C10E942C6E3096F3C1A09175
:1068B000EE0BBB27E091ED0B9AC0F9DF329774F035
:1068C0000E94336EE091ED0B0E943A6E0E94446D7F
:1068D000E091ED0BEA93DDDFE093ED0B08950E946C
:1068E000336EE091EE0B0E943A6EFA93EA930E94A7
:1068F00041610895EBEDFBE00E94426E0E94336E11
:10690000E091EE0B0E943A6E0E94446DE091EE0B16
:10691000EA93BFDFE093EE0B08950E947C76E0E0FF
:10692000E093ED0BE093EE0B10E030E0343680F5B1
:10693000A8950E94336E3A93B6DFFA93EA93EBED93
:10694000FBE00E94616D00E0A091DB0BA13010F034
:10695000A03808F001C001E0E12FE03041F401303F
:1069600029F43093EE0B3093ED0B11E00FC0E130C2
:1069700031F4003019F43093ED0B12E007C0E2302F
:1069800029F4013019F43093EE0B13E03F5FCECFC2
:10699000B0C11A93A091860BA870B9F010E0E981FC
:1069A000FA810E946666AE17BF077CF4ED81E09322
:1069B000DB0BEB81FC81E851FC4F0E94496EE0E06B
:1069C000F0E00E94DF6D1F5FEACF18810C9444391C
:1069D000E881EF5FE883A881A43610F0E0E0E88367
:1069E000E88158C1A091F00BBB27E091EF0BF0E0DC
:1069F00031960E94426AEC59FF4FDF01E4E6F0E075
:106A00000E94517408950E942C6EE050FE4F42C1C6
:106A1000E0EEFBE00E94426EE881EA9335D13AC194
:106A20001A930BDBE1E0E0933D0B1EC1A89510E04B
:106A3000143680F41A9321D1A091E00BAF3F31F4CA
:106A40000E944E6EAF3FEFEFBE0711F01A93E0DFEA
:106A50001F5FEECF0E94536E689420F805C10E941C
:106A60007C761091F00BAD81AA23C2F5E091EF0B7B
:106A7000E11719F0AD81AA230AF02FC01A93FDD0B7
:106A80000E944E6EEE81FF81EA17FB0729F4E8852C
:106A9000A091E00BEA1709F01DC00E94F06AEC819A
:106AA000FD810E948E73EA17FB0754F40E94056D66
:106AB0000E94596E0E944A6BE0E0EC83ED8308C0AF
:106AC0000E94056D0E94596EEC83FD830E940A6B43
:106AD0001A93DAD00E945E6EC9CF48C0E091EF0BE6
:106AE000E11729F0AC81BD810E9470760CF01DC0C9
:106AF0001A93C3D00E944E6EEE81FF81EA17FB0706
:106B000029F4E885A091E00BEA1709F00BC00E9478
:106B1000056D0E94596E0E944A6B1A93B5D0E0E051
:106B2000EC83ED830E945E6ED9CFAC81BD810E9463
:106B300070761CF457DF33970CF418C0E885E093A7
:106B4000E00BEE81FF810E942E6BEC81FD810E94A3
:106B50004A6BE091EF0BEA9397D0E091EF0BEA9349
:106B600037DFE093EF0BE0E0EC83ED83689420F8EF
:106B7000EC81FD810E9483760C94DD381A93A895F0
:106B80001091F00BE091EF0BE117A1F00E94E06A89
:106B900054F4EB81A091E00BEA1729F40E944E6EA9
:106BA0000E94636E09F003C0E12F1881A4C00E9407
:106BB0005E6EE8CFEFEF18819EC00E94F06A0E94DF
:106BC000707684F4E0911006E87031F4E091E60705
:106BD000A091E00BEA1731F40E94246B0E94336B02
:106BE000E33608F002C0E1E00895E0E0089508957A
:106BF000A895E091EF0BA881EA1759F0E8810E946F
:106C0000C16C11F0E88146C0E881EA93E1DEE883D7
:106C1000F0CFEFEF3FC01A93A8951091F00BE091E1
:106C2000EF0BE117C1F00E94E06A7CF4E0911006DE
:106C3000E87031F4E091E607A091E00BEA1729F43F
:106C40000E944E6E0E94636E09F002C0E12F04C0E4
:106C50000E945E6EE4CFEFEF1881239608951A9399
:106C60001091F00B1A93C4DF19910895E881EA930B
:106C7000AFDEE883EA93BCDF0DC00E94336E0E9452
:106C8000686E0E94616D06C00E94336E0E94686E3D
:106C90000E94446D219608950E947C760E94536E56
:106CA00010E030E0343628F5A8953A93E6DF00E0AE
:106CB000A091E00BA03808F401E0E12FE03041F4AE
:106CC000013029F43093F00B3093EF0B11E00FC03B
:106CD000E13031F4003019F43093EF0B12E007C0CB
:106CE000E23029F4013019F43093F00B13E03F5FE8
:106CF000D9CF0E9483762496089524970E947C76AB
:106D00000E948944EAEFF9E10E9475690E942845D2
:106D10000E94C244E091D907E03061F0E5E0FAE179
:106D20000E9475690E942845E091D9070E94716E02
:106D30000E94756E0E94C2440E94793200E00A30BF
:106D4000A0F40A930E94F1300E94A168EFE0EA9358
:106D50000E940245E02FAAE5B6E00E94796E0E94EB
:106D6000786C0E947D6E0F5FEACF0E94D644EEE001
:106D7000FAE1FA93EA93EFE0EA930E9428450E9431
:106D800089680E94DF440E94C2440E94D8440E9445
:106D9000C24410E0103110F00C945F370E94066975
:106DA000E117E9F5E4E1FAE10E9475690E942845DE
:106DB0000E944D67FA93EA930E94756EE0E0E093BB
:106DC000D507A091D507A33640F5E091D907EA93FE
:106DD000E091D507EA930E94FC320E94C368309785
:106DE000C9F0E091D507EA930E94B1300E94C368D0
:106DF000FA93EA930E94836E0E9428450E948C6C4D
:106E0000EAE0EA930E9402450E94CC680E94DF44B7
:106E10000E94C2440E94D768D4CF0E94886E0E940C
:106E20004D670E94F66D11F00C945D37E4E1FAE1D4
:106E30000E9475690E9428450E944D67FA93EA9363
:106E40000E94756E0E948C6EE0E30E94026E29F42F
:106E50000E94076E0E9435589F0100240216030607
:106E600054F50E945D6C0E946458EC83FD836E8330
:106E70007F830E945D6C0E94946E3A932A930E94D5
:106E8000836E0E9428450E94986EEAE0EA930E9471
:106E90000245EC81FD816E817F810E947D6E0E94A2
:106EA0008C6EE1E30E94026E29F40E94076E0E943C
:106EB00035589F01D2CF0E94886E1F5F6BCF0E9412
:106EC0009D440E948376289608950E947C76AD8129
:106ED000BE812C910E949D6E0E944D670E94AB6600
:106EE0000E948F67ECE3EA930E948A5CEC81EA934C
:106EF0000E94E45C2A93ED81EA930E948243EEE3D0
:106F0000EA930E948A5C0E946E6B0E94AB660E94AC
:106F1000746B0E94A26E333409F431E2313320F0F5
:106F2000EC81E05DE31708F407C0E32F0E94B56B26
:106F3000E255FF4FE4912E273D3311F0313209F431
:106F400001C0CACF3D3319F4AD81BE812C93E32F2C
:106F50000E948376279608950E947A7620E0AF817A
:106F6000B8855C910E949D6E0E944D670E94AB6641
:106F70000E948F67E2E0EA930E94E45C5A930E94C9
:106F8000D9430E946E6B0E94AB660E94746B0E9494
:106F9000A26E303310F03A3308F00EC0203009F4FE
:106FA00050E021E0A52FEAE00E944E74AAE0EA9F9B
:106FB000F001E30FE0535E2F3B3211F4533608F03B
:106FC00001C05F5F3D3211F4513008F401C05150EF
:106FD000333429F4203009F431E250E020E03D332D
:106FE00019F4EE81E51708F005C0AF81B8855C9112
:106FF00030E020E03D3311F0313209F401C0B4CF6C
:107000003D3319F4AF81B8855C93D4C00E947A7681
:1070100020E0AF81B8854D915C910E949D6E0E94E9
:107020004D670E94AB660E948F67AE81A23051F41B
:10703000E6E0EA930E94E45CFA010E949E670E94E7
:10704000AF4308C0E5E0EA930E94E45C5A934A9398
:107050000E94BB430E946E6B0E94AB660E94746BE1
:107060000E94A26E303310F03A3308F020C0203076
:1070700011F440E050E021E04031E7E25E0734F0F7
:10708000DA01E0E1F7E20E945174AF01493BEBE025
:107090005E0734F0DA01E8EEF3E00E945174AF01CC
:1070A000DA010E94A76E0E94AC6ED097AD013B3210
:1070B00021F44033E5E75E070CF002C04F5F5F4FFD
:1070C0003D3221F40024041605060CF002C04150A4
:1070D0005040333431F4203009F431E240E050E0E4
:1070E00020E03D3311F0313209F401C098CF3D3337
:1070F00021F4AF81B8854D935C935CC00E947A7691
:107100000E949D6E20E050E04FEF0E944D670E946C
:10711000AB660E947467EF81F885FA93EA93E8857D
:10712000EA930E94B65CE52FE10FF0E00E94AB66A7
:107130000E94746B0E94A26E303310F03A3308F054
:1071400021C03053431729F04F3F09F05F5F20E023
:1071500005C0A22FAF5FEA2FE3702E2FE52FAF817E
:10716000B8850E94B16E0F01E32FA2EFB5E00E9437
:10717000796EAE0FBF1FE22F0E94B16EE491D00175
:10718000EC93432F3B3219F4EE815E1708F002C0F6
:107190005F5F4FEF3D3211F4513008F402C051509F
:1071A0004FEFEE815E1720F4313211F03D3309F4D8
:1071B00001C0ABCFE32F0E948176299608951A93E0
:1071C0000A93A091510BECEDEA231E2F00E00D3045
:1071D00040F40E94B56E0E94B96EE11711F00F5F86
:1071E000F6CF0E94B56EEA0FFB1F0E94A7740E94A3
:1071F0000966E02F3DC4A1E5BBE0E8810E94BE6EB8
:1072000011F4E3E701C0E9E4EA930E948A5C3AC41E
:107210000E947A760E949D6E0E944D670E94AB6626
:107220000E947467CCDF5E2F0E946E6B0E94AB667B
:107230000E94746B0E94A26E3D3211F0363311F43D
:10724000503009F401C051503B3211F0333311F486
:107250005C3008F001C05F5FA091510BE1E0EA23D0
:107260002E2FE52FA0E0B2E00E94796E0E94B96E49
:10727000E20FE093510B3D3311F0313209F401C0BC
:10728000CBCFE32F0E948176269608950E947C76CC
:107290000E949D6E0E944D670E94AB660E947467BB
:1072A0000E94C46EAE0FBF1FEC91E17019F4E1E2D1
:1072B000FAE102C0E5E2FAE1FA93EA930E94A15CE6
:1072C0000E946E6B0E94AB660E94746B0E94A26E5D
:1072D000303310F03A3308F00EC00E94C46EEA0F4B
:1072E000FB1F0F010E94C46EAE0FBF1FAC91E1E007
:1072F000EA27D001EC933D3311F0313209F401C09B
:10730000C9CFE32F0E948376259608950E947C764C
:107310000E94C76E0E94CD6E0E940D660E94F45CB2
:107320000E948C6CEAE0EA93E9DEE13209F45CC485
:107330000E940D660E940D660E94786BE9E2FAE1F8
:107340000E940966ECE4FBE00E9475695FDEE132B1
:1073500009F44AC40E940D660E940D660E94786B73
:10736000EFE2FAE10E940966E0914E0BEF5F0E2F0B
:10737000EDB7FEB7FA93EA930F93EAE0EA93ECDDF8
:107380000F91E13209F430C400240216030624F4FC
:10739000E02FE150E0934E0B0E940D660E940D66B7
:1073A0000E94786BE8E3FAE10E940966E3E6FBE0FD
:1073B0000E94D16E09F418C40E940D660E940D66E9
:1073C0000E94786BEEE3FAE10E940966E5E6FBE0D5
:1073D0000E94D16E09F408C40E940D660E940D66D9
:1073E0000E94786BE4E4FAE10E940966E0E5FBE0C4
:1073F0000E94DA6E09F4F8C30E940D660E940D66C1
:107400000E94786BEDE4FAE10E94096601DFE13247
:1074100009F4EAC310E0133010F00C94C03A0E9453
:107420000D660E940D660E94786BE12F0E947C6BB6
:10743000E3E5FAE10E9409660E94E26E0E94F45CB4
:10744000A4E5BBE00E944D670E94E66E09F4CCC340
:10745000E9E0F0E00E9470660E94F45CA7E5BBE002
:107460000E944D670E94E66E09F4BEC30E940D663D
:107470000E940D660E94786BE12F0E947C6BEEE506
:10748000FAE10E9409661A9301DFE13209F4ACC304
:107490000E94E26E0E94F06E49F40E94756A0E949A
:1074A000B9690E94FA6E09F49FC30AC00E94756A06
:1074B0000E94B9690E947569A9DDE13209F494C39B
:1074C0000E940D660E940D660E94786BE12F0E945B
:1074D0007C6BE0E6FAE10E9409660E94E26E0E947F
:1074E000F45CA0E6BBE0EE27A10FBE1F2C91332772
:1074F000EDB7FEB73197FA93EA933F932F93E0E00D
:10750000EA9384DD2F913F91E13209F46DC3A0E647
:10751000BBE00E944D67EA0FFB1F2083123070F51D
:107520000E940D660E940D660E94786BE12F0E94FA
:107530007C6BE7E6FAE10E9409660E94E26E0E9417
:10754000F45CA7E6BBE0EE27A10FBE1F2C9133270A
:10755000EDB7FEB73197FA93EA933F932F93E0E0AC
:10756000EA9354DD2F913F91E13209F43DC3A7E640
:10757000BBE00E944D67EA0FFB1F20831F5F4BCFCC
:1075800033C30E947C7610E01A930E94F36B0E9432
:10759000CD6E0E940D660E94026F0E94296B0E94B0
:1075A0009A670E940D660E94FF650E94F45C0E942B
:1075B00080690E949E670E9499430E940E6F0E94FC
:1075C000FF650E94F45CE091650BF091660B0E94F0
:1075D0009E670E9499430E940D660E94AD67EEE689
:1075E000FAE10E940966E0914E0B0E94136F0E941F
:1075F0000E6F0E94AD67E3DD0E94C868E091500BFA
:10760000E03029F0E091500BEA930E94D94300E06A
:107610000330C8F50E940D66E02F0E94EE660E94BE
:10762000F45C0E94A56AEA930E94D943EBE2EA93D4
:107630000E948A5C0E94AC6AEA930E94D9430E942D
:10764000C8680E94B36A51F40E94BB6A0E949367A3
:107650000E949E670E94AF43E3E707C00E94BB6A97
:107660000E9493670E949A67E9E4EA930E948A5C09
:107670000E94C8680E94C86AEA930E94DF430E9481
:10768000176F0F5FC5CF0E9489453E2F3B3211F423
:10769000133608F001C01F5F3D3211F4113008F4B9
:1076A00001C011503D3439F41A930E94B1302EDEDE
:1076B0001A930E94DA30313209F066CF95C20E94E7
:1076C0007C7610E00E94195D012F0E940D660E94D9
:1076D0000D660E94F45CE2E7FAE10E94096631E07F
:1076E000363020F5103800F50E940D660E948A663B
:1076F0000E948F671A930E941D31E12F0E94136F21
:107700000E94C868A091EB0BE3E00E941B6FA09160
:10771000EC0BE7E00E941B6FE0911006EA93E8E0B3
:10772000EA930E94824313953F5FDACF0E94C10E15
:107730000E9489453E2F3D34F1F50E94546B102F75
:107740001038C8F51A930E941D310E940D660E94E0
:107750000D660E94786BE6E8FAE10E940966E12F67
:107760000E94136F0E94206F0E94246F0E94F45C9D
:10777000E9E8FAE10E940966EBEEFBE0FA93EA938E
:10778000E3E00E94286F09F42FC20E94246F0E9438
:10779000786BEFE8FAE10E940966ECEEFBE0FA9301
:1077A000EA93E7E00E94286F09F41EC21A930E9430
:1077B00054311F5FC5CF313211F0103808F001C0CD
:1077C00081CF12C20E947C760E94195D0E94CD6E0C
:1077D0000E940D660E94F45CE5E9FAE10E940966E8
:1077E00010E0133008F51A930E9463310E940D6671
:1077F0000E9486670E948F67E12F0E94136F0E948C
:10780000206FE091E60B0E942D6FE091E90B0E9442
:107810002D6FE091E70B0E942D6FE091E80BEA934A
:107820000E94DF431F5FDDCF0E9489450E2F0D347C
:1078300011F00C94613C0E94546B10E0133010F076
:107840000C94613C1A930E9463310E940D660E9461
:107850000D660E94786BE8EAFAE10E940966E12F62
:107860000E94136F0E94206F30E0343028F50E9490
:10787000246F0E94786B0E948A660E94316F0E947A
:10788000A7740E9409660E94D56D0E94FF650E9440
:10789000786B0E948A660E94316F32960E9455670B
:1078A0000E948A660E94316F3596E4910E94286F8B
:1078B00009F49AC13F5FD9CF1A930E948B311F5FA1
:1078C000BDCF92C11A930A930E94C76E00E008329E
:1078D00010F00C94383D0E94860E0E940D660E94A6
:1078E0000D660E94366F0E94226E0E94A774319628
:1078F0000E9409660E94C8680E94D56D0E94FF65BB
:107900000E94366F0E94226E3496E491E038A9F40A
:107910000E9406691E2FEDB7FEB7FA93EA931F93F4
:10792000E0E1EA9319DB1F91E13209F4A1C0E12FF4
:10793000A9E0B0E00E94DA7497C0E238A9F40E948E
:1079400016691E2FEDB7FEB7FA93EA931F93E0E195
:10795000EA9302DB1F91E13209F48AC0E12FAEE025
:10796000B0E00E94DA7480C0E138E1F40E941A6D40
:107970001E2FEDB7FEB7FA93EA931F93E3E0EA9365
:10798000EBDA1F91E13209F473C00E94860E0E9467
:107990001A6DE11731F0E12FA8E0B0E00E94DA742F
:1079A000FFCF62C0E03069F40E94A3660E94226E9D
:1079B00032960E945567E1E00E94286F09F458C092
:1079C00053C0E13079F40E94A3660E941A6E0E94AF
:1079D000AB660E94226E3596E4910E94286F09F4EE
:1079E00047C042C0E23069F40E94A3660E94226E42
:1079F00032960E945567EFE0EA9308DBE132C1F16D
:107A000033C0E330E9F40E94A3660E94226E3596EB
:107A1000E491ABE00E94BE74EA1B0E94716E0E946A
:107A2000FF650E94366F0E941A6E0E94AB660E942C
:107A3000226E3596E491EA9348DAE132C9F014C037
:107A4000E43091F40E94A3660E941A6EE0931F0C2A
:107A5000F093200C0E94AB660E94226E3596E49152
:107A6000EA934CDBE13221F00E94F12F0F5F2FCF20
:107A7000099119910895E8810E947C6BECE2FAE18A
:107A80000E940966219608951A930E94546B10E093
:107A9000133010F00C949C3D0E940D660E940D6600
:107AA0000E94786B1A93E7DFECE0F0E00E947066CA
:107AB0000E94F45C1A939FDB0E94E26E0E94F06EBB
:107AC00049F40E94756A0E94B9690E94FA6E09F42D
:107AD0006CC30AC00E94756A0E94B9690E947569E8
:107AE00095DAE13209F461C3123020F50E940D6687
:107AF0000E940D660E94786B1A93BDDFEBEAFAE1F3
:107B00000E940966ECE0F0E00E9470660E94F45C5E
:107B10000E94176FEAE0F0E00E9470660E94F45C39
:107B2000A7E6BBE00E944D67EA0FFB1F0E94DA6EDA
:107B300009F43BC31F5FACCF38C30E947C7610E0D2
:107B40001A930E94F36B0E94CD6E0E940D660E94F4
:107B5000026F21E000E0033060F50E945067E22FE1
:107B60000E941A6B0A9387DF0E94B36A49F40E944D
:107B7000BB6A0E9493670E949E670E94AF4306C043
:107B80000E94BB6A0E9493670E949A670A9333DB44
:107B90002F5F023060F40E940E6FE22F0E941A6B7A
:107BA0000E94C16A0E94AB670E94176F2F5F0F5F30
:107BB000D2CF0E9489453E2F3B3211F4133608F094
:107BC00001C01F5F3D3211F4113008F401C01150A3
:107BD0003D3439F41A930E94B13056DF1A930E9453
:107BE000DA30313209F0ACCF0E94837624960895C2
:107BF0000E94546B0E940D660E940D660E94F45C08
:107C0000E1EBFAE10E940966E1E0E093D907E9EDD2
:107C1000F7E0FA93EA93E0E2EA939ED90895229777
:107C20000E947A760E9489450E2FE091D207E030BB
:107C300011F00C94C53F0132D1F4E6E7F5E0A091D4
:107C4000F10BB091F20BEA17FB0761F4E7E0E09368
:107C5000CF07EAE2EA93EAEBFAE10E9475690E9433
:107C6000165AE1C1E0E0E093BB050E943A6F0D3384
:107C700031F4E091BB05F0E00E94AE6604910D3452
:107C800041F4EAE2EA93EDEBFAE10E9475690E94A1
:107C9000165A063449F4EEE9F5E0E093F10BF0935F
:107CA000F20BE0E0E093BB05003311F00B3229F456
:107CB000E091BB05EF5FE093BB050D3229F4E09145
:107CC000BB05E150E093BB05013329F491DFED33AF
:107CD00011F40E94416F033321F48ADFED3309F47C
:107CE0000CD8063329F4E0E0E093D9070E947D36F2
:107CF000043329F4E0E0E093D9070E94416FA0919A
:107D0000DB07A13010F40C94593F023311F570DFFA
:107D1000ED33F9F40E944E6F0E2F0D33D1F4E09144
:107D2000D907EA930E94323330E0303190F40E9458
:107D30008A660E94F66D59F4E32FE05DEA93E0EC69
:107D4000FAE10E94FB6DE0E3EA930E94375A3F5F3D
:107D5000ECCF053341F5E0E0E093D9070E944E6F88
:107D60000E2F0D3301F511E01132E8F41A930E9441
:107D7000323330E03031A8F40E948A660E94F66DFA
:107D800071F4E32FE05DEA93E0ECFAE1FA93EA9311
:107D9000E12FE05DEA93E0E3EA930E94375A3F5F08
:107DA000E9CF1F5FE1CF013451F4EAE2EA93E3EC5B
:107DB000FAE10E946B6CE1E0E093CF0734C10A3432
:107DC00009F4BBDE073311F00C94593F0E94195D92
:107DD000E0E0EA930E94160FE1E0E093D307E0E0D1
:107DE000F0E0E093CB07F093CC07E4E1F6E00E94EB
:107DF0007569E5E4F0E00E9488690E945962EE83AB
:107E0000FF830E94526F0E9442680E946562E030C8
:107E1000B1F00E9491120E945962EE83FF83A091FB
:107E2000D00BA03021F00E946A2CE03009F407C08A
:107E30000E94E768EF56F84FAEE00E94ED68E5E07B
:107E4000F0E0FA93EA930E94A54540E050E00E94DA
:107E50009C1BE03868F00E949C1BEF573E2F31308E
:107E600010F0313108F004C0E32F0E945469AF01D3
:107E70005A934A930E944B194093CB075093CC07D7
:107E80000091D605E0E0E093D605013211F00B3207
:107E900009F401C0B6CF0B3221F4E1E0EA930E946D
:107EA000160F013209F0A1CFE0E0E093D307E09391
:107EB000D605A091DB07A23011F00C94BE3F093328
:107EC00009F400DD053409F47DDC033611F40E9469
:107ED000910E083309F455DB023409F4F0DB033466
:107EE000B9F51091F00B0E94195D00E0E091EF0BE5
:107EF000E11711F0063008F01EC00E940D660E94C6
:107F0000A3660E948F671A930E943D361A930E94BF
:107F1000D9430E94C868E091E00B0E942D6FE09168
:107F2000E30B0E942D6F0E94246B0E949A670E94AF
:107F30005E6E0395DBCF0E94C10E0E9489450E2F15
:107F4000013221F0E091EF0BE11709F401C0CBCF32
:107F50000434A1F40E944E6F0E2F0D3379F4A091DA
:107F60008A0BA03021F4A091880BA03029F00E9448
:107F7000BD6B0E940D665FD30E941035E091D20761
:107F8000E03011F40E94480F49C0E130D1F4A091D3
:107F9000D807AB3010F4013209F405C00E944B162B
:107FA0000E94C10E0DC0E0E0E093D5070E94576F1C
:107FB0000E946B6CE0E00E945C6FE2E0E093D2070D
:107FC0002DC0E23059F5013269F4E0E0E093D207C8
:107FD0000E94195DEAE2EA93EDEBFAE10E946B6C14
:107FE0000E94480F0B3211F00D3359F40E94576F65
:107FF000FA93EA93E1E3EA930E94165AE1E00E94C1
:108000005C6F0D3259F40E94576FFA93EA93E2E3E2
:10801000EA930E94165AE2E00E945C6FA091CF079B
:10802000A33009F4FFCD0E948176289608951A9313
:10803000E3E0E093D0070E94195D0E940D660E9464
:108040000D660E94F45CE9ECFAE10E9409660E9468
:108050000D660E94FF650E94F45CE8EFF5E00E9467
:108060007569E0E1F0E00E94886910E0E091800B22
:108070001E1700F50E940669E117D1F0E12FE05DBF
:10808000EA93E1EDFAE1FA93EA93E0E3EA93E0E0C0
:108090000E94026E49F40E944D67E850FA4FA1E039
:1080A000A083E12FE05D01C0EEE2EA930E948A5CCA
:1080B0001F5FDCCF0E943A6FE0E0E093BB05E093E6
:1080C000D2070E94480F71C00E94616FE89422F8A5
:1080D0000E947D6CE2E7EA930E94F558E091F20776
:1080E000EA930E94F558EFE0EA930E94F558A091B8
:1080F000EF07AA3221F41A930E945F4B1BC0A09194
:10810000F2070E944D67E55EF44FE081EA1721F423
:10811000E091F207E03351F40E946666A55EB44F29
:10812000E091F207EC931A930E945F4B22FC02C08D
:108130000E94D2593AC00E94616FE091F207E05369
:10814000AE2F0E944D67E45DF44FE081EA1769F5B8
:108150001A930E945F4BA091ED07A23019F40E9480
:10816000696F09F402C00E946F6FA091ED07A33000
:1081700019F40E94696F09F402C00E946F6FE0E079
:10818000E093ED07E093230C0E944D67E45DF44F0C
:10819000BF010E944D67E45DF44FE081EF5FAE2FB9
:1081A000EAE00E944E74DB01EC9319910895E88196
:1081B000E03029F4E0E3EA930E94F55806C0E88134
:1081C000E8500E94716E0E9425590C9487440E94C9
:1081D0007A7625FC2DC20E94696F11F40C946B42D3
:1081E0000E94756FE057F84F9F01D9011196EC91ED
:1081F000E43041F50E947B6FF901A681A03021F4A3
:10820000A281B381109709F007C0EAEDFAE10E945C
:10821000826C0E94956F15C00E94996F0E949C6F9E
:108220000E94A06FEDEDFAE10E94826C0E94A36FA4
:108230000E94A96FF901A085B185BA93AA930E9403
:10824000255914C0E730C9F40E947B6FE0EEFAE1D3
:108250000E94826C0E94A36F0E94A06FE3EEFAE17D
:108260000E94826C0E949C6F0E942559D9010E9435
:10827000AF6F0E94817626960895E93089F40E94B6
:108280007B6FE6EEFAE10E94826C0E94B56F0E945D
:10829000A06FD9010E94AF6F0E9481760C94C545F2
:1082A000E63031F5EAE2EA930E94B759E9EEFAE1E5
:1082B0000E94826CD901EC910E94B86FE091840B0E
:1082C0000E94B86FEBE4EA930E94F5580E949C6FFD
:1082D0000E942559E4E5EA930E94F5580E94A36F95
:1082E0000E94BC6F0E946F6F0E9481760C94C545FE
:1082F000E53021F50E94236CF096EA930E94B7596D
:10830000E2E7EA930E94F558D901EC91EA930E94C2
:10831000F5580E94C06F0E949C6F0E94A06FE7ED0D
:10832000FAE10E94826C0E94A36F0E942559D90134
:108330000E94AF6F0E9481760C94C545E83031F5FC
:108340000E947B6FECEEFAE10E94826CF901A6813B
:10835000AA930E942F6C309719F00E94296B04C0D9
:10836000D9011696EC91F0E0FA93EA930E94255910
:108370000E94956F0E94D259D9011196E0E0EC93CA
:108380000E946F6F0E9481760C94C545E130B1F573
:10839000A091D007A53029F4E091840BE65F1E2F51
:1083A00001C011E0E12F0E94C56F0E944D670E943D
:1083B000CD6F0E94C06F0E949C6F0E94A06FEFEE75
:1083C000FAE10E94826C0E94A36F0E94A96FD901FA
:1083D0001796EC910E94716E0E942559A091D007CA
:1083E000A53041F40E94D16FA481B581BA93AA93BC
:1083F0000E948C590E94D76F0C94C545E330B9F4A4
:108400000E94236CF0960E94E86F0E94236C0E94E9
:10841000CD6F0E94EF6FE2EFFAE10E94826C0E9442
:10842000A36F0E94BC6F0E94F36F0C94C545EB30A4
:1084300071F50E9402700E9405700E94EF6FE5EFD7
:10844000FAE10E94826CF901A681AA93B0DE0E9433
:10845000D16FA781AA93ABDE0E94D16FA085B185B1
:10846000BA93AA930E94A96F0E94A36F0E94A96F5A
:10847000F901A481B581BA93AA930E94A96F0E94C1
:10848000B56F0E94BC6F0E94F36F0C94C545EC3031
:1084900091F40E9402700E9405700E94EF6FE8EF55
:1084A000FAE10E94826C0E94B56F0E94BC6F0E942C
:1084B000F36F0C94C545EE3071F40E9402700E9477
:1084C00005700E94EF6FEBEFFAE10E94826C0E9450
:1084D000D76F0C94C5450E94097061F0A091ED071B
:1084E000A03041F4A091890BA13021F40E940669CB
:1084F000E13009F427C0A0913C0BA03041F0E0919D
:108500003E0BF0913F0B0E944D6CE130D9F4E1E35A
:108510000E94E86FE0912D0B0E94B86F0E94EF6FF0
:108520000E940669EA930E940C4BE093ED070E94BB
:10853000D2590E945962E093210CF093220CE0E0A2
:10854000E0933C0BA091ED07A03051F0E091210C9D
:10855000F091220C0E9450680E946562E13009F09F
:1085600025C0A091ED07A23019F40E94696F09F4AB
:1085700002C00E946F6FA091ED07A33019F40E9412
:10858000696F09F410C0A091230CA33030F00E9451
:108590006F6FE0E0E093230C06C00E94756FEF560A
:1085A000F84FA8E0A083E0E0E093ED07A0913D0B39
:1085B000A130F1F5E091F00BA091EF0BEA1799F1E2
:1085C000EAE20E94E86FE0912B0B0E94B86F0E94D4
:1085D000EF6FE091F00BEA930E943D360E94996F95
:1085E000E091E00B0E94716E0E94A06FEEEFFAE145
:1085F0000E94826C0E94246BFA93EA930E94A96FF6
:108600000E94056D0E940F700E94D259E091F00BFC
:10861000EA930E940835E091F00BEA930E94E83457
:10862000E093F00B05C0E0E0E0933D0B689420F888
:108630000E948176AAC21A930A930E946A2CE030A3
:10864000D9F00E94E768E057F84F8F01EC81FD8177
:10865000D8011296ED93FC93EA81FB81D80118961C
:10866000ED93FC93EE81D8011696EC93D801119608
:10867000E4E0EC930E945E6A198108810C942D4617
:10868000E881E03011F40E941270A881A13021F439
:10869000EAE1F6E00E941970A881A23021F4E6E236
:1086A000F6E00E941970A881A33021F4E4E3F6E01B
:1086B0000E941970A881A43021F4EAE3F6E00E9438
:1086C000197025C10E94127008951A930A93E0E070
:1086D000E0937805E093790510E0143190F400E020
:1086E000033068F4A3E01A9FF001E158FA4FDF016C
:1086F000EE27A00FBE1FE0E2EC930F5FF1CF1F5FEC
:10870000ECCFE2C31A9311E0E981E11788F00E94EF
:108710004D67E255FF4FE491AA81EA2319F0E12F5A
:10872000E05D01C0E0E2EA930E948A5C1F5FECCF4B
:108730003AC12A97A091D20BA13040F0EA85FB857F
:108740006C857D850E94AB740AD008C00E941E70A3
:108750000E9422700E941E700E94925C44C12A975F
:108760000E941E700E942D700E9436700E941E7022
:108770000E94925C38C12A970E941E700E94497024
:108780000E94F06C0E941E700E94925C39C12A9770
:108790000E941E70EDE1FBE1FA93EA93EE85FF85FE
:1087A0000E949E670E94F06C0E941E700E94925C64
:1087B00027C12A970E941E70E0E2FBE105C02A97BC
:1087C0000E941E70E4E2FBE1FA93EA93EE850E94B8
:1087D000D96C0E941E700E94925C2B9608950E9494
:1087E0007C7610E0E1E3E093EF08E89431F8EA9357
:1087F0000E94B759E8E2FBE10E94826C00E0E09140
:108800007D050E17E0F40E94A366E158FA4FE0815F
:10881000E03258F4E3E2EA930E94F5580E94A3661E
:10882000E158FA4FE081E05D05C00E94A366E1587F
:10883000FA4FE081EA930E94F5580F5FE0CF0E9463
:10884000D2590E9459629F010E94CD153A932A93F2
:10885000E8ECF0E00E94CF6B0E2FA0E031FCA1E02D
:10886000A03011F4003009F001C0EECF31FE07C096
:10887000E0E0E0937D05E89431F8E1E007C01F5F98
:10888000123008F4AFCFE0E0E0937D050E948376DC
:1088900024960895E0917C05E03021F4E881EA9384
:1088A0000E94AB55A0917C05A13079F4A0E092998B
:1088B000A1E0A13031F4A8950E9447680E94797325
:1088C000F5CFE881EA930E944857A0917C05A23039
:1088D000F1F4E0917D05F0E0E158FA4FA881A08322
:1088E000E0917D05EF5FE0937D05E0917E05EF5F10
:1088F000E0937E05A03218F4EF5FE0937E05A0912F
:108900007E05A83320F06BDFE0E0E0937E05219642
:108910000895A091800BA13020F0E2E0E0937C0567
:108920000BC0E1E0E0937C05E0919A00EF76E093E4
:108930009A00E3E3E093990008950E94886E0E94F4
:10894000886E20D0EBE1EA93A5DFE9E6EA93A2DFA7
:10895000A0917C05A13051F40E945368E0919A00E7
:10896000E069E0939A00E9E1E0939900A0917C0529
:10897000A23021F434DFE0E0E0937E05E0E0E09314
:108980007C050895EDE0EA9385DFEAE0EA9382DF73
:1089900008951A9310E0E9811E1728F4EA81EA93FA
:1089A00079DF1F5FF8CF188123960895EDE201C0AB
:1089B000EDE3EA93E8E2EA93ECDFE4DF08952A9737
:1089C000A091D20BA13038F00E941E700E942D7031
:1089D0000E94367004C00E941E700E942270FE0128
:1089E0000E9475690FD02E9608952A970E941E70D6
:1089F0000E9449700E94F06CFE010E94756902D0CD
:108A00002C9608951A930A9310E0EA81E03011F44D
:108A100008E201C00A81AB81BC81EE27A10FBE1F15
:108A2000AC91A03011F0101708F007C0AB81BC81E9
:108A30000E9451700E945670EECFEA81E03039F00A
:108A4000EA811E1720F4E0E20E945670F9CF27C099
:108A50001A930A9310E0EA81E03011F408E201C0B1
:108A60000A81E12FAB81BC810E94B16EE491E030BC
:108A700011F0101708F009C0E12FAB81BC810E94F2
:108A8000B16EE4910E945670ECCFEA81E03039F08B
:108A9000EA811E1720F4E0E20E945670F9CF198196
:108AA000088125960895E091BF05A091BE05EA17BB
:108AB000C1F00E945B700E94B169EC91E093C10526
:108AC0000E945B700E94B969E181E093C005A091AA
:108AD000BF05AF5FEAE00E944E74E093BF05E1E09E
:108AE0000895E0E008950E946170A981A0830E942A
:108AF00061703196A881A083A091BE05AF5FEAE0C6
:108B00000E944E74E093BE050C945D4BE091D60537
:108B100008951A93E091D605E03059F40E94CD15DE
:108B20000E94646A21F4A091D605A03009F001C02A
:108B3000F5CF1091D605E0E0E093D6050E94646A77
:108B400009F011E2E12F0C94D14A0E947C760E9438
:108B500059628F010E94CD15EC81FD81E00FF11F5C
:108B6000FF93EF930E945962AF91BF91AE1BBF0B71
:108B70009D010024021603061CF40E94646A09F099
:108B800001C0E8CFE0E00E948376269608951A930C
:108B90000E944A69E050FD4FA0E0A0830E944A690C
:108BA000E55FFC4F108117FF05C0E12F0E94677041
:108BB000A0E0A08316FF05C0E12F0E946E70A0E028
:108BC000A0830E944A69E55FFC4FA0E0A0830E9459
:108BD0004A69E65FFC4FA0E0A0830C945C4B0E94C6
:108BE0007C7630E0EE81ADE0EA9FF001E55FFC4F7E
:108BF000108116FF17C0E12FEF730E2F0E947570C2
:108C000011F03A3008F009C00E947D70DF010E9427
:108C10008A660E9483703F5FF1CF0E947D700E9440
:108C2000AC6EEC9317FF17C0E12FEF730E2F0E946D
:108C3000757011F0343108F009C00E948970DF01AD
:108C40000E948A660E9483703F5FF1CF0E94897004
:108C50000E94AC6EEC930E94837627960895A097AD
:108C60000E947A76EDA5FEA5A9A9BAA9EA0FFB1F75
:108C7000AF01E0E0F3E0EE83FF8310E01431C0F5D4
:108C8000AE81BF81AC91A03049F1EE81FF81A3811B
:108C9000B481EFA5F8A9EA17FB0701F5EE81FF8182
:108CA000A181B281E9A9FAA9AE17BF07BCF0EE8194
:108CB000FF81A181B2814A175B0784F00E948F7007
:108CC000AE0FBF1FE9A9FAA9AE17BF073CF00E947B
:108CD0008F70AE0FBF1F4A175B070CF402C01A93C8
:108CE00056DFEE81FF813D96EE83FF831F5FC6CF87
:108CF000E0E0F3E0EE83FF8310E0143110F00C9419
:108D00002447AE81BF81EC91E03011F00C941D47F7
:108D1000EAA5EC93E9A9FAA9AE81BF811196ED937A
:108D2000FC93EFA5F8A9AE81BF811396ED93FC9358
:108D3000EDA5FEA5AE81BF811596ED93FC93EBA545
:108D4000AE81BF811796EC93E0910404A0910A04D0
:108D5000EA27AE81BF811896EC93E0910B04AE81B7
:108D6000BF811996EC93E0910C04AE81BF811A96F5
:108D7000EC93AE81BF811B960E9401671C96E0E0D8
:108D8000EC93E887E8A5F9A5309741F00E949A7026
:108D90000E949F70E4E1EA930E941E63EEA1FFA18E
:108DA000309751F00E949A70E8A5F9A5FA93EA93DA
:108DB000E4E1EA930E940A63E0E0EC8F0E949A707B
:108DC0000E94F5623E2F3B30C8F000E00E9489709F
:108DD000E081E03011F0053008F002C00F5FF6CFFF
:108DE0000E948970E081E03049F40E9489700E94FD
:108DF000A470E058AE81BF811B96EC93E0E0EA8B53
:108E00003130C8F000E00E947D70E081E03011F068
:108E1000043108F002C00F5FF6CF0E947D70E08140
:108E2000E03049F40E947D700E94A470E05CAE8145
:108E3000BF811B96EC93E12F08C0EE81FF813D9628
:108E4000EE83FF831F5F59CFEFEF0E948176E39699
:108E500008951A930A930E94AF703097A9F1E09198
:108E60005D05E03061F50E94AF70049000925D05F1
:108E7000E0915D05E03031F4E0E0F0E00E9419702F
:108E8000E0E01AC00E94B4700E94AF700E94A77404
:108E9000F595E7958F01D801E0E0F1E00E941F749D
:108EA000E0938700D801E0E0F1E00E945174E09384
:108EB00086000E94B470E0E4E0938B0005C0E0916E
:108EC0005D05E150E0935D050991199108950E94B7
:108ED0007C7600E020E033E010E01431B8F5D901F1
:108EE000EC91E03079F111960E9498740E94BC7068
:108EF00024F5D90113960E949874AC81BD81EA17BC
:108F0000FB07DCF4F90101801280D90115960E945B
:108F10009874E00DF11DAE81BF81AE17BF076CF4F0
:108F2000F90103801480D9011796EC910E946A6AB6
:108F3000AC81BD81AE17BF070CF004C0E12FEF5F1D
:108F40000E2F04C0235F3F4F1F5FC7CF003049F093
:108F5000E0915E05E01721F0A0915E05A03009F4D4
:108F600001C022C0A0915F05A53079F40A93E1E029
:108F7000EA93B9DD00935E0500936005D901EC9199
:108F8000E0936105E3E0E0935C05A0915F05AE31FD
:108F900019F4E4E0E0935C05A0915C05A33018F0BF
:108FA000E5E0E093630507C0E0E0E0935F05E09350
:108FB0005C050E94C1700E94837628960895E09116
:108FC0005E05E03091F0A0915F05A93220F4EA93AC
:108FD000E2E0EA9388DDA0915F05AD3330F0E091E7
:108FE0005E05EA93E4E0EA937EDDE0E0E0935C0571
:108FF000E0935F050E94C170E0E0E0935E05E093BE
:10900000620508950E94195D60DB0895E981EBBB5C
:10901000E7E1E09365001F98E6E1E0936500E7E192
:10902000E0936500E881EBBBEFE1E0936500EEE1E2
:10903000E0936500EFE1E09365001F9A0C945D4BAF
:109040001F9808951F9A08950E9447680E94797397
:10905000EBE1E0936500EAE0F0E00E940269EFE1F5
:10906000E09365000E94A3670E947973E1E0EA93B0
:10907000E2E0EA93CBDF0E942E6621F4E2E0EA937D
:10908000E2E403C0E2E0EA93E2E8EA93BFDFE7E06C
:10909000EA93EFE7EA93BADFE8E0EA93E7E1EA93DD
:1090A000B5DF0E94C770E1E2EA93E8E8EA93AEDF39
:1090B000E2E2EA93E3E3EA93A9DFE3E2EA93ECEC8A
:1090C000EA93A4DFE4E2EA93ECECEA939FDFE5E2C3
:1090D000EA93EBEBEA939ADFE6E2EA93EBEBEA93AF
:1090E00095DFE7E20E94CD70E8E20E94CD70E9E2F0
:1090F0000E94CD70E5E0EA93E8E0EA9387DFE6E0DE
:10910000EA93E7ECEA9382DFE0E0F0E00E94D270BD
:10911000E0E0F0E0E0935A05F0935B050E9477668B
:10912000E3E00E947D66E0E0E0930D04EDE0E09373
:109130000E04089521970E947A764A85EF810E9455
:10914000D7700E94A7748F01E0E1EA93EF85EA935C
:109150005DDFE2E1EA93EB85FC85AF85B889EA0F34
:10916000FB1FEA9353DFE9E00E94DB70E1E1EA9341
:109170000E94E070EA0FFB1FEA9348DFE9E1EA93FF
:10918000EF850E94E5700E94DB705ADF2EE13FE11F
:10919000E0E0EE83E885F985AE81B0E0EA17FB07F1
:1091A0009CF050E0451760F01BBB209365003093A6
:1091B00065000BBB20936500309365005F5FF2CFC5
:1091C000EE81EF5FEE83E6CF0E942248E0E10E944D
:1091D000EA70E2E1EA93EFE9EA930E940648E9E0E7
:1091E0000E94EA70E1E1EA93EFE7EA930E94064801
:1091F0000C94004A0E947A76EE810E94D7700E94F9
:10920000A7748F010E94E070EA17FB0739F4EF8121
:10921000F885AB85BC85AE17BF070CF023C0E7E12E
:109220000E94EA70E7E10E94EA70E9E1EA93EE85C4
:109230000E94E5700E94EF702EE13FE15B854F8157
:10924000451760F01BBB20936500309365000BBB96
:1092500020936500309365005F5FF2CF0E94224843
:109260000E94C7700E94E070AE17BF073CF4EF8108
:10927000F885AB85BC85EA17FB0709F01BC0E9E15F
:10928000EA93EE850E94E5700E94EF702EE13FE1C7
:109290005D854985451760F01BBB209365003093C1
:1092A00065000BBB20936500309365005F5FF2CFD4
:1092B0000E9422480E9481762F96089524970E944A
:1092C0007A76EB85F0E0EE0FFF1F0E94A273E8872D
:1092D000F98730910804EA850E94D7700E94A7742C
:1092E0000E94AB731E2FEA850E94D7700491E0E0C4
:1092F000EF83AF81A03110F00C94004AE0E0EE83E0
:10930000E0910904AE81AE1710F00C94F649E8E143
:109310000E94DB7040E0423010F00C94EC49E42FE6
:10932000EE0FEE0FEE0FE39FF001AE85BF85F0E08C
:10933000EA0F5E2FE42FA885B9850E94B16EEC5824
:10934000F94F2491203011F40C94E94927FF3BC0D8
:10935000E9E1EA935A930E9406481F98EFE1FEE183
:109360000BBBF0936500E09365001BBBF0936500B9
:10937000E093650031FF0AC00BBBF0936500E093FA
:1093800065001BBBF0936500E093650026FF1AC0E3
:109390000BBBF0936500E09365001BBBF093650089
:1093A000E093650031FF0BC00BBBF0936500E093C9
:1093B00065001BBBF0936500E09365005F5F220FC3
:1093C0005F5FE4CF1F9A220F31FD5F5F5F5F0C94F8
:1093D000A2494F5F0C948B49EC85FD853196EC8753
:1093E000FD87EE81EF5FEE830C948049E885F98577
:1093F0003296E887F987EF81EF5FEF830C94794924
:109400000E9481766096089523970E947A76A895A7
:10941000E9850E94D7700E94A7740E94AB730E2F3B
:10942000E9850E94D770149130910804E0E0EF8341
:10943000EA85AF81AE1710F00C94A64AE0E0EE8307
:10944000E0910904AE81AE1710F00C94A14AE8E156
:109450000E94DB70E0E0E887EB85A885AE1710F08E
:109460000C94974AE885F0E00E94A473DF010E9403
:109470008A660E94F473AE85BF85EA0FFB1FAF01B9
:10948000E889F98924913196E88BF98B203011F421
:109490000C94924A27FF3DC0E9E1EA934A930E9467
:1094A00006481F98EFE1FEE10BBBF0936500E093E7
:1094B00065001BBBF0936500E093650031FF0AC0B7
:1094C0000BBBF0936500E09365001BBBF093650058
:1094D000E093650026FF1CC00BBBF0936500E09392
:1094E00065001BBBF0936500E093650031FF0CC085
:1094F0000BBBF0936500E09365001BBBF093650028
:10950000E09365004F5F5F4F220F4F5F5F4FE2CFE9
:109510001F9A220F31FF02C04F5F5F4F4F5F5F4FB7
:109520000C94464AE885EF5FE8870C942C4AEC855A
:10953000FD853196EC87FD87EE81EF5FEE830C941D
:10954000204AEF81EF5FEF830C94184A0E948176E6
:1095500062960895E091F90AEA930E94F558E09125
:10956000FA0AEA930E94F5580895F4DF0E94F67013
:109570000E94F670E881F9810E940F709EC01A93D4
:109580000E9435581E2F103021F0E12FE150E0935A
:10959000F70AE0DFE091F70AEF5F0E94716E0E9428
:1095A000A06F199108950E947C7631E00E94576C5B
:1095B000A03320F00E94576CA43308F028C030E09C
:1095C0000E940071E270E6951E2F0E940071E1700A
:1095D0000E2FA091110B1A1729F4E1E0EA27E0936E
:1095E000110B31E0A091120B0A1729F0E1E0EA27F4
:1095F000E093120B31E0E091120BEE0FE05DA091D1
:10960000110BEA0FEA930E94F5580E945D6CE32F5C
:109610000E948376249608951A9310E00E940970A0
:1096200011F40C94594B0E946F34ECE2FBE10E9460
:10963000826CE091DB0B0E94716E0E94A06FEFE2E2
:10964000FBE10E94826CE091DE0BF091DF0B0E9447
:109650000F70A091DC0BB091DD0BA031E7E2BE07EB
:109660004CF4E2E3FBE10E94826CE091DC0BF091B0
:10967000DD0B18C0E5E3FBE10E94826C0E942967C4
:10968000A4E6B0E00E94F473A091DC0BB091DD0B76
:10969000EA0FFB1F0E94496EE091DC0BF091DD0B9D
:1096A000E051F742FA93EA930E9425590E94956F80
:1096B00011E00E940671E12F1881229608952497E7
:1096C0000E947A760E9406710E94DF57E13010F402
:1096D0000C944A4EE091F90AEB3441F4E091FA0A15
:1096E000E33219F40E9435581E2FD1C2E435B9F483
:1096F000E091FA0AE33221F40E943558EE83FF83A9
:10970000E091FA0AEF3451F40E9435581E2F1A9353
:10971000EF81F885FA93EA930E940730B8C2E234E9
:1097200011F00C94DF4CE091FA0AE13259F4AA8569
:10973000AF3F31F40E94BD6B0E940D660E941B4337
:109740000E941035E091FA0AE134E1F40E943558A4
:109750001E2F113071F4A091ED07A13019F40E9471
:10976000097009F402C00E947A34E0E0E0933C0BF7
:1097700009C0E1E0E0933C0B0E945962E0933E0B8C
:10978000F0933F0BE091FA0AE534A9F4E8E3FBE13A
:109790000E94826C0E945734F3973CF00E94355827
:1097A0000E94496E0E940D7101C0E0E3EA930E949D
:1097B000F5580E94956FE091FA0AE634E1F40E94B0
:1097C000197119F40E943558AF01E885F9850E9496
:1097D000336B0E2F033620F0A0918A0BA13021F4B9
:1097E0000E9425710E942F35AA85AF3F21F40E9467
:1097F00025710E941B43E091FA0AE23511F00C94A6
:109800009C4C0E94197119F40E943558AF0130E048
:10981000A0918A0BA03021F40E940669E13009F082
:1098200027C00E94702CE03011F10E943E6BE55A77
:10983000F84FA885B985A083B1830E943E6BEF598C
:10984000F84FDF01EA850E945A6A0E943E6BE15A96
:10985000F84F10830E943E6BE05AF84F40830E94FD
:109860003E6BE65AF84FA1E0A0830E94446B62C0B1
:109870000E946A2CE23010F40C949A4C1A930E94C5
:109880002D710E94BE353E2F3F3F29F00E94F06AA5
:10989000A417B5070CF412C00E94056DE41BF50B6C
:1098A0000E944A6B0E94FF6A19F4E0E0E093E00B2B
:1098B0003A930E944436689420F803C0E0E0E887B9
:1098C000E9870E94E768E057F84FDF01EA85F0E09A
:1098D000E55EF44FE081EC930E94E768EE56F84FA6
:1098E000A885B985A083B1830E94E768E856F84F40
:1098F000DF01EA850E945A6A0E94E768EA56F84F3B
:1099000010830E94E768EF56F84FA5E00E94ED68CB
:10991000E885F985309771F01A930E942D71FA014C
:109920000E948E73FA93EA930E941B430E94257152
:109930000E94C934689422F8E091FA0AE335F1F5FF
:109940000E943558E887F9870E94756FEF56F84FE7
:10995000E081E23089F40E94756FE856F84F00808C
:1099600011800E9406690E940B6AEA17FB0721F426
:10997000A091ED07A23009F01FC00E94756FEE564E
:10998000F84FDF010E949874DF01E885F985EA1736
:10999000FB0779F40E94756FE656F84FE081EA9371
:1099A0000E94756FE057F84FE081EA930E946120B2
:1099B00003C0E7E0E0930906689422F868C1E43444
:1099C00011F00C944A4DE091FA0AE33559F4EBE3B7
:1099D000FBE10E94826C0E94D1550E94B86FE1E0C9
:1099E000E093F008E091FA0AE03511F00C94494D4B
:1099F0000E943271E03011F40C94494D20E00E9435
:109A0000576CA03240F00E94576CA23221F00E94A5
:109A1000576CAB3309F43DC0E22FE03061F40E9493
:109A2000576CA33211F421E005C00E940071EA9343
:109A30000E94AB552BC0E13049F40E94576CA43210
:109A400011F422E001C020E010E020C0E23011F06B
:109A5000E330E1F40E940071EA930E943162EF3F2B
:109A6000A1F0E12FE295E07FEF930E940071EA936D
:109A70000E943162AF91EA0F1E2F2F5F243021F434
:109A80001A930E94AB5520E001C020E00E945D6C5B
:109A9000B6CFFDC0E33411F00C94B44DE091FA0A56
:109AA000E534B9F4E8E3FBE10E94826C0E9457348C
:109AB000F3974CF00E943558E05FF84D0E94496ED4
:109AC0000E940D7101C0E0E3EA930E94F5580E94E4
:109AD000956FE091FA0AE634A9F441E050E00E9463
:109AE00035580E2F0E943671E13019F40E94355816
:109AF000AF011A930E94A366E05FF84D0E943A718D
:109B00000E942F35E091FA0AE335A1F40E943F71DB
:109B10000E94986AE83141F4E091400BEA930E9478
:109B2000AC2F689420F806C0E885EA93EFEFEA933B
:109B30000E946120E091FA0AE134A9F4EEE3FBE12E
:109B40000E94826C0E943F71EA930E94B1300E9491
:109B50009D1FE03011F0E1E301C0E0E3EA930E94D1
:109B6000F5580E94956F93C0E63511F00C941F4E86
:109B7000E091FA0AE33411F00C941E4E0E9435581D
:109B80001E2F113010F40C941E4EA091D007A1305E
:109B9000C1F50E943671E03021F0A09159061A17E4
:109BA00009F02EC011500E943558AF011A930E943F
:109BB000381B3E2F0E94806B0E94B9690F010E94E2
:109BC000806B0E949367E40FF51FD001ED93FC9327
:109BD0000E943671E03089F00E943558AF010E9432
:109BE000896B0E94B9690F010E94896B0E9493677B
:109BF000E40FF51FD001ED93FC931A930E944D12D0
:109C00001DC01630D8F41150A12FEAE00E94FE7357
:109C1000A3E2EA9FF001E15AF94FBF01A12FEAE068
:109C20000E944E74F0E0BB01AAE0B0E00E94CC7349
:109C3000DB01AE0FBF1F14960E94216928C0E934D2
:109C400031F5E091FA0AE03551F40E9435581E2FA3
:109C5000E0E0EA931A930E948430E0931306E091C7
:109C6000FA0AEC34A1F40E94F957E0930D060E9421
:109C70003671E03021F00E94F957E0930E060E9401
:109C80003671E03021F00E94F957E0930F060E94F0
:109C900093571ACD0E9481762B960895A0910F0BB1
:109CA000A03521F4A091100BA33608F005C0E09177
:109CB000100BEA930E94DA30A0910F0BA33521F428
:109CC000A091100BAA3008F005C0E091100BEA93A8
:109CD0000E941031A0910F0BAB3421F4A091100B16
:109CE000A03808F005C0E091100BEA930E945431AF
:109CF000A0910F0BA63521F4A091100BA03108F014
:109D000005C0E091100BEA930E948B31A0910F0BDC
:109D1000A43511F40E94F12FA6D60895EAE5F6E0E5
:109D2000FA93EA93E091F90AEA93E0E8F0E00E94FE
:109D3000886908950E944671A0E0A083E091F70A27
:109D4000E093100BE091F90AE0930F0B08950E9445
:109D50007A760E94DF57E13010F40C94BC51E09108
:109D60000F0BA091F90AEA1709F098DFE091F90AC0
:109D7000E33239F5E091FA0AEC3431F4CFDFE4E074
:109D8000E093CF070E944C71E091FA0AE435C1F4E8
:109D9000C5DFE091260CE03029F0EF77A9E0B0E0D4
:109DA0000E94DA74E091270CE03029F0EF77AEE002
:109DB000B0E00E94DA740E944C71E7E0E093CF07B4
:109DC00002C0EB34E1F5E091FA0AE13211F4A6DFCA
:109DD00035C0E53211F462DF31C0E33299F40E94FC
:109DE000527121F00E945D710E941D310E944671E6
:109DF000E081EB3429F4E0E0E093EB0BE093EC0B33
:109E000099DF1CC0E134D1F40E9435589F012093A2
:109E1000EB0B0E94637191F00E9435589F01A09155
:109E2000EB0BF901E270F070EA2BE093EB0B0E9470
:109E3000637121F00E943558E093EC0B9AC2E33530
:109E400081F5E091FA0AE13211F468DF29C0E332CA
:109E500099F40E94527121F00E945D710E94F130CC
:109E60000E944671E081E33529F4E091F70AEA9314
:109E70000E945A335FDF14C0EE3491F40E94946E56
:109E800010E01A3068F4AAE6BBE0EE27A10FBE1F6F
:109E90000E944D67E550F54FE081EC931F5FF1CFD5
:109EA00068C2E63511F00C949D4FE091FA0AE13258
:109EB00011F434DF41C0E33299F40E94527121F071
:109EC0000E945D710E9463310E944671E081E63517
:109ED00029F4E091F70AEA930E949D312BDF2CC010
:109EE000E63531F40E9435589F012093E70B24C0DA
:109EF000E53471F40E9435589F012093E60B0E94CF
:109F0000637129F00E9435589F012093E90B14C01A
:109F1000E43591F440E050E00E9435589F01022E54
:109F2000032A11F042E050E00E94637119F00E9490
:109F30003558AF014093E80B1CC2E43511F00C9486
:109F40007250E091FA0AE33231F40E9435583197A9
:109F5000E093F70AC6C0E03511F00C94715010E0A0
:109F60000E94576CA03250F00E94576CAD3331F014
:109F70000E94576CAB3311F01E3008F00DC00E94E8
:109F80004D67E550F54F0F010E940071D001EC9331
:109F90001F5F0E945D6CE4CF0E944D670E94697153
:109FA000EDE30E946E7111F00C947150E4E5E093C2
:109FB0000F0B10E00E944D670E94226E3496E491D0
:109FC000EF3F11F40C947150EBEFFAE00E946667DA
:109FD0000E94226E0E9455670E94CD62E03011F00F
:109FE0000C946F500E944D670E94226E3496E4914B
:109FF000E03851F40E943558E058FF4FE093260CAA
:10A00000E0E8E093270C6BC0E23839F40E94355841
:10A01000E058FF4FE093270C62C0E13839F40E940A
:10A020003558A8E0B0E00E94DA7459C0E03011F071
:10A03000E13061F40E944D670E941A6EFF93EF9326
:10A040000E943558AF91BF91EC9349C0E23069F45A
:10A050000E944D670E941A6EFF93EF930E9435583D
:10A06000AF91BF91ED93FC933AC0E33061F40E944D
:10A070004D670E941A6EFF93EF930E941658AF919E
:10A08000BF91EC932CC0E43051F50E944D670E94C3
:10A09000226E3596E491EA930E94CC580E944D6757
:10A0A0000E941A6EE093240CF093250C00E00E94AD
:10A0B0004D670E94226E3596E4910E1780F40E943F
:10A0C000A366E550F54FE081A091240CB091250CDA
:10A0D000EC93A4E2BCE00E9468680F5FE8CF1F5FCA
:10A0E00069CF47C1E03511F00C94B951E091FA0AFB
:10A0F000E33299F40E94527121F00E945D710E9436
:10A10000B1300E944671E081E03529F4E091F70A10
:10A11000EA930E946F330EDE2CC1E13211F4FEDDB2
:10A1200028C1E134D1F40E9435581E2F00E00D30D3
:10A1300098F40E94B56EEA0FFB1F3396E491E11785
:10A1400049F40E94B56E0E94B96EA091510BEA2BA2
:10A15000E093510B0F5FEBCF0CC1E63559F5E0E012
:10A16000E093F80AA4E5BBE00E947371FF93EF93BC
:10A170000E943558AF91BF91EC93EBE2EA930E94B5
:10A18000A657E03059F0A7E5BBE00E947371FF933A
:10A19000EF930E943558AF91BF91EC930E94767176
:10A1A000A091F80AA33018F40E94637109F401C069
:10A1B000D9CFDFC0ED34D1F4E0E0E093F80AA0E6B7
:10A1C000BBE00E947371FF93EF930E943558AF91EB
:10A1D000BF91EC930E947671A091F80AA33018F415
:10A1E0000E94637109F401C0EACFC3C0E735D1F41E
:10A1F000E0E0E093F80AA7E6BBE00E947371FF93EA
:10A20000EF930E943558AF91BF91EC930E94767105
:10A21000A091F80AA23018F40E94637109F401C0F9
:10A22000EACFA7C0E434C9F5E0E0E093F80A0E9461
:10A2300035589F01E2E0EA930E94B257AF01E3E78D
:10A240000E946E7159F40E947C71BF01D9010E9475
:10A25000556AE40FF51FDB01ED93FC93E9E40E94DE
:10A260006E7179F40E947C7120833183A1E5BBE09B
:10A270000E9473710F01A1E5BBE00E9483710E94EF
:10A280008C6B0E947671A091F80AA33018F40E949A
:10A29000637109F401C0CBCF6CC0EE3499F40E9415
:10A2A000946E10E01A3068F4A1E4BBE0EE27A10F31
:10A2B000BE1F0E944D67E550F54FE081EC931F5F94
:10A2C000F1CF57C0E33449F40E9432710E943558EF
:10A2D000E0934C0BF0934D0B4CC0E33589F40E9496
:10A2E00035589F0100240216030624F42B30E0E0C9
:10A2F0003E070CF004C0F9013197E0934E0B39C0D2
:10A30000E53529F40E943558E093500B32C0EF3404
:10A3100091F40E9435581E2FECE2EA930E94A65752
:10A32000E12FE295E07FEF930E943558AF91EA0F5D
:10A33000E0934F0B1EC0E035E1F4E0E0E093F80A53
:10A34000A3E6BBE00E9483710E94B969FF93EF937B
:10A350000E94AC58AF91BF91ED93FC930E9476712F
:10A36000A091F80AA23018F40E94637109F401C0A8
:10A37000E7CF0E949357EDCCE0E0E093FA090E940A
:10A380008176269608950E947C760E94DF57E13000
:10A3900010F40C946654E091F90AE332A9F4E091C8
:10A3A000FA0AE03519F4E1E4FBE109C0E83419F4F4
:10A3B000E2E6FBE104C0E33531F4EDE7FBE1FA93BB
:10A3C000EA930E94055980C2E43511F00C9474524E
:10A3D000E091FA0AE43221F40E944268C6D883C0B0
:10A3E000E33211F4CCD87FC0E03511F00C947352F5
:10A3F000B1D8A091F70AA83210F00C9473520E94C1
:10A4000087710E9455670E940559EDE3EA930E9407
:10A41000F5580E9487713496E491E03839F40E942F
:10A4200006690E94716E0E9425595DC0E23839F4B8
:10A430000E9416690E94716E0E94255954C0E1382D
:10A4400039F40E941A6D0E94716E0E9425594BC00A
:10A45000E03011F0E13041F40E948B71E0810E9404
:10A46000716E0E9425593FC0E23041F40E948B7109
:10A47000DF010E9498740E948F7135C0E33039F477
:10A480000E948B71E081EA930E9435592CC0E43020
:10A4900051F50E948B71E093240CF093250C10E091
:10A4A0000E9487713596E4911E1790F40E944D67C3
:10A4B000E550F54F0F01A091240CB091250CEC91C3
:10A4C000D001EC93A4E2BCE00E9468681F5FE8CF73
:10A4D0000E9487713596E491F0E00E9469710E94B4
:10A4E000986E0E948059F0C1E33579F5E091F70A42
:10A4F000EA930E94F130E091FA0AE43229F4EAE0AA
:10A50000F0E00E94937120C0E33211F438D81CC0EF
:10A51000EE34D1F41FD810E01A3068F40E944D6771
:10A52000E550F54F0F01AAE6BBE00E945170D00143
:10A53000EC931F5FF1CFE0E0E093050B0E94986E73
:10A540000E9480590E94956FBFC1E63511F00C94AE
:10A55000E652E091F70AEA930E946331E091FA0A29
:10A56000E43229F40E9450670E94B54A2EC0E332BB
:10A5700019F40E94BF4A29C0E53459F40E94AA4A3E
:10A58000E091E60B0E94716E0E949771E091E90BD9
:10A5900019C0E63529F40E94AA4AE091E70B12C0DF
:10A5A000E43599F40E94AA4AE091E80BE03011F0FA
:10A5B000E1E301C0E0E3EA930E94F5580E949D7137
:10A5C000E091E80BF0E00E940F707EC1E03511F0E1
:10A5D0000C943154E091F70AEA930E94B130E09173
:10A5E000FA0AE43229F4E3E6F0E00E94937138C1FC
:10A5F000E33219F40E94BF4A33C1E13411F00C94E4
:10A6000043530E94AA4A12E0A091510BECEDEA23B9
:10A610003E2F00E00D3078F40E94B56E0E94B96EB6
:10A62000E31739F40E94B56EEA0FFB1F33961491BD
:10A6300002C00F5FEFCF0E944D670E940F70E09144
:10A640004F0BE03089F0E8E9FBE10E94826C0E9448
:10A65000156D0E94716E0E949771E0914F0BEF7023
:10A660000E94716E0E94A06FE091500BE03051F09B
:10A67000EBE9FBE10E94826CE091500B0E94716E4D
:10A680000E94A06FEDC0E43479F50E94A171A09101
:10A69000F80AA33040F5E091F80AE03011F00E948A
:10A6A0009D71A1E5BBE0E091F80A0E94BE6E61F4E5
:10A6B000AAE5BBE00E9483710E949367FA93EA9334
:10A6C0000E948C59E3E709C0AAE5BBE00E948371B0
:10A6D0000E9493670E948F71E9E4EA930E94F55803
:10A6E0000E947671D4CFB8C0ED34C1F40E94A1713C
:10A6F000A091F80AA33088F4E091F80AE03011F054
:10A700000E949D71A0E6BBE00E9483710E94A77128
:10A710000E9425590E947671EBCF9EC0E735C1F4A7
:10A720000E94A171A091F80AA23088F4E091F80A81
:10A73000E03011F00E949D71A7E6BBE00E9483719A
:10A740000E94A7710E9425590E947671EBCF84C0A8
:10A75000E63521F50E94A171A091F80AA330E8F432
:10A76000E091F80AE03011F00E949D71A4E5BBE091
:10A770000E9483710E94A7710E942559EBE2EA931F
:10A780000E94F558A7E5BBE00E9483710E94A77163
:10A790000E9425590E947671DFCF5EC0EE34D1F45D
:10A7A0000E94AA4A10E01A3068F40E944D67E550F2
:10A7B000F54F0F01A1E4BBE00E945170D001EC9372
:10A7C0001F5FF1CFE0E0E093050B0E94986E0E94BE
:10A7D000805942C0E33499F40E94AA4A0E94986EBC
:10A7E000E3EAFBE1FA93EA930E94296B0E949E67D9
:10A7F0000E94F06C0E94986E0E9480592DC0E03536
:10A8000099F40E94AA4A0E948069FA93EA930E94EE
:10A81000A3590E949D71E091650BF091660BFA932C
:10A82000EA930E94A35918C0E33531F40E94AA4A62
:10A83000E0914E0BEF5F0DC0EF3491F40E94AA4AF5
:10A840000E94156D0E94716E0E949771E0914F0BEE
:10A85000EF70F0E00E948F71EBE3EA930E94F558ED
:10A8600033C0EB3489F5E091F70AEA930E941D3179
:10A87000E091FA0AE43229F4E0E8F0E00E949371F2
:10A8800023C0E33219F40E94BF4A1EC0E134E1F450
:10A890000E94AA4AA091EB0BE1E0EA230E94716EAC
:10A8A0000E949771A091EB0BE3E0EA230E94716E86
:10A8B0000E949771E091EC0B0E94716E0E942559E5
:10A8C000E6EAFBE10E94826C2ED35FCD0E94067106
:10A8D000AEC21A930E94916AE7EFF8E00E94526CB0
:10A8E0000E9406710E94AB71E181E43471F40E9410
:10A8F000AB7102800E940669E05DE01529F00E94BC
:10A90000AB71E281EA3209F401C057C00E94B07114
:10A910000E94AB71E1810E94B4710E94AB71E2812F
:10A920000E94B4710E94BA711C910E94AB7133965F
:10A930000E94526CE12FE23131F40E94BF71E6E0D7
:10A94000EC9305DA3AC0E13131F40E94BF71E2E1E3
:10A95000EC9319DD32C0EF30A9F40E94BF71EEE034
:10A96000EC930E94D34AE13039F4A091EC07A03077
:10A9700019F00E94097009F402C00E947A340E9402
:10A98000C5711BC0EE30C9F40E94BF71EFE0EC93BB
:10A990000E94D34AE13089F4A091EC07A03019F06D
:10A9A0000E94097009F402C00E947A34E0E0E0934A
:10A9B000EC07EFEFEA930E945F4B53C01A930E949B
:10A9C0007D6C0E94076EEAE7EA930E94F5580E94A8
:10A9D000BA7111971C91E12FE23131F4E6E0EA936C
:10A9E0000E94F558B4D937C0E13131F4E2E1EA937D
:10A9F0000E94F558C8DC2FC0EF3099F40E94EF6F29
:10AA00000E94D34AE13039F4A091EC07A03019F04C
:10AA10000E94097009F402C00E947A340E94C57134
:10AA20001AC0EE30C1F4EFE0EA930E94F5580E949C
:10AA3000D34AE13081F4A091EC07A03019F00E94D4
:10AA4000097009F402C00E947A34E0E0E093EC0758
:10AA5000EA930E945F4BA091EF07AA3211F00E9487
:10AA6000D25919910895EFEFE0930F0BE093100B7B
:10AA70000895AC81A03310F0AA3308F006C00E94FC
:10AA8000CC71E0530E94D47198C2AC81A13410F013
:10AA9000A73408F006C00E94CC71E7530E94D4711D
:10AAA0008CC2A881B981E0E0EC9387C2AA93EA93B3
:10AAB000FA93EFB7EA931A930A931BB10CB1E091A2
:10AAC000600CF0E0E25DF34F0083A091600CAF5F9B
:10AAD000A093600CA23319F4E0E0E093600C0991BC
:10AAE0001991D0C10A921A92FA926A937A938A9330
:10AAF0009A93AA93BA93EA93FA93EFB7EA930E94D0
:10AB0000D97149F0A091F008A03021F00E941B0EED
:10AB1000E13009F401C011C0E091C70CF0E0EE593A
:10AB2000F34FE081ECB9A091C70CAF5FA093C70CC5
:10AB3000A43619F4E0E0E093C70CE991EFBFF99176
:10AB4000E991B991A9919991899179916991F99036
:10AB50001990099018951A930E94D97159F45D9B28
:10AB600009C0A091F008A13021F40E941B0EE03032
:10AB700009F013C01091C60C0E944D67EE59F34FB7
:10AB8000A981A0831F5F143609F410E0E091C70C7F
:10AB9000E117E1F31093C60C02C0E981ECB918810A
:10ABA000E4C30E94D97121F40E941B0EE13009F028
:10ABB00001C01BC21CC2AA93BA93EA93FA93EFB7DF
:10ABC000EA931A930A9310919B0000919C00E12F45
:10ABD000EC71A9F4E091900DF091910DE853F34FD1
:10ABE0000083A0E9BDE00E946868E83CA0E0FA07A5
:10ABF00031F4E0E0F0E0E093900DF093910D0991D5
:10AC00001991E991EFBFF991E991B991A99118953D
:10AC10001A930E94DF710E94E471D9F30E94DF71E0
:10AC2000E853F34F1081A2E9BDE00E946868E83C58
:10AC3000A0E0FA0731F4E0E0F0E0E093920DF09349
:10AC4000930DE12F2AC50E94DF710E94E47109F083
:10AC5000CCC1CDC10E947C76F6DFE03021F0A0911E
:10AC6000290CA03009F0E3C0D3DF1E2FA0919C0D6A
:10AC7000A53618F0E0E0E093960D3091960DE09146
:10AC8000960DE03059F4113019F4E4E0E093960D9C
:10AC90001A3519F4EAE0E093960DC1C0E430C1F42E
:10ACA000E0E0E093960D1A3229F00E940669E05D1B
:10ACB000E11769F41093EF071093970DE5E0E09327
:10ACC000960DE0E0E093290CE1E0E093990DA7C038
:10ACD000E530A9F4E0E0E093960D0E940669E05D9E
:10ACE000E11761F00E94EB710E94F471E091990DFF
:10ACF000EF5FE093990DE6E0E093960D90C0E630AB
:10AD000091F4E091990D0E94F4710E94EB71EF5F54
:10AD1000E093990DE0E0E0939A0D133019F4E7E029
:10AD2000E093960D7CC0E73011F0E83059F41A93A7
:10AD3000EAE9FDE0FA93EA93E6E9FDE0FA93EA93A3
:10AD400098DE6DC0E93081F4E0E0E093960D1731B4
:10AD500031F4E0919A0DA091970DEA1709F003C024
:10AD6000E4E5E093290C5BC0EA3041F4103011F4C3
:10AD7000EBE001C0E0E0E093960D51C0EB3071F4E0
:10AD8000E0E0E093990D1093980D1093970DECE08F
:10AD9000E093960DE0E0E093290C41C0EC3091F592
:10ADA0000E94F97110830E94EB71EF5FE093990D9F
:10ADB000E091980DE150E093980DA091980DA0308E
:10ADC00021F4A091970DA03009F00FC0EDE0E093C1
:10ADD000960DE091990D0E94BE6AE950F74FA0E0F0
:10ADE000A0830E94F971A0E0A083A091980DA030EB
:10ADF00021F4A091970DA03009F403C0E0E0E093A6
:10AE0000960D0DC0ED3059F4E0E0E093960D1D3045
:10AE100031F4EAE5E093290CEFEFE093280CE091A0
:10AE2000960DE31719F0E0E0E0939C0D15CF0E941A
:10AE3000837624960895AA93EA93FA93EFB7EA9358
:10AE4000E0919E0EA0919D0EEA1791F0E091EE0721
:10AE5000E03019F0E89426F80AC00E94FF71F0E093
:10AE6000E030A1E0FA0719F4E0E0E0939E0E03C0A1
:10AE7000E89425F826F8E091280CE03019F0E0E09D
:10AE8000E093960DE991EFBFF991E991A991189599
:10AE90001A93E0919E0EA0919D0EEA1721F4E09185
:10AEA0009B00E072C1F4E0919D0EF0E0E356F24F9A
:10AEB000A981A08310919D0E1F5F0E946666A0303D
:10AEC000E1E0BE0709F410E0E0919E0EE117E1F326
:10AED00010939D0E03C0E981E0939C00188145C248
:10AEE000E0E0E0939E0EA0919D0EA13020F00E9424
:10AEF000FF71689426F80895AA93BA93EA93EFB77E
:10AF0000EA93E091280CE03041F4E0E0E0939E0EFB
:10AF10000E940669EF5FE093EE07E991EFBFE991C8
:10AF2000B991A99118950E94576CA03220F00E9407
:10AF3000576CAB3309F403C00E945D6CF4CF0E94E0
:10AF4000576CAB3311F40E945D6C08950E94576CEE
:10AF5000E881EA1729F40E945D6C3197E1E0E0C4D2
:10AF6000E0E0DEC40E947C7600E010E0EEE20E94A9
:10AF70006E7101F520E030E0EC81D901F0E0AE1710
:10AF8000BF07C4F4D8010E94A76E8F010E94576CBE
:10AF9000A03320F00E94576CAA3308F008C00E942A
:10AFA00000710E94B56B0E0F1F1F0E945D6C2F5F1A
:10AFB0003F4FE2CFF8010E948376259608950E94C4
:10AFC000576CA03228F00E94AB71E181E03208F4A6
:10AFD0000EC00E940071E093F90A0E945D6C0E940D
:10AFE0000071E093FA0A0E945D6CE1E00895E0E0F0
:10AFF00008950E940D720E940071EA930E943162CE
:10B00000EF3F91F0F8010E94A273FF93EF930E942B
:10B010000071EA930E943162AF91BF910E94B16EBC
:10B020008F010E945D6CE7CFF80112C31A930A9357
:10B0300010E00E94BA710C910B3311F0003208F449
:10B0400012C0013310F0093308F007C0E02F0E944E
:10B05000B56BE255FF4FE4911E2B0E945D6C0E9480
:10B06000BA710C91E9CFE12FF3C20E947C7600E027
:10B0700010E00E94576CAD3221F40E945D6C31E00B
:10B0800001C030E00E94576CA03320F00E94576C42
:10B09000AA3308F00DC0D8010E94A76E0F010E94CC
:10B0A0000071E0530E946A6A8F010E945D6CEACFD2
:10B0B000303021F4F8010E948376B9C4F8010E946F
:10B0C0008E730E948376B3C424971A93E0E0E983D9
:10B0D000EA83EB83EC830E94576CAD3221F40E942B
:10B0E0005D6C11E001C010E00E94576CA03320F0AD
:10B0F0000E94576CAA3308F021C0A981BA818B81C4
:10B100009C81EAE0F0E060E070E00E94F9737F93D8
:10B110006F93FF93EF930E940071E053AF91BF9143
:10B120008F919F91FF27662777270E948973E98374
:10B13000FA836B837C830E945D6CD6CF103029F438
:10B14000E981FA816B817C81D6C4E981FA816B81C6
:10B150007C810E949273CFC40E947C7686DF8F012F
:10B1600020E030E0EEE20E946E7111F47EDF9F017C
:10B17000112322F4F9010E948E739F01A091D20B3A
:10B18000A13030F0D8010E94556AE20FF31F8F0101
:10B19000F8010E9483764BC41A9310E00E9432712A
:10B1A000E030E9F00E94576CA03258F00E94576CD2
:10B1B000A23239F00E94576CAB3319F0E9811E17A7
:10B1C00008F00DC00E944D67E550F54F0F010E9439
:10B1D0000071D001EC931F5F0E945D6CE3CF0E9471
:10B1E0004D670E9469711881C0C0E8810E94B471E6
:10B1F000E881A091130BEA0FE093130BE881A09173
:10B20000140BEA27E093140B8BC31A9310E0E12F81
:10B21000A981BA810E94B16EE491E03049F0E12F3A
:10B22000A981BA810E94B16EE4910E941272EFCF9F
:10B2300085C31A9310E00E941772E03029F00E9433
:10B2400017720E941272F7CF79C364970E941E7022
:10B250000E941A72E88DF98D0E949E670E94F06C20
:10B260000E941E70E6DF669608951A93ECE3EA9357
:10B27000BCDF11E0193080F40E944D67E255FF4FAA
:10B28000E491A981EA2319F0E12FE05D01C0E0E239
:10B29000EA93ABDF1F5FEECFEEE3EA93A6DF188100
:10B2A00064C064971A930E941F720E941A72EA8DFA
:10B2B000FB8D0E949E670E94F06C0E941F720E948C
:10B2C000F5621E2FED891E1720F4E0E30E94127232
:10B2D000F9CF0E941F72ADDF188110C064970E94E1
:10B2E0001E700E941A72E88DF98D6A8D7B8D0E9406
:10B2F000AB740E94F06C0E941E709BDF68960895EC
:10B30000E2E2EA9372DFE881F981FA93EA9391DF4E
:10B31000E2E2EA936ADF29C0A881B981E4E6F0E0BD
:10B320000E941F740E948F71EEE2EA935EDFA88193
:10B33000B981E4E6F0E00E945174FA93EA93E2E006
:10B34000EA93AFDF12C0A091D20BA13030F0E881B8
:10B35000F981FA93EA93E0DF08C0E881F9810E945D
:10B360008F71E4EBFBE10E94826C2296089525FE2A
:10B3700006C0E5E0F0E00E940269A895F8CFEDE98B
:10B38000FDE0E093150BF093160BE1E0EA932DDF5F
:10B39000E0E0E093130B0E9424720E9406690E9471
:10B3A000B86FBEC21A930A93A091800BA03021F40B
:10B3B0000E940669E03009F001C04AC1E091280C02
:10B3C000E03009F045C1E3E0EA930FDFE091130BB1
:10B3D000E295EF70EA930E9448621E2FE091130BF2
:10B3E000EF70EA930E9448620E2F1A93FEDE0A93D2
:10B3F000FCDEE7E1EA93F9DEEDE9FDE0A091150B53
:10B40000B091160B0E94BB74EA1BE0939D0E6894EA
:10B4100025F81EC1EE81EA93AADFEC81FD810E942E
:10B42000826C0E9428725ADFBDDF1DC2EB81EA9355
:10B430009EDF0E949169E9DE0E942472B3DFF7C2A9
:10B44000ED81EA9394DFEB81FC810E94826CEA81BA
:10B45000EA93CBDEE981E03011F0EA93C6DEE881C1
:10B46000E03011F00E9424729DDF269608950E941C
:10B470007A7610E0E8EBFBE1A885B985EA17FB07CF
:10B4800019F444E150E002C048EC50E0EA85E09352
:10B49000EF08E89431F8EA930E942D71EA85EA9367
:10B4A000EA85EA93E0E0EA93CBDF0E9459629F01CC
:10B4B0000E94CD150E942F720E9465620E2F31FCF2
:10B4C00002C0003009F001C0F3CF31FE04C0E8949F
:10B4D00031F8E1E004C01F5F1230C0F2E0E00E94EA
:10B4E00081762B9608951A930A93E091F709E0303C
:10B4F00009F4AEC0E0E0E093F008E2E0EA932BDB71
:10B5000010E003E00E944D670E94347271F00E94C7
:10B510004D67E950F64F0E948D6A0E944D67E950D1
:10B52000F64FE0810E271F5FEDCFE3E0EA9313DBD8
:10B53000E02FE295EF700E943972E02FEF700E94C9
:10B540003972E7E1EA9307DB83C01A930A93E0912B
:10B55000F709E03009F47CC00E941669E03021F060
:10B56000E091F909EA3209F405C00E941669E05D2C
:10B57000E093F909E0E0E093F008EAE5EA93EBDA1A
:10B58000E0E0EA93E8DA10E00E944D670E9434722E
:10B5900011F01F5FF9CF1F5F012F0A93DCDA10E073
:10B5A0000E944D670E94347271F00E944D67E9500D
:10B5B000F64F0E948D6A0E944D67E950F64FE08178
:10B5C0000E0F1F5FEDCFE02FE195EA93C4DAEDE0B7
:10B5D000EA93C1DA3DC01A930A93F894E0E0E0934D
:10B5E000EE07E0919E0EE0939D0E7894E091F709AE
:10B5F000E03071F1EAE5EA934BDCE0E0EA9348DC05
:10B6000010E00E944D670E94347211F01F5FF9CF65
:10B610001F5F012F0A933CDC10E00E944D670E94DF
:10B62000347279F00E944D67E950F64FE081EA9359
:10B630002FDC0E944D67E950F64FE0810E0F1F5F2F
:10B64000ECCFE02FE195EA9323DCEDE0EA9320DCF8
:10B650000991199108951A930E94916AE091F20755
:10B66000EA93C3DDE4E4EA93C0DDE091F007EA93F6
:10B67000BCDD14E00E944D67E151F84FE081E430F9
:10B6800040F00E944D67E151F84FE0810E94127234
:10B69000F1CFE0E0EA93A9DD58DF19910895DADAF5
:10B6A000A091290CA43529F4A0E025FCA1E0A0304C
:10B6B00009F03AC0E091F107E03581F4E091F2073A
:10B6C000EA93E6E0EA930E947345A091F207A0385E
:10B6D00020F0E091F207E093600523C0E03721F409
:10B6E000E0E0E09360051DC0EA3519F40E94DE54E5
:10B6F00018C0EA3711F4AFDF14C0E23519F40E9424
:10B7000064400FC0E23719F40E949B400AC00E94B7
:10B710004029E091F007A091EF08EA1711F468942E
:10B7200031F8E0E0E093290CA091290CAA3531F41E
:10B730000E94695450DFE0E0E093290C0C9495607E
:10B74000A0912C0CA13050F0E0912C0CE150E09332
:10B750002C0CE03019F4E1E0E0932D0CA0E025FC86
:10B76000A1E0A13049F4A0E026FCA1E0A03021F442
:10B77000A091EE07A03009F001C0B2DBE091EE0726
:10B78000E03019F0E150E093EE070895E0919C0D50
:10B79000EF5FE0939C0DE0912B0CEF5FE0932B0C9F
:10B7A000E091280CE03019F0E150E093280C089566
:10B7B000A0919B0BA13021F0A0919B0BA23029F40A
:10B7C000E3E0E0939000E8E3E9B90895EA81E093CB
:10B7D0007A05E881E0937B05E0910504E061E09360
:10B7E000050425C10E947A76A0917A05A43120F43F
:10B7F000A0917B05A33008F034C0E0917A05F0E019
:10B80000ACE0B0E00E94F4738F01E0917B05F0E0C2
:10B81000A4E1B0E00E94F4739F010E943F72ECE04B
:10B82000F0E00E944472F0E00E94A2730E94A867B8
:10B83000EE81E030B1F0E0917A05A3E0EA9FF001FB
:10B84000E158FA4FDF01E0917B05F0E0AE0FBF1F3A
:10B850004C9155270E943F724A93E0E0EA930E9480
:10B860005E490E94817627960895E0910504E07173
:10B8700041F0E2E0EA93B6DFE0910504EF7EE09369
:10B88000050408950E944972AF39E0E0BE0744F410
:10B89000A091F50BB091F60BAF37E0E0BE070CF0CE
:10B8A00037C00E944E720E94DA6D0E945E49A091DC
:10B8B0005805B0915905549734F4A0915A05B091A8
:10B8C0005B0513970CF012C0E0915805F0915905F3
:10B8D000A3E0B0E00E94CC73E158FA4FA0915A0562
:10B8E000B0915B05EA0FFB1FA981A083E0910804DA
:10B8F000ACE0EA9FF0010E9449720E94B16E0E9482
:10B900005B72E0915805F091590531960E94D27012
:10B910000C94F260E881EA93E0910B04EA93B2DFC1
:10B92000219608951A9310E00E941772E03031F0CA
:10B930000E941772EA93EEDF1F5FF6CF18812396FD
:10B9400008950E940D720E946072E03021F008326A
:10B95000E0E01E070CF007C00E946072EA93DADF95
:10B960000F5F1F4FF0CF1981088161C00E940D72D7
:10B97000F801AB81BC810E94677231F0EA81D80185
:10B98000F0E0AE17BF070CF009C0F801AB81BC8135
:10B990000E946C72BFDF0F5F1F4FEACF19810881D1
:10B9A000ABC00E947C760E944972EFE9F0E0EA1B8E
:10B9B000FB0B31978F010E9471720E943F720E94AF
:10B9C0001C660E94837633C00E947C76AC810E9404
:10B9D00079720E2F11270E9471720E943F720E948D
:10B9E0001C660E94837688C0EA81FB810E94D27027
:10B9F000E881F981E0935A05F0935B05AA81BB8148
:10BA0000ECE0F0E00E94F4730E945B72A881B981BF
:10BA1000E4E1F0E00E94F47306C0EA81FB810E9439
:10BA20005B72E881F981E093F50BF093F60B2496B5
:10BA300008950E948172143128F41A930E94C74518
:10BA40001F5FF9CF0E940D660E940D660E9412666C
:10BA5000EFE7F0E00E94A86710E0153048F4A5E198
:10BA60001A9FF001E551FB4FA0E0A0831F5FF5CFC7
:10BA700010E0143148F4ABE01A9FF001E15FFB4F96
:10BA8000A0E0A0831F5FF5CFE0910504EF7EE09377
:10BA900005040C9490600E9481721431E0F40E94BD
:10BAA0008972DF01EB81FC81AE17BF0774F00E9441
:10BAB0008972DF010E94636E44F0ADE01A9FF001CD
:10BAC000E55FFC4FE081E03009F403C01A930E9467
:10BAD000C7451F5FE2CF0E940D66ED81FE81FA939C
:10BAE000EA930E941266A985BA85EF81F885EA1B60
:10BAF000FB0B0E94A867188125960895A2970E94C3
:10BB00007A76E9A5ADE0EA9FF001E050FD4F8F01A4
:10BB1000D8011B96EC91E03009F403C2D8011B96C2
:10BB2000EC91E9A3E07859F0FE013696FA93EA9396
:10BB3000EBA10E946770FA93EA930E94DF62E9A189
:10BB4000E07459F0FE013696FA93EA93EBA10E9455
:10BB50006E70FA93EA930E94DF62FE013696FA93C2
:10BB6000EA930E94F562E8A3E0910804EB8FE0916C
:10BB70000904EA8F0E947766D80111962D913C91B5
:10BB8000D80113964D915C91D80115960E94987436
:10BB9000EEA3FFA3D8011796EC91F0E0ECA3FDA370
:10BBA000D8011896EC91EC8FE0910904A0E10E9475
:10BBB0002066EAA3FBA30E942F720E949F700E943E
:10BBC0009F70ECA1EA930E949A48D8011996EC91D3
:10BBD000EC8FAC8DAF3011F4E8E0EC8F0E942F7247
:10BBE0000E948E720E943A710E9493720E94977214
:10BBF0000E949E720E94A1720E942F723A932A9311
:10BC0000EAA5FBA5E40FF51F0E94AA72EEA1FFA111
:10BC1000E20FF31F0E943A710E948E720E94A1727D
:10BC2000A8A5A130A1F43A932A93FA0131960E9473
:10BC30009E72FA93EA93FA0131960E94AA72F90170
:10BC400031960E943A71F90131960E94A172A8A51D
:10BC5000A230D1F40E94977231970E949E72FA939B
:10BC6000EA93EAA5FBA5E40FF51F31970E94AA729B
:10BC7000EEA1FFA1E20FF31F31970E943A710E94DB
:10BC80008E7231970E94A172E8A5E03011F40C94F5
:10BC9000615FD8011996EC91EC8FE0910804ACE05B
:10BCA0000E94AD720E941F74ED8FA8A1EA1710F4D4
:10BCB0000C949F5EE1E0E0930904E03021F0ECA1F8
:10BCC000FDA1B5970CF402C00E94B372AAA1BBA15A
:10BCD000ECA1FDA1EA1BFB0BDF010E949669EAA320
:10BCE000FBA3ABA1AA231AF4E0E0EAA3EBA3A8A16B
:10BCF0000E947972AEA1BFA1F0E00E94BB72EE8FEC
:10BD0000A8A5A13021F40E94BF720E94C472A8A508
:10BD1000A23021F40E94BF720E94CE72E0E0E9A33B
:10BD20000E94D672AE0FBF1FEC91E03039F00E9436
:10BD3000D6720E946C720E94DB72F2CFC2C0E1E048
:10BD4000E0930904E03031F0ECA1FDA1E734A0E07C
:10BD5000FA070CF402C00E94B372E8A1EF8FEAA1C7
:10BD6000FBA1EE0FFF1FACA1BDA1AE1BBF0BE3E01B
:10BD7000F0E00E941F74EAA3FBA3ABA1AA2322F464
:10BD8000E1E0F0E0EAA3FBA3EF8DE150EF8FEF8D50
:10BD9000F0E0DE011696AE0FBF1FAC91A03219F095
:10BDA000AF8DA13008F404C0EF8DE150EF8FEFCFDD
:10BDB000AF8D0E947972AE2FEEA1FFA1B0E0EA171D
:10BDC000FB0714F3EF8DE03011F4ED8DEF8FAF8DA5
:10BDD000ECE00E94AD720E94BB72EE8FA8A5A1306C
:10BDE00021F40E94BF720E94C472A8A5A23021F45F
:10BDF0000E94BF720E94CE72E0E0E9A30E94D67258
:10BE00000E94677221F0EF8DA9A1AE1708F007C05C
:10BE10000E94D6720E946C720E94DB72EFCFAF8DCF
:10BE2000E8A1EA1BAE2FED8DEA1768F0AF8DE8A10F
:10BE3000EA1BACE0EA9FF001A09108040E94AD72F9
:10BE40000E94BB7201C0E0E0EE8FA8A5A13069F4AA
:10BE50000E94BF7231960E944472AFE00E94206639
:10BE60000E94E37231960E944C68A8A5A23059F452
:10BE70000E94BF720E944472AFE00E9420660E943E
:10BE8000E3720E944C680E94D672AE0FBF1FAC9145
:10BE9000A03219F4E9A1EF5FE9A30E94D6720E94D3
:10BEA000677239F0AF8DE9A1EA1BAE2FED8DEA176D
:10BEB00008F407C00E94D6720E946C720E94DB7266
:10BEC000ECCFD8011C96EC91E03029F10E94776606
:10BED0000E942F72A2DDF801A485A43698F4E0E058
:10BEE000E0930B04F801A485AA3028F0A485AA9356
:10BEF0000E94D94306C0D8011C96EC91E05DEA93FC
:10BF000009DD09C0ECE0E0930B04E2E5EA9302DD11
:10BF1000EDE4EA93FFDCEB8DE0930804EA8DE09317
:10BF200009040E948176AA9608951A9310E0E89475
:10BF300027F8143170F40E947368E03011F00E9409
:10BF400080681F5FA895E12FE37011F40E94C61569
:10BF5000F0CFE0E0E0930B040E94C615E1C01A9315
:10BF600010E01431D0F40E947368E03081F00E9438
:10BF70008972DF01EB81FC81EA17FB0744F40E9420
:10BF80008972DF01E981FA81AE17BF070CF002C0A8
:10BF90000E9480681F5FA895E4CFE0E0E0930B0467
:10BFA00018810C94CB621A9310E0143190F40E9423
:10BFB0007368E03029F00E947A68E081E17009F44A
:10BFC00006C01A93E0910504E170EA9397DD1F5FC4
:10BFD000ECCFA6C02C970E947A76AD89BE890E94CC
:10BFE0009669ED8BFE8BAB89BC890E949669EB8BC1
:10BFF000FC8BED89FE89A98DBA8DEA0FFB1FE98FB5
:10C00000FA8FEB89FC89AF89B88DEA0FFB1FEF8BA4
:10C01000F88FED89FE89AD89BE890E94EA72EE87AC
:10C02000FF87688B798BEB89FC89AB89BC890E947F
:10C03000EA720E94F1720E942776EA87FB876C877A
:10C040007D8700E010E0EB89FC89E017F10714F42C
:10C050000C946B60F8010E94B6730E9451750E94A7
:10C06000F672AE81BF81888599850E94D975AA85AF
:10C07000BB858C859D850E94D9750E94F1720E94B6
:10C08000FB720E941A75AF015A934A930E94486549
:10C090002E2F33270E940073E98DFA8DE01BF10BE0
:10C0A0000E940773ED8DFE8DE01BF10B0E94117352
:10C0B0000E940073F801A98DBA8DEA0FFB1F0E9440
:10C0C0000773F801AD8DBE8DEA0FFB1F0E9411733F
:10C0D0000F5F1F4FB8CF0E9481766B960895E0E006
:10C0E0000E94E365E1B3E360E1BB8BE18A95F1F780
:10C0F000E1B3EC7FE1BBE4E4E09374000E94F565FA
:10C1000008951A9314EAE4EA0E94177341F40E9416
:10C110001C73183011F0103111F4E0E001C0E2E0BE
:10C1200019910895E4E9E0937400E0E008951A930A
:10C13000E981E1600E94217331F40E941C73103484
:10C1400011F4E0E04EC04CC01A93E9810E942173C3
:10C1500031F40E941C73183111F4E0E042C040C079
:10C160001A93E9810E94217331F40E941C731832E2
:10C1700011F4E0E036C034C01A93E981E03011F0E8
:10C18000E4EC01C0E4E80E94177379F40E941C7388
:10C19000E0917300AA81BB81EC93103511F0183542
:10C1A00021F4E0E018810C94B365E1E018810C946F
:10C1B000B3651A93E981E093740010E0E091740094
:10C1C000E07811F4163908F005C08DE08A95F1F792
:10C1D0001F5FF4CFE0917400E07811F0E0E001C05F
:10C1E000E1E01881229608950E947C763D810C81C1
:10C1F00020E087DFE03011F5EE810E94326DF1F42E
:10C200003A93AEDFE030D1F40E942573B9F479DFC0
:10C21000E030A1F4EE810E94EC6581F4EDB7FEB749
:10C22000FA93EA931F930E94F1651F91E03031F475
:10C2300079DFE12F0E9483760C945D6350DFD9CFC4
:10C240000E947C7630E00E811D815BDFE03099F446
:10C25000EF810E94326D79F40E94257361F41A9384
:10C260007FDFE03041F4EC81EA937ADFE03019F4CB
:10C2700059DFE0E002C033DFE8CF0E9483762896E2
:10C28000089522970E947A7650E02B853A85A895EA
:10C2900038DFE03011F00C94A361EE850E94326D1E
:10C2A00011F00C94A3612A935BDFE03011F00C9441
:10C2B000A3613A9355DFE03011F00C94A36121DFC4
:10C2C000E03011F00C94A361EE850E94EC65D9F585
:10C2D000E0E0EE83EF83EC85FD8531970E94BC7032
:10C2E00049F4EDB7FEB7FA93EA931F930E94F16504
:10C2F0001F9109C0EDB7FEB7FA93EA931F93E1E0EF
:10C30000EA933ADF1F910E2FEE81FF81A885B98550
:10C31000EA0FFB1F1083EE81FF813196EE83FF83CE
:10C32000003039F4EC85FD85AE81BF81AE17BF07C3
:10C3300008F001C0D0CFEC85FD850E94BC7019F4D7
:10C34000F1DEE0E002C0CBDEA3CF0E9481762F9623
:10C35000089568970E947A7620E0E0E0EC8FED8FF8
:10C3600031E0A895E9A1FAA1662777270E945175C7
:10C37000EA87FB876C877D87EE8D0E942A730E9477
:10C38000F672AA85BB858C859D850E942776EA8BEF
:10C39000FB8B6C8B7D8B0E94AB74FE017296FA93C3
:10C3A000EA930E94B565EE8BFF8B688F798F0E94B0
:10C3B00030730E941875AF010E943073AE8DBB2799
:10C3C000882799270E94B2740E94FB72DE015A9658
:10C3D0000E941875ED93FC930AA119A192DEE0303A
:10C3E000D1F5EDA10E94326DB1F50E94257399F54A
:10C3F0001A93B6DEE03079F5303051F14F5F5F4F80
:10C40000EC8DFD8D3196EC8FFD8FAC8DBD8D119730
:10C41000EBA1FCA1EA17FB0711F430E018C0EC8D8A
:10C42000FD8D3197AF8DB8A10E946C7299DEEE8DB3
:10C43000DA01F0E0EA17FB0751F474DEEA8DFB8DB8
:10C44000A9A1BAA1EA0FFB1FE9A3FAA38BCFD4CF0E
:10C4500069DEE0E002C043DEC1CF0E948176A6968D
:10C460000895A881A03310F0AA3308F004C0E88131
:10C47000E0530C943663A881A13410F0A73408F07F
:10C4800004C0E881E7530C943663EFEF0C943663F5
:10C49000A881AA3020F4E881E05D0C943663A8817D
:10C4A000AA3020F0E881E95C0C943663E8E50C944E
:10C4B00036631A930A93F8940091190B10911A0B92
:10C4C0007894F8010991199108951A930A93F1DF6C
:10C4D0008F01EA81FB810E94596EE01BF10BDF01A5
:10C4E0000E9470762CF4E0E0198108810C94E165DB
:10C4F000E1E0198108810C94E1650E94FF650E94CA
:10C500000D660E94F45C0E941568ECEBFBE10E9452
:10C5100009660E9477660895E4E7F6E1FA93EA93E4
:10C52000EAE6F0E0FA93EA930E942F68E4E0EA93E7
:10C53000E6E2EA93EEE0EA930E94044AECE0F7E1D7
:10C540000E946966E3E5F0E0FA93EA93E8E0EA9393
:10C55000E2E3EA93E1E0EA930E94044A08959981B4
:10C560008881009641F0BD81AC81FB81EA81059014
:10C570000D920197E1F7FD81EC810C94E165B981A1
:10C58000A881109631F0FC81EB816A81619311974B
:10C59000E9F7EB81FC8125960895E991F991A9913C
:10C5A000B9911D900590011421F40020D1F7EE27D8
:10C5B00008951018E1F3E1E008F4E2500895E991DC
:10C5C000F991A991B991CD0161916D936623E1F73C
:10C5D000FC010895E991F991A991B991CD010590D6
:10C5E0000D920020E1F7FC010895A991B991EE2781
:10C5F000FF276D91662311F03196FBCF0895AA278E
:10C60000BB27E991F9910590002011F01196FBCF1D
:10C61000FD0108957991E991F991A991B991CD011F
:10C62000772351F07A9561916D936623C9F777234B
:10C6300019F07A956D93FBCFFC0108956991E9910A
:10C64000F991A991B991CD01662351F06A950590B0
:10C650000D920020C9F7662319F06A950D92FBCF61
:10C66000FC0108955D9BFECFE881ECB92196089509
:10C670001A930A93AC81BD810E9498743097C1F0DF
:10C68000AA81BB810E9498748F01309749F00230D3
:10C69000E0E01E0760F0F80131978F01ED93FC9305
:10C6A000AC81BD810E9468683197AE81A08303C0D0
:10C6B000EE81EA93D7DF19810881279608952C9798
:10C6C0000E947A7610E0E88DF98D3196E88FF98F27
:10C6D0003197E4912E2FE03011F40C941B65E12F7B
:10C6E000E03039F4253211F411E002C00E943C73AD
:10C6F000A1C1E130C1F4253219F40E943C7399C103
:10C7000012E0E0E0E98B00E02D3211F401E092C18B
:10C710002B3219F4EBE2E98B8DC1203219F4E0E2FF
:10C72000E98B88C102C0E23039F450E013E02033D5
:10C7300011F400687FC102C0E330A1F4203310F08F
:10C740002A3308F009C0A52FEAE0EA9FF0015E2F26
:10C75000E22FE0535E0F6EC140E02E3211F414E080
:10C7600069C110C0E430A1F4203310F02A3308F07E
:10C7700009C0A42FEAE0EA9FF0014E2FE22FE05318
:10C780004E0F58C12C3619F4026015E053C104C095
:10C79000E53011F00C941A65E22FE33649F40E945B
:10C7A0004773EE89FF89A481AA930E944D7341C10A
:10C7B000E33741F40E9447730E9457730E94F56269
:10C7C0001E2F0AC0E037A1F40E9447730E945773DE
:10C7D0000E94FF621E2F08600F77403011F0411752
:10C7E00008F001C0142F40E0E0E0E88B30E078C0B2
:10C7F000E43611F0E93611F4046002C0E537A1F423
:10C80000EAE0E88B01FF08C0E0E0FAEC6AE97BE3CC
:10C810000E94E3671AE023C0E0E1F7E260E070E025
:10C820000E94E36715E01BC0E83511F4086004C0FE
:10C83000E83711F00C941965E0E1E88B01FF08C0BE
:10C84000E0E0F0E060E070E10E94E36718E007C01C
:10C85000E0E0F0E160E070E00E94E36714E0403067
:10C8600011F00F7701C041E001FF08C00E9447733B
:10C87000AE89BF8914960E949C7415C002FF0AC03D
:10C880000E944773AE89BF8914960E9498740E94D3
:10C89000B67309C00E944773AE89BF8914960E947F
:10C8A000987466277727EC87FD876E877F8702FF5E
:10C8B00016C0AF85AA2362F4EC85FD856E857F8561
:10C8C0000E949273EC87FD876E877F87EDE2E98B8C
:10C8D000E989E03019F01F5F4F5F01C00B7F342FF3
:10C8E00000FD14C0151710F4351708F00FC007FF2E
:10C8F00008C002FF04C00B7F2989115001C020E34A
:10C9000001C020E20E943C735150ECCF1417B0F4E8
:10C91000006102FF0AC00B7FE989EA930E944D7310
:10C92000503009F0515011504150E0E3EA930E9419
:10C930004D73503009F051504150E8CF312FE88904
:10C94000E030D1F43030B9F003FF08C0EE81FF8150
:10C950003196EE83FF833197E49105C0AE81BF81AC
:10C96000ED91AE83BF83EA930E944D73503009F07E
:10C9700051503150E7CF53C00E945F730E9424741E
:10C980002E2F2A3030F003FF02C0295C01C0295A43
:10C9900001C0205D04FD23C0213350F40E94E867EC
:10C9A000A130E0E0BE07E0E08E07E0E09E0709F47A
:10C9B0000BC0431740F4531710F000FF01C014C020
:10C9C00020E207FF0CC020E3006102FF08C00B7FDC
:10C9D000E989EA930E944D73503009F051500E944A
:10C9E0003C73503009F0515031500E945F730E94E7
:10C9F0005F74EC87FD876E877F87E8890E94E86710
:10CA0000FF27662777270E9424740E94E367E88542
:10CA1000F9856A857B850E946C7609F0ADCF00FFB1
:10CA200008C0503031F05150E0E2EA930E944D735B
:10CA3000F8CF10E048CE0E9481766A960895FF9262
:10CA4000F82E22971A930A93DE010E9485738D01B6
:10CA5000DE0116960E9485730E949874EA83FB8318
:10CA6000DE0114960E9485730E949874FA93EA93EB
:10CA70001A930A93FE0136960E94706620DEAA8100
:10CA8000BB81E0E0EC93198108812496FF90089522
:10CA9000A991B991EE27002460E8E894162E169427
:10CAA00007941E2A1EF0A015B10518F0A019B109AF
:10CAB000E62BB7FBAA0FBB1F669580F708957B8115
:10CAC0006A81F981E88177FB770F67FD7160972FA5
:10CAD0009E5781F078F0983190F4AA27BB278827D9
:10CAE00008948795B795A7959A95D1F7EA23FB23E4
:10CAF000682305C0E8947727EE27FF2766276F771E
:10CB0000769508F4606877F9A991B991899199911E
:10CB1000EA17FB076807790797FB08950E942872B8
:10CB20000E94687319F40E946F731DC0E6F7A88114
:10CB3000B9818A819B81E0E0F0E060E87FE30E94B8
:10CB4000FB7211C00E9428720E94687319F40E943F
:10CB50006F7309C0E6F30E946F73A0E0B0E080E855
:10CB60009FE30E948B75249608950E9474730E941F
:10CB70006C7639F4A881B9810E94666C0E94A27417
:10CB800020C0AA81BB818C819D810E94747634F47F
:10CB90000E9474730E94AB74C1DF05C00E9474735D
:10CBA0000E94AB74CFDFA881B9810E94A274A881D2
:10CBB000B9810E949C74AA81BB818C819D810E9455
:10CBC000FB7226960895E0937100E0E0E093740014
:10CBD000E2B3E360E2BB0895EA930E949760E0301D
:10CBE0000895E0E0EA930C94BC6088EC90E0019733
:10CBF000F1F70895E4E6F0E0FA93EA930895E1E0AE
:10CC0000F0E0FA93EA930895E4E0F0E0FA93EA930F
:10CC10000895FA93EA930C94A15CE0E0F0E0FA93B3
:10CC2000EA930895EFE9F0E0FA93EA930895E0E2D9
:10CC3000F0E0FA93EA930895EFE0EA930C949A48AF
:10CC4000EA9FF001F0E008950E941A110C948945C2
:10CC5000E0E0E0930A04E0930B040895A8E0B0E05C
:10CC60000E94C674E0300895EBE9F0E0FA93EA938D
:10CC70000895E4E1F0E0FA93EA93EEE1F0E0FA934C
:10CC8000EA9308950E942F46EFCFEDE2EA93C5CFD5
:10CC9000E0E4F0E0FA93EA93ECCFEBE2EA93BDCF65
:10CCA000E1EFFFEFFA93EA9308950E942F46F8CF41
:10CCB000E0E6F0E0FA93EA93DCCFEDE4EA93ADCF5F
:10CCC000A5E01A9FF001E45CFD4F0895A12FB0E0AC
:10CCD0000895FA93EA93EAE5F0E0FA93EA93089567
:10CCE000FA93EA939ACF0E94C10E0C94955FE1E00B
:10CCF000E0930804E09309040895E0930A04E0E057
:10CD0000E0930B040895FA93EA93EEE1F0E0FA93CE
:10CD1000EA930895E32FF0E00895A091F10BB0910C
:10CD2000F20BBD01A3E0B0E00E94CC73E60FF71F49
:10CD3000E491E0300895A091BB05E3E0EA9FF001A3
:10CD4000EF5F0E2F0895E02FF0E00895E6E9F0E0A0
:10CD5000FA93EA930895FA93EA93F5CFA091F10B31
:10CD6000B091F20BBD01A3E0B0E00E94CC73E60FDE
:10CD7000F71F0895ABE03A9FF001E45BFD4F089583
:10CD8000FA93EA930C942F46E091780BA0EA0E9464
:10CD9000FE732E2FE091790BA0E80E94FE735E2FA8
:10CDA00008953A930E94B130A091410BAD3208959D
:10CDB000E0914F0BE295EF70E0930A04E0914F0B86
:10CDC000EF70E0930B040895A02FBB27E22FF0E053
:10CDD0000E94F4733396FA93EA930895ED5FF0E0BE
:10CDE000FA93EA930895E22FE450F0E0FA93EA937D
:10CDF000E52FE450F0E0FA93EA93E32FE058EA934A
:10CE00000CCFE0E0EC93AE81BF810895E1E0E093C8
:10CE10000804E2E0E09309040895E52FF0E00895A6
:10CE2000EA1BA9E0B7E0F0E00E94A6730895A0E035
:10CE300021FCA1E0A1300895E1E6F0E0FA93EA9345
:10CE4000EAE4F0E0FA93EA93ECE1F0E0FA93EA9393
:10CE50000895E981F0E00895EE0FFF1FEA5CFD4FB1
:10CE60000E94A7740895A4E3B2E0F0E0EE0FFF1F64
:10CE7000EA0FFB1F0E94A7740895DB01AE1BBF0BD6
:10CE8000E2E0F0E00E94BB74EA1B0895FA93EA9393
:10CE9000E4E1F0E0FA93EA930895E12FF0E00895D9
:10CEA000E3E0F0E0FA93EA9308950E94A774FA93FE
:10CEB000EA930895EA81F0E00895EC81F0E00895A6
:10CEC000ABE0EA9FF001E752FA4F0895FA93EA9334
:10CED000E4CFE150ADE0EA9FF0010895ED5FFC4F33
:10CEE000DF010E9498740895FA93EA930E94F45C1B
:10CEF0000C94D15CEA930E94B130E1E4FBE0FA9338
:10CF0000EA93EAE0EA930E94B65C87CEE12FEF5FF6
:10CF1000F0E00895E6E0F0E0FA93EA93F7CFFA93B1
:10CF2000EA930C94F45CEE0FFF1FAE0FBF1F0E943C
:10CF300098740895FA93EA930C94BB430E94B673D5
:10CF40000E94AB740895E4E1F0E0FA93EA93089547
:10CF5000FA93EA9371CEF0E0EDCFE2E0F0E0DFCFBC
:10CF6000E0916805F09169050895E0916405F091FC
:10CF700065050895AE0FBF1FE3E0F0E00E941F7447
:10CF80000895FA93EA931A930A930C94DF12FA9392
:10CF9000EA933A932A930C94DF12A0916C05B09116
:10CFA0006D050895A0916E05B0916F050895A0E0FC
:10CFB000B0E00E94C27408950E94BB74EA1BFB0B90
:10CFC0000E94B6730895E887F9876A877B8708957A
:10CFD000A885B9858A859B850895A2E0B0E00E9466
:10CFE000C27408950E94B6730E9449740895A4E023
:10CFF000B0E00E94C2740895EC83FD836E837F834A
:10D00000AC81BD818E819F810895A6E0B0E00E9431
:10D01000C2740895E0E9F1E0FA93EA930C9479730D
:10D02000E6E3F0E0FA93EA930895E2E0E09308047F
:10D03000E09309040895EA930E948A5C58CEEAE0DE
:10D04000EA930E944043E0916C05F0916D050895CC
:10D05000E8E1F0E0FA93EA93E8E2F0E079CFE6E481
:10D06000F0E0FA93EA930895E8E8F0E0FA93EA939F
:10D07000D7CFEAE0EA930E944043E0916E05F09139
:10D080006F050895E8E2F0E0FA93EA930895E2E389
:10D09000F0E0FA93EA930895FA93EA930C940D5D05
:10D0A000FA93EA93A7CDE8ECF0E0FA93EA930C94B4
:10D0B00079730A921A92FA926A937A938A939A935C
:10D0C000AA93BA93EA93FA93EFB7EA931A9308955F
:10D0D000ED91FD913196FE93EE930895E4EFF1E02A
:10D0E000FA93EA930895ADE01A9FF001E050FD4FE6
:10D0F000E0810895ADE01A9FF001E65FFC4F0895CE
:10D100001A93E1E0EA930C947E5DE2E0EA930C94DA
:10D110007E5DE091E007F091E1076091E207709198
:10D12000E3070E94AB740895E091D807E150AAE5A7
:10D13000B6E0F0E00E94A673AE0FBF1F0E949C7481
:10D140000895EAE6FBE0FA93EA930895EAE0EA93A9
:10D150000C94B65CE091D907EA93E091D507EA9385
:10D160000E94FC32A091D50BB091D60B1097089578
:10D17000A091D70BB091D80B8091D90B9091DA0B7D
:10D180000E9474760895E091D50BF091D60B089526
:10D19000E0E2EA930C948A5CE091D70BF091D80B13
:10D1A0006091D90B7091DA0B0E94AB740895E091F5
:10D1B000D507EF5FE093D5070895EF5F0E94DA741B
:10D1C000E150EAE0F0E0FA93EA930C947973E0918D
:10D1D000C907ABE0EA9FF0010895A083E9ECF7E00E
:10D1E000FA93EA930C945D2CE5E0F0E098CEE1E050
:10D1F000EA930E947E0E4BCF0E947973E0E0EA939F
:10D200000C947E0EFA93EA930C947973A9E0B0E043
:10D210000E94C6740895E091040CEF5FE093040C43
:10D220000895E1E0EA930E947E0E90CDAEE0B0E07A
:10D230000E94C6740895E0E0E0930B0CE0930A0CA2
:10D240000895E0E0F0E0ED93FC930895EA81D801C1
:10D25000EC93E9ECF7E0FA93EA930E945D2C1981D4
:10D2600008810895E12FACE8B0E0F0E0EE0FFF1F79
:10D27000EA0FFB1F0E94A7740895A3E21A9FF00112
:10D28000E65AF94F0895A3E21A9FF001E45AF94FC4
:10D29000E0810895E981ADE0EA9FF0010895E65F3D
:10D2A000FC4FA1E0A0830895ACE8B0E0F0E0EE0F01
:10D2B000FF1FEA0FFB1F0E94A7740895A091CD07DE
:10D2C000B091CE07EA2BFB2BE093CD07F093CE076E
:10D2D0000895E150A7E1EA9FF0010895A7E10A9FB0
:10D2E000F001EC5EF94FAF010895FA93EA93E0E0A4
:10D2F000EA930895F0E0A4E6B0E00E94F473089584
:10D30000E091630BF091640B0895EAE5F6E0EDCF50
:10D31000FA93EA930C94BF62E881F0E0E65AF94F81
:10D320000895E981FA81FA93EA930895E2E0F0E042
:10D330000E941F740895A1E5BBE0E091D107F0E0E1
:10D340000895A4E5BBE0E091D107F0E0AE0FBF1F68
:10D350000895A7E5BBE0E091D107F0E0AE0FBF1F55
:10D360000895EE0FFF1FAE0FBF1F0895ADEFB6E09B
:10D3700054CDEE0FFF1FEA0FFB1F0895A7E11A9F80
:10D38000F001EC5EF94FEE83FF83AE81BF8108951B
:10D39000EE81FF81A481AA930C94FD190D901C903D
:10D3A000AE81BF811296EC91F0E0E00DF11DDB0142
:10D3B000ED93FC930895ED91FD913197FE93EE93DB
:10D3C00008950E949C1BEF770E2EAA85BB851296AE
:10D3D000EC91E0150895A3E20A9FF001E15AF94F9C
:10D3E0000895BD01AAE0B0E00E94CC73E60FF71FDC
:10D3F000E887F987A1810895E057F84FEC87FD870A
:10D40000AC85BD85119608951296EC91AC85BD85CD
:10D410001696EC930895D001F0E00895A885B9859B
:10D4200018960E9498740895AC85BD85EC93E9EC3C
:10D43000F7E0FA93EA930C945D2CE885F985A281D4
:10D44000AA930895EA85FB85FA93EA930E94DE1970
:10D45000E0300895AA85BB85EC91EA93E3E0EA9376
:10D460000C947345AA85BB85E0E0EC93E2E0E09381
:10D4700009060895BF0100801180AE81BF81129618
:10D48000EC9108950E94BB74EA1BFB0B0895DB012D
:10D49000ED93FC93AE81BF811296B3CCE45FFC4F59
:10D4A000E081E058DB01EC930895E4E6F0E00E94AF
:10D4B000F4730895F0E0ED93FC930895E9ECF7E040
:10D4C000FA93EA930C945D2CE091D007A091CF07DA
:10D4D000EA170895F0E0E00DF11D0895A091780B92
:10D4E000E091790BEA9FF0010895AAE5BBE0D5CC65
:10D4F000A4E5BBE0EE27A10FBE1FEC910895A7E5C0
:10D50000BBE0EE27A10FBE1FEC910895BD01AAE07C
:10D51000B0E00E94CC73DB010895E081EA930C94A3
:10D52000AB55E7EFF9E0E093150BF093160B089578
:10D53000EA930E94B1300C94A719BD01AAE0B0E0B3
:10D540000E94CC73E60FF71F0895A4E5BBE0EE2719
:10D55000A00FBE1FEC910895A7E5BBE0EE27A00F3A
:10D56000BE1FEC910895A1E5BBE0EE27A00FBE1F02
:10D57000EC91E1700895AAE5BBE0E5CBE150F0E065
:10D580000895A7E6BBE0EE27A00FBE1FEC9108951B
:10D59000A0E6BBE0EE27A00FBE1FEC910895EA8144
:10D5A000ADE0EA9FF001E65FFC4FA0E0A083EA81D6
:10D5B000EA930895ABE00A9FF001E952FA4F08950B
:10D5C0001A930E943D36A091E30BB091E40B0E94A8
:10D5D00070760895ABE00A9FF001E352FA4F089588
:10D5E000A091E30BB091E40B0895FA93EA930C94A5
:10D5F000D72DFA93EA930E94EF453A9386CDE091B6
:10D60000E30BF091E40B30970895AFEFBFEFA083E9
:10D61000B1830895E0E0F0E0E093E30BF093E40BD6
:10D62000E093E00B08950E945962E093100CF09390
:10D63000110C0895F0E073CCFA93EA9387CDFA9336
:10D64000EA93E0E0F0E80895E091E10BF091E20B5D
:10D650000895E0914C0BF0914D0B0895E093E10B90
:10D66000F093E20B0895FA93EA930C945430E05748
:10D67000F84FFA93EA930E94F12220CFE091C70776
:10D68000ABE0EA9FF0010895E7ECF7E0FA93EA9344
:10D690000C945D2CE093E30BF093E40B0895E88D7C
:10D6A000ABE0EA9FF00108950E94195DE0E0EA9383
:10D6B0000C94C10FE0E0F0E0E093DC07F093DD07AD
:10D6C000E1E0E09309040895E0910E04E550F0E0F4
:10D6D00007CBE091DC07F091DD072CCCE0915805F9
:10D6E000F091590531970895FA93EA930C94E65B0B
:10D6F0000E94F45C0C94D15CEF5CEA930C948A5C1D
:10D70000ADEBB6E007CBAAE5BBE0E091D107F0E0D6
:10D7100030CEADEFB6E0FECAAE0FBF1FEC91E160B8
:10D72000D001EC930895E7E0E093CF07EA93E0E0BF
:10D73000EA9373CAEA930E9440430E9489451E2FD0
:10D740000895EAE2EA93EBECF9E1CFCD0E94CE2412
:10D75000E1E0EA930C94B6241F771A930C94B1304D
:10D76000A091DC07B091DD070895E053F0E0089543
:10D77000A0E024FCA1E0A0300895E0E0EA934DCAC7
:10D780000E945962E093EA07F093EB070895E09155
:10D79000DE07F091DF07FA93EA930C944C1BFA939F
:10D7A000EA930C946562E0E0E0930A0C0895D8DFF8
:10D7B000EA17FB070895FA93EA930E94751BE0307D
:10D7C0000895E093DE07F093DF070895E093CF0715
:10D7D000E0E0E093E70708950E94165A0E943E2673
:10D7E000E093DB0708950E94B1300C94195DE1E4E9
:10D7F000FBE022CFE091D007EA93E0E0EA930E94B9
:10D80000E3250C94A3220E9489451E2F1A930E949F
:10D810007126103808951A93E091C105EA9308958E
:10D82000E091DE07F091DF07C6CFE091400BEA936D
:10D830000E94BC2FE03008950E945962E093120CC0
:10D84000F093130C0895D90118960E9498740895C6
:10D85000E4E6F0E060E070E00E94497408950E9400
:10D86000B130F7CE0A93E091C105EA930895E091B3
:10D87000E607EA930A930C940D32ABE03A9FF0016D
:10D88000EF51FA4FE0810895ABE03A9FF001E15289
:10D89000FA4FDF010E9498740895FA93EA93E8EE34
:10D8A000F3E07DCFE093170BF093180B0895A09150
:10D8B000170BB091180BAC910895A7E1BBE008CC11
:10D8C000E091F307E053E093D9070895E0E0F0E03A
:10D8D00060E070E00895FA93EA93E0E3EA930C9431
:10D8E000165AE12FAAE5B6E0F0E00E94A67308956B
:10D8F000AE0FBF1F0E949C740895E091F007EA9359
:10D900000C94B759FA93EA930C9405590E946E59F6
:10D91000EBE3EA930C94F558E1E4FBE0FA93EA9325
:10D920000895E89423F8E0E0F0E04BDFE0E0E093D6
:10D93000D5070A93E1E0EA930C94E325E89423F8F1
:10D94000E0E0F0E03EDFE0E0E093D507EA930C94FE
:10D95000B624A881B981EC91EF5FEC930895ABE018
:10D960001A9FF001EF56F84FE0810895ABE00A9F4F
:10D97000F001E852FA4F0895A083ABE00A9FF0014E
:10D980000895EA930E943D360E94DD35E030089507
:10D99000ABE00A9FF001E652FA4F0895FA93EA933A
:10D9A000E2EFF9E1FA93EA93EA85ABE0EA9FF0014E
:10D9B0000895FF27662777270E94AB7484E00E94B2
:10D9C0001F6528960895AC81BD81EE27A00FBE1F6C
:10D9D0000895E02FAC81BD81F0E0EA0FFB1F0895B0
:10D9E00084E00E941F6528960895EE27A30FBE1FAE
:10D9F000EC91D001EC930895A9E0B7E08BC90E94A7
:10DA0000A673EA0FFB1FAF010895E091E30BF091BD
:10DA1000E40B0895E32FA091D507EA0F0895ADE038
:10DA20002A9FF001E85FFC4F0895E0914F0BE295CB
:10DA3000EF700895A8E0B0E00E94C67408951A93AC
:10DA4000E0EAEA9337CAE050F84FFA93EA930E946B
:10DA5000F4601E2F0895E050F84FFA93EA931A935A
:10DA60000C942061EA930E94A460E0300895E0EAFB
:10DA7000EA93EEE5F0E0FA93EA93E0E0FFE0FA9350
:10DA8000EA93E5E7FBE00895FA93EA93E0E2EA938C
:10DA90000C94A961E0EAEA93E981FA81E050FC4F35
:10DAA000FA93EA930895A8E2B0E00E94F47308950F
:10DAB000E0EAEA93E2E0F0E0FA93EA931A930A9339
:10DAC0000895FA93EA930C944161FA93EA930C94C3
:10DAD000F460EDE2EA93EAE0F0E01ACC1A930A93DC
:10DAE000E9C9ABE0B0E00E94F473E050F24F8F015F
:10DAF000AA81AA300895E0EAEA93EBE0F0E0FA9315
:10DB0000EA931A930A93E9E6FBE00895EE0FFF1FEC
:10DB1000E050F04F8F01AA81A03808950E94A673AB
:10DB2000E058F14F8F01AA81A33008950E94F47349
:10DB3000DF01EA85F0E0AE0FBF1FE8E0F0E00E94F1
:10DB4000F473E050F04D8F01E0EAEA93E8E0F0E092
:10DB5000FA93EA931A930A93E3EDFBE0B2CF4E0FE8
:10DB60005F1FE091D70BF091D80B6091D90B7091AA
:10DB7000DA0BAE81BF81888599850E948973EE8317
:10DB8000FF836887798708954093D50B5093D60B10
:10DB9000EE81FF8168857985E093D70BF093D80BF0
:10DBA0006093D90B7093DA0B0895E8E0F0E0FA93F4
:10DBB000EA930895ED81EA93ED81EA930895E09365
:10DBC000DE0BF093DF0B0C945D34E093E007F093F1
:10DBD000E1076093E2077093E3070895E0914E0B2D
:10DBE000AAE5B6E0F0E00E94A6730895E850FA4F67
:10DBF000E081E1300895FA93EA93E091D907E05D7E
:10DC0000EA930895EA930E94375AE1300895E3EFCA
:10DC1000F7E048CE0E94AF62A881AF5FEAE00E94C1
:10DC2000FE73E05D0895A881AF5FEAE00E944E7444
:10DC3000E05D08950E94A473E854FF4F32960E945D
:10DC4000A77408950E94A473E854FF4F0895369670
:10DC5000E491D901EC930895E881F0E0A5E0B0E00B
:10DC60000E94F4730895E0EAEA93E5E0F0E0FA93A5
:10DC7000EA930895EA930E945334FA93EA93EBED02
:10DC8000FBE00895FA93EA93EFEFEA93E5E0F0E022
:10DC90003FCBE093DC0BF093DD0B0895A091E10BFB
:10DCA000B091E20B0895E0E0E093EF0BE093F00B0E
:10DCB0000895AC81BD81EA0FFB1F08951A930E945D
:10DCC000E8341E2F0895E981FA81EA17FB070895C9
:10DCD000EB81EA930E940335FA93EA93E0EEFBE0CE
:10DCE0000895F0E0FA93EA9308950E94F5440C94A5
:10DCF000C244F0E00E94A67308950E94AB740E9493
:10DD0000DF440C94C2440E94F544EBE1FAE1EDCA11
:10DD10000E94C2440C94C24420E030E0E12FE05D58
:10DD2000EA93EEE1FAE167CFEAE0EA930C94CC588B
:10DD3000EBEFFAE0FA93EA930895109158050091F9
:10DD40005A0508950E9489453E2F0C94355CEAE0FF
:10DD5000F0E00E94F4730895DF01EE27A30FBE1FC9
:10DD60000895F0E0EA0FFB1F0895E02FA0E0B2E075
:10DD7000C0CFEA0FFB1F3296E4910895F0E0AE0F9A
:10DD8000BF1FEC91E1700895A1E5BBE096C80E9429
:10DD9000195DE1E0EA930C94C10F0E94C10E0C944E
:10DDA0000D66FA93EA93E091D20BEA930E9406384B
:10DDB000E1320895FA93EA93E3E6EA930E94AC37DE
:10DDC000E1320895E6E0F0E00C947066EA0FFB1F84
:10DDD000FA93EA93E0E1EA930E94AC37E1320895C6
:10DDE0000E94F45CA1E5BBE0EE27A10FBE1FEC9101
:10DDF000E1700895FA93EA93E2E0EA930E9406380C
:10DE0000E13208950E94F45CE12FEF5FEA930E94F3
:10DE1000D943EAE3EA930E948A5CE9CCE7E0F0E0C8
:10DE2000FA93EA930895EF5FEA930C94D943E3E7FA
:10DE3000EA930C948A5CEA23EA930E94DF43A8C920
:10DE4000EAE3EA930C948A5CE8E0F0E00C947066F4
:10DE5000EA930E94AC37E1320895EA930E94DF43CF
:10DE600097C90E94A473EE52FA4F08950E94F45C81
:10DE70000C94A366E6E7F5E0E093F10BF093F20B68
:10DE800008950E947932E0E0E093D8070E944B1693
:10DE90000E94C10EE1E0E093D20708950E94195D4F
:10DEA0000C942466EE81FF81FA93EA930895EAE2E6
:10DEB000EA93E6ECFAE10895EA930E949B160C942B
:10DEC000C10E1A93E091F007E0531E2FE4EFF7E044
:10DED000E9CCE091C907A091CA07EA170895EAECD6
:10DEE000F7E0FA93EA930C945D2CE091CA07ABE05B
:10DEF000EA9FF0010895A0912B0BAF5FEAE00E942A
:10DF00004E74E0932B0BEAE2EA930E94B759E2E5E4
:10DF1000EA930E94F558E0912B0BE05AEA930E9495
:10DF2000F558EEE0EA930C94F558EBE3EA930C9481
:10DF3000F558E4EDFAE1E6CCD9011696EC91D1CE94
:10DF40000E942559F2CFF901A281B381BA93AA9315
:10DF500008950E942559EAE3EA930C94F558119626
:10DF6000E0E0EC930E94D259BACFD901EC91B9CE3E
:10DF7000E05DEA930C94F5580E9425590C94D2590F
:10DF8000EEE0EA930E94F558D4CFE05DEA930E9458
:10DF9000B759E2E5EA930C94F558E45DF44FE0815B
:10DFA000E7CFEAE3EA930E94F558F90108950E9449
:10DFB000D2590E945962E093210CF093220CE2E0C6
:10DFC000E093ED07D9011196EC930E9481760895B4
:10DFD000EA930E94B759E2E5EA930C94F558EEE013
:10DFE000EA930C94F5580E945962E093210CF09347
:10DFF000220CE2E0E093ED07D9011196EC930E9428
:10E0000081760895E091D00BC0CFE091D00BF0E085
:10E01000C4CFE091EE0BA091ED0BEA170895FA93AF
:10E02000EA938ECFE0E2F6E0E093BC05F093BD0505
:10E030000895E093BC05F093BD050895FE01FA93A1
:10E04000EA930895ECE0FBE1FA93EA93EE85FF850D
:10E05000688979890E94AB74C3CCE0E1FBE1FA9353
:10E06000EA93AE85BF8588899989F2CB0E94AB740B
:10E07000AA89BB898C899D89E4E6F0E060E070E0C4
:10E080000E9463740E94AB7488E00E941F652C9606
:10E090000895E9E1FBE1FA93EA93EE85FF850C949C
:10E0A0009E67EE27A10FBE1FEC910895EA930E9490
:10E0B0004A441F5F0895E091BF05A2ECB5E0F0E08F
:10E0C0000895E091BE05A2ECB5E0F0E052C9EF730F
:10E0D000A5E1EA9FF001E551FB4F0895EF73ABE036
:10E0E000EA9FF001E15FFB4F0895AC81BD81EE270F
:10E0F000A30FBE1FAC91A0300895ABE00A9FF001C2
:10E10000E15FFB4F0895EA0FFB1F0F01AC81BD815A
:10E110006CCCA5E10A9FF001E551FB4F0895EE811B
:10E12000FF8101801280AE81BF8115960E94987494
:10E13000D0010895FE013896FA93EA930895EAA56E
:10E14000FBA5FA93EA930895FA93EA93FE013A96AF
:10E15000FA93EA930E94DF6230E0E02F0895E091A5
:10E16000BC05F091BD050895ACEBB5E0ED91FD91D6
:10E170003296FE93EE930895AE81BF81EA17FB07B6
:10E180000895E0E0E0936005E09361050895E7E11C
:10E19000EA93E1E0EA930C940648EA93E7E7EA930E
:10E1A0000C940648E0935805F09359050895A4E5AA
:10E1B000B6E0F0E0DEC8EA93ED85EA930C940648F9
:10E1C000E985FA85AD85BE850895EA930E940648E3
:10E1D000E8E10895EA93E0E0EA930C940648EA93B4
:10E1E000EC85EA930E9406480C942048E881F98166
:10E1F000FA93EA930E942559ECE2EA930C94F558BD
:10E20000A091170BB091180BEC910895A091150BEC
:10E21000B091160BE0E0EC930895EE81FF81E0935E
:10E22000DE0BF093DF0B1093DB0B0E945D34E1E318
:10E23000089541E050E00E943558E887F987EAE305
:10E24000EA930E94A657E13008951A93E985FA856A
:10E25000FA93EA935A934A930895E985FA85FA93D3
:10E26000EA930895E2E2EA930C94A657EAE3EA936C
:10E270000C94A657FA93EA935A934A9308950E94EE
:10E2800035583197E887F987E8850895E091F70ACE
:10E29000F0E0E65AF94F0895E0E0E093260CE093B1
:10E2A000270C08950E9435583197E093F70AE091C2
:10E2B000100BA091F70AEA1708950E944E4EE091C4
:10E2C000F70AEA930895ECE2EA930E94A657E03039
:10E2D0000895E550F54FA0E0A0830895EA930E94C9
:10E2E000A657E1300895E091F80A3BCDE091F80A95
:10E2F000EF5FE093F80A0895AAE5BBE0E091F80A21
:10E30000F0E00C94B969E091F80AF0E00895E0912A
:10E31000F70AF0E097CCE091F70AF0E08BCCFA93A3
:10E32000EA930C942559FA93EA930C94B54A0E9407
:10E330002559ECE2EA930C94F558ECE2EA930C943C
:10E34000F5580E94AA4AE0E0E093F80A0895AE0F5B
:10E35000BF1FEC91C6CCE091170BF091180B0895FC
:10E36000A5E1BBE00C946868A091150BB091160B69
:10E37000EC93F6CFA091170BB091180B0895A091D4
:10E38000150BB091160B13970895E0E0EA930E94E5
:10E390000C4BE093EC070895AA81BB81EC91E295C8
:10E3A000E07FAE2FEC810895EA0FAA81BB81EC9348
:10E3B000D0CAE091C70CA091C60CEA170895E0916D
:10E3C000920DF091930D0895A091900DB091910D43
:10E3D000EA17FB070895E12FA091970DEA0FE0934C
:10E3E000970DE091990D0895F0E0E151F84F1083F9
:10E3F0000895E091990DF0E0E950F74F0895E0910C
:10E400009E0EF0E0E356F24FE081E0939C00E09135
:10E410009E0EEF5FE0939E0E08951A930A9300E01C
:10E4200010E00895EA930E94F5581F5F0895A981AE
:10E43000BA8137CEECEAFBE1FA93EA930895FE0144
:10E440003196FA93EA930895E881EA930C94F5588B
:10E45000E881F9816A817B810E94AB7408953A93C7
:10E460002A935A934A930895E950F64FE081E03099
:10E470000895EA930E944862EA930C94AB551A936C
:10E480000A933A932A930895FA93EA93E091090440
:10E490000895A091F30BB091F40B0895E091F30B64
:10E4A000F091F40BFA93EA93E091F50BF091F60BEF
:10E4B000FA93EA930895E093F30BF093F40B089525
:10E4C000F801AA81BB81EA0FFB1FE4910895AE0F0A
:10E4D000BF1FAC91A0300895AE0FBF1FEC91EA931F
:10E4E0000895A0910904E4E1EA9FF0012E2F33275B
:10E4F000D5CFECE0EA9FF001A0910804EA9FF0017B
:10E5000008951A93E1E0E0930904E093080410E011
:10E510000895ADE01A9FF0010C946E67EAA5FBA583
:10E52000E20FF31F0895ECA1EA930C94FA483A9392
:10E530002A93EEA1FFA1E40FF51F0895FA93EA9341
:10E54000EDCFFA93EA93EAA5FBA5E40FF51FFA9342
:10E55000EA93E9CFFA93EA93E6CFEA9FF001AEA1FE
:10E56000BFA1F0E00895E2E0E0930904E0E2F0E00A
:10E57000EAA3FBA30895AE1BBF0B0C949669EE8D26
:10E58000F0E0E20FF31F08953196FA93EA93ECA1BD
:10E59000FDA1E40FF51F31960C944C68FA93EA93B1
:10E5A000ECA1FDA1E40FF51F0C944C68E9A1F0E08B
:10E5B000DE0116960895ED8DEA930E94425CE9A172
:10E5C000EF5FE9A30895E40FF51FDF01ECA1FDA1C2
:10E5D0000C94B9690E94F4730E94B6730E9451753D
:10E5E0000895AE85BF85888999890895EE83FF8354
:10E5F0006887798708950E94B5740E94847508958C
:10E60000E98DFA8DE21BF30BFA93EA930895FA93DE
:10E61000EA93F901AD8DBE8DEA0FFB1FFA93EA93E1
:10E620000895FA93EA93EA8DEA930C94FA48EA93F0
:10E630000E94D960E0300895E0917100E87F1E2FBC
:10E640000895E0937300E4E8F2CF0A930E94B0606B
:10E65000E0300895FF27662777270E9451750895B7
:10E66000EE8DBFDFF7DF0E94D975A9A1BAA1882777
:10E6700099270E94B274BFCF2A93ED89FE89FA933D
:10E68000EA93FE017596FA93EA930C943863EE8947
:10E69000FF893497EE8BFF8B0895ED89FE89FA93FD
:10E6A000EA93FE017596FA93EA930C943863AE8967
:10E6B000BF8914960E949874EE83FF83F3CBE8859C
:10E6C000F9856A857B85AC85BD858E859F85089596
:10E6D0000E945F65E883F9836A837B830895E881FC
:10E6E000F9816A817B810895EA81FB816C817D815A
:10E6F0000895E991F991309639F080ED97E001970E
:10E70000F1F7A8953197C9F708950024AF0DB01D12
:10E710000895EA0FFB1F681F791F0895F195E19591
:10E72000F0400895F09560957095E195FF4F6F4F1B
:10E730007F4F0895EE230E2EEA2F19F0EE0F0A9464
:10E74000E9F70895EE0FFF1FEE0FFF1FEE0FFF1FFB
:10E75000EE0FFF1F0895EF2FFF27E7FDFFEF08954E
:10E76000FE2FFF0FFF0B6F2F7F2F08956F2F660F68
:10E77000660B762F0895BA2FBB0FBB0B8B2F9B2FE9
:10E7800008958B2F880F880B982F0895EA17FB07A1
:10E79000E1E00CF0EE270895FA9FF02DEB9FF00DCD
:10E7A000EA9FE02DF10D08957A9F702D6B9F700DFB
:10E7B000F89F700DE99F700D6A9F602D710DFB9F92
:10E7C000600D711DE89F600D711D8827FA9FF02D67
:10E7D000610D781FEB9FF00D611D781FEA9FE02D02
:10E7E000F10D681F781F089582D0D6DF0EF496DFF2
:10E7F00008958BD0D9DF0EF495DF0895002498E0BA
:10E80000AA0F001C0E1A10F40E0E01C0A1609A95FA
:10E81000B9F7EA2FA02D08950024112490E1AA0F42
:10E82000BB1F001C111C0E1A1F0A18F40E0E1F1E0F
:10E8300001C0A1609A9599F7FD01D001089557D0C4
:10E84000EBDF0EF46BDF08953F934F935F9300244B
:10E8500011244427552730E2AA0FBB1F881F991F98
:10E86000001C111C441F551F0E1A1F0A460B570B84
:10E8700028F40E0E1F1E461F571F01C0A1603A95B7
:10E8800059F7FD01BC01D001CA015F914F913F9141
:10E8900008953BD0D9DF0EF445DF0895AFDFEA2FAE
:10E8A0000895E894B7FF04C0A095B09511966894B8
:10E8B000F7FD34DFB1DFFD010EF430DF0895C4DF72
:10E8C000FD01BC010895E89497FF09C0A095B0959B
:10E8D00080959095AF5FBF4F8F4F9F4F689477FDA6
:10E8E00021DFB2DFFD01BC010EF41CDF0895E894C6
:10E8F000F7FF02C013DF6894B7FF06C0A095B0957C
:10E90000119600F8039400FA0895E89477FF02C086
:10E9100009DF689497FF0BC00024A095B0958095FF
:10E9200090951196801D901D00F8039400FA0895AB
:10E93000ED91FC9111970895ED91FD916D917C9170
:10E9400013970895ED93FD936D937C93089505902F
:10E95000F491E02D08957A936A93FA93EA930895D7
:10E96000689401C0E89401D09DD0182E862F612DA7
:10E97000192E972F712D1B2EBF2FF12D1A2EAE2F72
:10E98000E12D0895119602D0FE2F1197E199FECF47
:10E99000FF93FFB7F894AEBBBFBBE09AEDB3FFBFE8
:10E9A000FF91089507D01196EF93EF2F03D0EF91C9
:10E9B00011970895E19B02C0A895FCCF9FB7F894EA
:10E9C000AEBBBFBBE09A8DB3E81719F0EDBBE29A7E
:10E9D000E19A9FBF0895552342F4503811F4E0FFA7
:10E9E00004C03196691F791F6BF050E8572711F466
:10E9F0005F93CDC05F3F31F0660F000C5795679570
:10EA0000752F08955F9300200AF0CDC0C6C050E86E
:10EA1000192E1522880F991F9527550F879550E8B5
:10EA2000072E0522660F771F7527550F67950895E6
:10EA3000689401C0E8945F93F2DF703818F07F3F6C
:10EA400008F4A5C056E1571BAAF4519558300EF4AE
:10EA5000593030F0EFEFFFEF6FEF7FE777F91AC033
:10EA600077275523B9F0EE0FFF1F661F771F5A95C2
:10EA7000D1F710C07727583028F0EF2FF62F672FE7
:10EA80005850F9CF552331F076956795F795E7956E
:10EA90005A95D1F700200AF445DE5F9108956894F5
:10EAA00001C0E894309760407040B1F0002426F037
:10EAB000772312F4009436DE172E7EE1112032F017
:10EAC0007A95EE0FFF1F661F111CF9CFEF2FF62F5F
:10EAD000612D5F938ADF5F9108954F93AF01FD0130
:10EAE000DA01AB01BC01CA01402D012C142E4F915B
:10EAF0000895EA0FFB1F681F0895E095F095609553
:10EB0000EF5FFF4F6F4F08955F9381DF903871F192
:10EB100050E8152604C05F937ADF903839F17038D9
:10EB200021F1572F591B13F112F4D7DFFACF5831C7
:10EB300018F0AA27BB278827583028F0AB2FB82F0A
:10EB400088275850F9CF552329F08695B795A79572
:10EB50005A95D9F7502D512562F0CBDF38F46795DF
:10EB6000F795E795739513F41EC0B7DF3EDF5F910D
:10EB70000895EA1BFB0B680B51F010F40094BDDF05
:10EB80006623A2F3EE0FFF1F661F7A95CBF7EE27E1
:10EB9000FF27662777275F910895EFEFFFEF6FE775
:10EBA0007FEF5F910895EFEFFFEF6FE77FE75F91F2
:10EBB00008955F932CDF703851F3903841F30124AE
:10EBC0000894791F23F41CF300203AF3ECCF0F9242
:10EBD0001F932F933F934F93112722279927689FC5
:10EBE000A0018F9F302D410D591F6B9F300D411D8E
:10EBF000591F8E9F27D0BF9F25D06A9F23D0BE9FCD
:10EC00001DD0AF9F1BD0AE9F110D291F391F491F6B
:10EC1000591FE32FF42F652F522F4F913F912F91C2
:10EC20001F910F9066232AF0550FEE1FFF1F661FDE
:10EC300002C073954BF2CFDE5F910895100D211D38
:10EC4000391F02C0200D311D491F591F08955F93C0
:10EC5000DEDE703821F411200AF49FCFA4CF903863
:10EC600009F495CF01240894970B1BF4D4F30020EA
:10EC7000F3CF792F1F932F933F934F931124112795
:10EC8000222733274427552790E2AE17BF07860770
:10EC9000410730F0AE1BBF0B860B410B089401C03F
:10ECA0008894551F221F331F111CAA1FBB1F881FCA
:10ECB000441F9A9551F7F901612D4F913F912F9182
:10ECC0001F91662332F0550FEE1FFF1F661F7A95C6
:10ECD00043F281DE5F91089530976040704008955F
:10ECE00000240A160B06089500240A160B060806CF
:10ECF000090608955A934A933A932A931A930A93CA
:10ED000008955D814C813B812A8119810881089594
:00000001FF
